:020000040802F0
:10000000FFFF0120918B0308597302080174020855
:10001000197402081B7402081D7402080000000015
:10002000000000000000000000000000FDBD02080C
:100030001F74020800000000C5BE020809BF0208C4
:10004000E18B0308E18B0308E18B03089D6A02083A
:10005000E18B0308E18B0308E18B0308E18B0308C4
:10006000E18B0308E18B0308E18B0308E18B0308B4
:10007000E18B0308E18B0308E18B0308E18B0308A4
:10008000E18B0308E18B0308E18B0308E18B030894
:10009000E18B0308E18B0308E18B0308E18B030884
:1000A000E18B0308E18B0308E18B0308E18B030874
:1000B000E18B0308E18B0308E18B0308E18B030864
:1000C000E18B0308E18B0308E18B0308E18B030854
:1000D000E18B0308797102087B7102087F710208C5
:1000E000E18B0308C56A0208E18B0308E18B030872
:1000F000C58F0208E18B0308E18B0308E18B03083D
:10010000E18B030821740208E18B0308E18B0308EB
:10011000E18B0308E18B0308E18B0308E18B030803
:10012000E18B0308E18B0308E18B0308E18B0308F3
:10013000E18B030825740208E18B0308E18B0308B7
:10014000E18B0308E18B0308E18B0308E18B0308D3
:10015000E18B0308E18B0308E18B0308E18B0308C3
:10016000E18B0308E18B0308E18B0308E18B0308B3
:10017000E18B0308E18B0308E18B0308E18B0308A3
:08018000E18B0308E18B030889
:1001F000425436373032000000000000000000009A
:1002000008B540F6B420074BC2F200001B1A062BBB
:1002100000D808BD40F20003C0F20003002BF8D064
:100220009847F6E7B70A002008B540F6B42040F634
:10023000B423C2F20000C2F200031B1A9B1003EBAE
:10024000D373591000D108BD40F20002C0F2000281
:10025000002AF8D09047F6E710B540F6B424C2F271
:100260000004237873B9FFF7CBFF40F20003C0F21C
:1002700000032BB145F2C800C0F60400AFF30080C4
:100280000123237010BD00BF08B540F20003C0F287
:1002900000034BB145F2C80040F6B821C0F6040097
:1002A000C2F20001AFF3008040F6B420C2F20000B9
:1002B00003682BB140F20003C0F2000303B198477A
:1002C000BDE80840FFF7B0BF81F0004102E000BF89
:1002D00083F0004330B54FEA41044FEA430594EA06
:1002E000050F08BF90EA020F1FBF54EA000C55EA41
:1002F000020C7FEA645C7FEA655C00F0E2804FEA12
:100300005454D4EB5555B8BF6D420CDD2C4480EAF3
:10031000020281EA030382EA000083EA010180EA23
:10032000020281EA0303362D88BF30BD11F0004F71
:100330004FEA01314FF4801C4CEA113102D04042A7
:1003400061EB410113F0004F4FEA03334CEA1333E2
:1003500002D0524263EB430394EA050F00F0A780FA
:10036000A4F10104D5F1200E0DDB02FA0EFC22FAF5
:1003700005F2801841F1000103FA0EF2801843FAE9
:1003800005F359410EE0A5F120050EF1200E012ADA
:1003900003FA0EFC28BF4CF0020C43FA05F3C01818
:1003A00051EBE37101F0004507D54FF0000EDCF191
:1003B000000C7EEB00006EEB0101B1F5801F1BD33A
:1003C000B1F5001F0CD349085FEA30004FEA3C0C3E
:1003D00004F101044FEA445212F5800F80F09A8034
:1003E000BCF1004F08BF5FEA500C50F1000041EB38
:1003F000045141EA050130BD5FEA4C0C404141EB3C
:10040000010111F4801FA4F10104E9D191F0000F62
:1004100004BF01460020B1FA81F308BF2033A3F1E5
:100420000B03B3F120020CDA0C3208DD02F1140CDC
:10043000C2F10C0201FA0CF021FA02F10CE002F117
:100440001402D8BFC2F1200C01FA02F120FA0CFC10
:10045000DCBF41EA0C019040E41AA2BF01EB045159
:10046000294330BD6FEA04041F3C1CDA0C340EDC57
:1004700004F11404C4F1200220FA04F001FA02F39A
:1004800040EA030021FA04F345EA030130BDC4F158
:100490000C04C4F1200220FA02F001FA04F340EA4D
:1004A0000300294630BD21FA04F0294630BD94F0FE
:1004B000000F83F4801306BF81F480110134013DE5
:1004C0004EE77FEA645C18BF7FEA655C29D094EA56
:1004D000050F08BF90EA020F05D054EA000C04BFD4
:1004E0001946104630BD91EA030F1EBF00210020BF
:1004F00030BD5FEA545C05D14000494128BF41F05E
:10050000004130BD14F580043CBF01F5801130BDC1
:1005100001F0004545F0FE4141F470014FF000004C
:1005200030BD7FEA645C1ABF194610467FEA655CFD
:100530001CBF0B46024650EA013406BF52EA03359F
:1005400091EA030F41F4002130BD00BF90F0000F8D
:1005500004BF0021704730B54FF4806404F13204C9
:100560004FF000054FF0000150E700BF90F0000F82
:1005700004BF0021704730B54FF4806404F13204A9
:1005800010F0004548BF40424FF000013EE700BF79
:1005900042004FEAE2014FEA31014FEA02701FBF09
:1005A00012F07F4393F07F4F81F06051704792F0DB
:1005B000000F14BF93F07F4F704730B54FF4607455
:1005C00001F0004521F0004120E700BF50EA0102A0
:1005D00008BF704730B54FF000050AE050EA01024D
:1005E00008BF704730B511F0004502D5404261EBBD
:1005F00041014FF4806404F132045FEA915C3FF4FE
:10060000DCAE4FF003025FEADC0C18BF03325FEA96
:10061000DC0C18BF033202EBDC02C2F1200300FA4B
:1006200003FC20FA02F001FA03FE40EA0E0021FA70
:1006300002F11444C1E600BF70B54FF0FF0C4CF45A
:10064000E06C1CEA11541DBF1CEA135594EA0C0F10
:1006500095EA0C0F00F0DEF82C4481EA030621EA4B
:100660004C5123EA4C5350EA013518BF52EA033586
:1006700041F4801143F4801338D0A0FB02CE4FF038
:100680000005E1FB02E506F00042E0FB03E54FF068
:100690000006E1FB03569CF0000F18BF4EF0010E60
:1006A000A4F1FF04B6F5007F64F5407404D25FEA5C
:1006B0004E0E6D4146EB060642EAC62141EA55510F
:1006C0004FEAC52040EA5E504FEACE2EB4F1FD0C51
:1006D00088BFBCF5E06F1ED8BEF1004F08BF5FEACF
:1006E000500E50F1000041EB045170BD06F0004681
:1006F00046EA010140EA020081EA0301B4EB5C042E
:10070000C2BFD4EB0C0541EA045170BD41F4801125
:100710004FF0000E013C00F3AB8014F1360FDEBF4A
:10072000002001F0004170BDC4F10004203C35DA26
:100730000C341BDC04F11404C4F1200500FA05F3A9
:1007400020FA04F001FA05F240EA020001F000424A
:1007500021F0004110EBD37021FA04F642EB0601C0
:100760005EEA430E08BF20EAD37070BDC4F10C04EA
:10077000C4F1200500FA04F320FA05F001FA04F2AE
:1007800040EA020001F0004110EBD37041F100019A
:100790005EEA430E08BF20EAD37070BDC4F12005A5
:1007A00000FA05F24EEA020E20FA04F301FA05F20D
:1007B00043EA020321FA04F001F0004121FA04F2B5
:1007C00020EA020000EBD3705EEA430E08BF20EA85
:1007D000D37070BD94F0000F0FD101F000464000BF
:1007E00041EB010111F4801F08BF013CF7D041EA41
:1007F000060195F0000F18BF704703F00046520045
:1008000043EB030313F4801F08BF013DF7D043EA15
:100810000603704794EA0C0F0CEA135518BF95EACB
:100820000C0F0CD050EA410618BF52EA4306D1D152
:1008300081EA030101F000414FF0000070BD50EA71
:10084000410606BF1046194652EA430619D094EAFB
:100850000C0F02D150EA013613D195EA0C0F05D1E5
:1008600052EA03361CBF104619460AD181EA030139
:1008700001F0004141F0FE4141F470014FF00000F1
:1008800070BD41F0FE4141F4780170BD70B54FF08C
:10089000FF0C4CF4E06C1CEA11541DBF1CEA13550C
:1008A00094EA0C0F95EA0C0F00F0A7F8A4EB0504EE
:1008B00081EA030E52EA03354FEA013100F08880E5
:1008C0004FEA03334FF0805545EA131343EA1263AE
:1008D0004FEA022245EA111545EA10654FEA002663
:1008E0000EF000419D4208BF964244F1FD0404F51C
:1008F000407402D25B084FEA3202B61A65EB030578
:100900005B084FEA32024FF480104FF4002CB6EB34
:10091000020E75EB030E22BFB61A754640EA0C00B4
:100920005B084FEA3202B6EB020E75EB030E22BFF4
:10093000B61A754640EA5C005B084FEA3202B6EB35
:10094000020E75EB030E22BFB61A754640EA9C00F4
:100950005B084FEA3202B6EB020E75EB030E22BFC4
:10096000B61A754640EADC0055EA060E18D04FEA82
:10097000051545EA16754FEA06164FEAC30343EA22
:1009800052734FEAC2025FEA1C1CC0D111F4801FEF
:100990000BD141EA00014FF000004FF0004CB6E7E8
:1009A00011F4801F04BF01430020B4F1FD0C88BF87
:1009B000BCF5E06F3FF6AFAEB5EB030C04BFB6EB92
:1009C000020C5FEA500C50F1000041EB045170BD85
:1009D0000EF0004E4EEA113114EB5C04C2BFD4EBB2
:1009E0000C0541EA045170BD41F480114FF0000E36
:1009F000013C90E645EA060E8DE60CEA135594EAB2
:100A00000C0F08BF95EA0C0F3FF43BAF94EA0C0FB4
:100A10000AD150EA01347FF434AF95EA0C0F7FF429
:100A200025AF104619462CE795EA0C0F06D152EA7D
:100A300003353FF4FDAE1046194622E750EA410661
:100A400018BF52EA43067FF4C5AE50EA41047FF472
:100A50000DAF52EA43057FF4EBAE12E74FF0FF3CD7
:100A600006E000BF4FF0010C02E000BF4FF0010CA8
:100A70004DF804CD4FEA410C7FEA6C5C4FEA430C21
:100A800018BF7FEA6C5C1BD001B050EA410C0CBF70
:100A900052EA430C91EA030F02BF90EA020F0020D2
:100AA000704710F1000F91EA030F58BF994208BF39
:100AB00090422CBFD8176FEAE37040F001007047F6
:100AC0004FEA410C7FEA6C5C02D150EA013C07D14D
:100AD0004FEA430C7FEA6C5CD6D152EA033CD3D098
:100AE0005DF8040B704700BF8446104662468C4692
:100AF0001946634600E000BF01B5FFF7B7FF0028C5
:100B000048BF10F1000F01BD4DF808EDFFF7F4FFED
:100B10000CBF012000205DF808FB00BF4DF808ED78
:100B2000FFF7EAFF34BF012000205DF808FB00BF9B
:100B30004DF808EDFFF7E0FF94BF012000205DF8BD
:100B400008FB00BF4DF808EDFFF7CEFF94BF012072
:100B500000205DF808FB00BF4DF808EDFFF7C4FF6B
:100B600034BF012000205DF808FB00BF4FEA4102BE
:100B700012F5001215D211D56FF47873B3EB6252EF
:100B800012D94FEAC12343F0004343EA505311F016
:100B9000004F23FA02F018BF404270474FF00000A8
:100BA000704750EA013005D111F0004008BF6FF0E6
:100BB000004070474FF00000704700BF4A0011D25C
:100BC00012F5001211D20DD56FF47873B3EB6252A7
:100BD0000ED44FEAC12343F0004343EA505323FAB3
:100BE00002F070474FF00000704750EA013002D128
:100BF0004FF0FF3070474FF0000070474FEA41025E
:100C0000B2F1E04324BFB3F5001CDCF1FE5C0DD96A
:100C100001F0004C4FEAC0024CEA5070B2F1004FB4
:100C200040EB830008BF20F00100704711F0804FB7
:100C300021D113F13872BCBF01F00040704741F47C
:100C400080114FEA5252C2F11802C2F1200C10FA80
:100C50000CF320FA02F018BF40F001004FEAC12364
:100C60004FEAD32303FA0CFC40EA0C0023FA02F308
:100C70004FEA4303CCE77FEA625307D150EA0133DE
:100C80001EBF4FF0FE4040F44000704701F00040AE
:100C900040F0FE4040F40000704700BF80F000408C
:100CA00002E000BF81F0004142001FBF5FEA410344
:100CB00092EA030F7FEA226C7FEA236C6AD04FEA44
:100CC0001262D2EB1363C1BFD21841404840414089
:100CD000B8BF5B42192B88BF704710F0004F40F43B
:100CE000000020F07F4018BF404211F0004F41F457
:100CF000000121F07F4118BF494292EA030F3FD023
:100D0000A2F1010241FA03FC10EB0C00C3F1200335
:100D100001FA03F100F0004302D5494260EB4000C4
:100D2000B0F5000F13D3B0F1807F06D340084FEA2F
:100D3000310102F10102FE2A51D2B1F1004F40EB24
:100D4000C25008BF20F0010040EA0300704749008C
:100D500040EB000010F4000FA2F10102EDD1B0FA57
:100D600080FCACF1080CB2EB0C0200FA0CF0AABF4C
:100D700000EBC25052421843BCBFD04018437047EA
:100D800092F0000F81F4000106BF80F400000132F0
:100D9000013BB5E74FEA41037FEA226C18BF7FEAC7
:100DA000236C21D092EA030F04D092F0000F08BF09
:100DB0000846704790EA010F1CBF0020704712F0F0
:100DC0007F4F04D1400028BF40F00040704712F12F
:100DD00000723CBF00F50000704700F0004343F094
:100DE000FE4040F4000070477FEA226216BF0846CA
:100DF0007FEA23630146420206BF5FEA412390EA8D
:100E0000010F40F4800070474FF0000304E000BF82
:100E100010F0004348BF40425FEA000C08BF704733
:100E200043F0964301464FF000001CE050EA0102F7
:100E300008BF70474FF000030AE000BF50EA01020C
:100E400008BF704711F0004302D5404261EB4101F9
:100E50005FEA010C02BF84460146002043F0B6431E
:100E600008BFA3F18053A3F50003BCFA8CF2083A43
:100E7000A3EBC25310DB01FA02FC634400FA02FC4C
:100E8000C2F12002BCF1004F20FA02F243EB020053
:100E900008BF20F00100704702F1200201FA02FCB5
:100EA000C2F1200250EA4C0021FA02F243EB0200A8
:100EB00008BF20EADC7070474FF0FF0C1CEAD052EC
:100EC0001EBF1CEAD15392EA0C0F93EA0C0F6FD0AD
:100ED0001A4480EA010C400218BF5FEA41211ED08B
:100EE0004FF0006343EA501043EA5111A0FB013177
:100EF0000CF00040B1F5000F3EBF490041EAD3714C
:100F00005B0040EA010062F17F02FD2A1DD8B3F1C7
:100F1000004F40EBC25008BF20F00100704790F036
:100F2000000F0CF0004C08BF49024CEA502040EA88
:100F300051207F3AC2BFD2F1FF0340EAC25070474E
:100F400040F400004FF00003013A5DDC12F1190F8C
:100F5000DCBF00F000407047C2F10002410021FAFE
:100F600002F1C2F1200200FA02FC5FEA310040F116
:100F7000000053EA4C0308BF20EADC70704792F08F
:100F8000000F00F0004C02BF400010F4000F013AC7
:100F9000F9D040EA0C0093F0000F01F0004C02BFC2
:100FA000490011F4000F013BF9D041EA0C018FE731
:100FB0000CEAD15392EA0C0F18BF93EA0C0F0AD037
:100FC00030F0004C18BF31F0004CD8D180EA01005D
:100FD00000F00040704790F0000F17BF90F0004FF6
:100FE000084691F0000F91F0004F14D092EA0C0FD8
:100FF00001D142020FD193EA0C0F03D14B0218BF6B
:10100000084608D180EA010000F0004040F0FE40B0
:1010100040F40000704740F0FE4040F4400070474C
:101020004FF0FF0C1CEAD0521EBF1CEAD15392EACB
:101030000C0F93EA0C0F69D0A2EB030280EA010CBB
:1010400049024FEA402037D04FF0805343EA111154
:1010500043EA10130CF000408B4238BF5B0042F1B2
:101060007D024FF4000C8B4224BF5B1A40EA0C0057
:10107000B3EB510F24BFA3EB510340EA5C00B3EB89
:10108000910F24BFA3EB910340EA9C00B3EBD10F77
:1010900024BFA3EBD10340EADC001B0118BF5FEAC9
:1010A0001C1CE0D1FD2A3FF650AF8B4240EBC250F2
:1010B00008BF20F0010070470CF0004C4CEA5020B3
:1010C0007F32C2BFD2F1FF0340EAC250704740F402
:1010D00000004FF00003013A37E792F0000F00F0F4
:1010E000004C02BF400010F4000F013AF9D040EA72
:1010F0000C0093F0000F01F0004C02BF490011F406
:10110000000F013BF9D041EA0C0195E70CEAD153FD
:1011100092EA0C0F08D142027FF47DAF93EA0C0FE4
:101120007FF470AF084676E793EA0C0F04D14B02C8
:101130003FF44CAF08466EE730F0004C18BF31F07A
:10114000004CCAD130F000427FF45CAF31F0004374
:101150007FF43CAF5FE700BF4FF0FF3C06E000BF0D
:101160004FF0010C02E000BF4FF0010C4DF804CD30
:101170004FEA40024FEA41037FEA226C18BF7FEA40
:10118000236C11D001B052EA530C18BF90EA010F42
:1011900058BFB2EB030088BFC81738BF6FEAE170D1
:1011A00018BF40F0010070477FEA226C02D15FEA6D
:1011B000402C05D17FEA236CE4D15FEA412CE1D0D9
:1011C0005DF8040B704700BF844608466146FFE7A0
:1011D0000FB5FFF7C9FF002848BF10F1000F0FBD82
:1011E0004DF808EDFFF7F4FF0CBF012000205DF87B
:1011F00008FB00BF4DF808EDFFF7EAFF34BF012000
:1012000000205DF808FB00BF4DF808EDFFF7E0FF98
:1012100094BF012000205DF808FB00BF4DF808EDE9
:10122000FFF7D2FF94BF012000205DF808FB00BF4C
:101230004DF808EDFFF7C8FF34BF012000205DF82E
:1012400008FB00BF4BB942B9002908BF002802D0F3
:101250004FF0FF31084600F03BB882B0EC462DE974
:10126000005000F01DF8DDF804E002B00CBC70473F
:101270002DE9F8439046994606460F4600F02AF8B5
:10128000089BA8FB004508FB01F800FB09825519E3
:10129000341B67EB0505C3E90045BDE8F88300BFD3
:1012A0002DE9F041904606460F461D4600F0C8F96C
:1012B00000FB05F3A0FB084508FB0138069B4544ED
:1012C000341B67EB0505C3E90045BDE8F08100BFAD
:1012D000704700BF2DE9F04F0025002985B01C465E
:1012E000C0F24981002CC0F241818C460F468246F3
:1012F0009146144606461946002B4BD1624559D9F2
:10130000B2FA82F343B1C3F120020CFA03F720FAD8
:1013100002F29C4017439E404FEA1448384641462B
:101320001FFA84F900F018FB41468246384600F067
:1013300041FC330C09FB0AF043EA014188420AD917
:1013400009190AF1FF3205D2884284BFAAF1020AC4
:10135000091900D89246C0EB010B41465846B6B277
:1013600000F0FAFA41460746584600F023FC09FB14
:1013700007F946EA0141894507D97B1E0C1980F01F
:101380005781023FA14540F2538147EA0A404FF09E
:10139000000804E0634558D94FF000084046024673
:1013A000434615B1524263EB43031046194605B05C
:1013B000BDE8F08F22B90120114600F0CDFA0446B5
:1013C000B4FA84F3002B40F0DC803F1B4FEA144951
:1013D0001FFA84FA4FF001084946384600F0BCFA7B
:1013E00049468346384600F0E5FB330C0AFB0BF018
:1013F00043EA014188420BD909190BF1FF3380F010
:101400001581884284BFABF1020B091940F20E81AD
:101410000B1A49461846019300F09EFA019B494673
:10142000B6B20746184600F0C5FB0AFB07FA46EAC3
:1014300001418A4506D97B1E0C1902D2023FA24502
:1014400000D81F4647EA0B40A9E7B3FA83F4002C03
:1014500000F0E480C4F1200301FA04F122FA03FA57
:101460002CFA03FB4AEA010A20FA03F80CFA04FCFE
:1014700058464FEA1A4748EA0C08394602FA04F976
:10148000CDF80C9000F068FA39468146584600F0D5
:1014900091FB1FFA8AFC4FEA18430CFB09F043EA60
:1014A000014398420CD913EB0A0309F1FF3180F094
:1014B000C380984284BFA9F10209534440F2BC8022
:1014C0001B1A39461846CDF808C0019300F044FABB
:1014D000019B39461FFA88F88346184600F06AFBDC
:1014E000DDF808C00CFB0BF348EA01418B420CD934
:1014F00011EB0A010BF1FF3080F09C808B4284BF1E
:10150000ABF1020B514440F29580039F4BEA094036
:10151000C91A1FFA80FCBAB24FEA1749070C02FB3E
:101520000CF802FB07F209FB0C2309FB07F903EB9C
:1015300018439A4288BF09F5803909EB1349494598
:1015400010D31FFA88F814BF0022012206FA04F40F
:1015500008EB03439C422CBF002302F00103002B45
:101560003FF415AF01384FF0000818E7524263EB23
:101570004303ED43B9E6404261EB41014FF0FF35D3
:10158000B0E69C40C3F1200B27FA0BF807FA03F7EB
:101590004FEA14494046494626FA0BFB9E4000F0AC
:1015A000DBF949461FFA84FA4BEA070B034640462B
:1015B000019300F0FFFA019B4FEA1B420AFB03F084
:1015C00042EA0141884206D95A1E091936D2884298
:1015D00034D9023B09190F1A49463846019300F0E5
:1015E000BBF949461FFA8BFB8046384600F0E2FA09
:1015F000019B0AFB08F74BEA01418F420AD90919FE
:1016000008F1FF3205D28F4284BFA8F10208091900
:1016100000D89046CF1B48EA0348DDE60120634529
:1016200028BF5245A0467FF6BAAEB5E69B46EFE628
:101630001F46AAE6834668E7894641E71346CAE79C
:101640002DE9F04F064683B00D46144607468846FE
:10165000002B4AD18A4255D9B2FA82F34BB1C3F179
:10166000200201FA03F820FA02F29C4042EA08083C
:101670009F40250C404629461FFA84FA00F06CF979
:1016800029468146404600F095FA3B0C0AFB09F0DA
:1016900043EA014188420AD9091909F1FF3205D20A
:1016A000884284BFA9F10209091900D89146C0EB0C
:1016B000010829464046BFB200F04EF929460646C9
:1016C000404600F077FA0AFB06FA47EA01418A45EC
:1016D00007D9731E0C1980F02281023EA24540F208
:1016E0001E8146EA0940002658E08B4254D8B3FADE
:1016F00083F4002C56D18B4228BF82424CD8264618
:1017000001204BE022B90120114600F025F90446E2
:10171000B4FA84F3002B40F0B9802D1B4FEA144833
:101720001FFA84FA01264146284600F015F9414681
:101730008146284600F03EFA3B0C0AFB09F043EADA
:10174000014188420BD9091909F1FF3380F0E98082
:10175000884284BFA9F10209091940F2E280C0EB76
:10176000010B41465846BFB200F0F6F84146054627
:10177000584600F01FFA0AFB05FA47EA01418A457C
:1017800007D96B1E0C1980F0CE80023DA24540F2B5
:10179000CA8045EA094001E000263046314603B0E0
:1017A000BDE8F08FC4F1200103FA04F322FA01F836
:1017B00025FA01F748EA030820FA01F105FA04F5D1
:1017C00038464FEA18490D43494602FA04F201929D
:1017D00000F0C2F849468246384600F0EBF91FFA9D
:1017E00088F22F0C02FB0AF047EA0147B84206D9FB
:1017F00017EB08070AF1FF31C0F09F808A463F1AB5
:1018000049463846009200F0A7F84946ADB28346F3
:10181000384600F0CFF9009A02FB0BF745EA014188
:101820008F4205D911EB08010BF1FF327DD39346AE
:10183000019B4BEA0A40C91B4FEA104C9DB24FEA8C
:10184000134A83B205FB03F205FB0CF50AFB0353B5
:101850000AFB0CFA03EB12439D4288BF0AF5803A5B
:101860000AEB134A51450ED392B214BF0021012155
:1018700006FA04F602EB03439E422CBF002601F059
:101880000106002E8AD00138002687E79C40C3F16C
:10189000200225FA02FA26FA02F94FEA14485046C5
:1018A000414605FA03F506FA03F700F055F84146FC
:1018B00049EA05098346504600F07CF91FFA84FA8C
:1018C0004FEA19430AFB0BF043EA0141884209D968
:1018D00009190BF1FF3338D2884284BFABF1020BF8
:1018E000091932D90D1A414628461FFA89F900F024
:1018F00033F841460646284600F05CF90AFB06F537
:1019000049EA01418D4206D9731E09191FD28D4241
:101910001DD9023E09194D1B46EA0B4603E71E4638
:10192000DFE699461BE71D4633E78F4284BFABF1E4
:10193000020B41443FF67CAF79E7B84284BFAAF17D
:10194000020A47443FF65BAF58E79B46CAE71E468C
:10195000E1E700BF000000004A1E08BF7047C0F06A
:101960002481884240F21681114200F01781B0FABA
:1019700080F3B1FA81F2A2EB0303C3F11F0304A2C7
:1019800002EB03134FF000029F4600BFAFF300804D
:10199000B0EBC17F00BF42EB020228BFA0EBC170D9
:1019A000B0EB817F00BF42EB020228BFA0EB817049
:1019B000B0EB417F00BF42EB020228BFA0EB4170B9
:1019C000B0EB017F00BF42EB020228BFA0EB017029
:1019D000B0EBC16F00BF42EB020228BFA0EBC160B9
:1019E000B0EB816F00BF42EB020228BFA0EB816029
:1019F000B0EB416F00BF42EB020228BFA0EB416099
:101A0000B0EB016F00BF42EB020228BFA0EB016008
:101A1000B0EBC15F00BF42EB020228BFA0EBC15098
:101A2000B0EB815F00BF42EB020228BFA0EB815008
:101A3000B0EB415F00BF42EB020228BFA0EB415078
:101A4000B0EB015F00BF42EB020228BFA0EB0150E8
:101A5000B0EBC14F00BF42EB020228BFA0EBC14078
:101A6000B0EB814F00BF42EB020228BFA0EB8140E8
:101A7000B0EB414F00BF42EB020228BFA0EB414058
:101A8000B0EB014F00BF42EB020228BFA0EB0140C8
:101A9000B0EBC13F00BF42EB020228BFA0EBC13058
:101AA000B0EB813F00BF42EB020228BFA0EB8130C8
:101AB000B0EB413F00BF42EB020228BFA0EB413038
:101AC000B0EB013F00BF42EB020228BFA0EB0130A8
:101AD000B0EBC12F00BF42EB020228BFA0EBC12038
:101AE000B0EB812F00BF42EB020228BFA0EB8120A8
:101AF000B0EB412F00BF42EB020228BFA0EB412018
:101B0000B0EB012F00BF42EB020228BFA0EB012087
:101B1000B0EBC11F00BF42EB020228BFA0EBC11017
:101B2000B0EB811F00BF42EB020228BFA0EB811087
:101B3000B0EB411F00BF42EB020228BFA0EB4110F7
:101B4000B0EB011F00BF42EB020228BFA0EB011067
:101B5000B0EBC10F00BF42EB020228BFA0EBC100F7
:101B6000B0EB810F00BF42EB020228BFA0EB810067
:101B7000B0EB410F00BF42EB020228BFA0EB4100D7
:101B8000B0EB010F00BF42EB020228BFA0EB010047
:101B9000104670470CBF012000207047B1FA81F257
:101BA000C2F11F0220FA02F0704708B14FF0FF3077
:101BB000FFF78EBB0029F8D02DE90340FFF7CCFEDC
:101BC000BDE8064002FB00F3A1EB0301704700BF34
:101BD000002101F0E7BD00BF00210A2201F0E2BEB2
:101BE00000220A2301F03CBE70B545F2E80645F23A
:101BF000E805C0F60406C0F60405761BB61007D04B
:101C0000043D002455F8043F01349847A642F9D119
:101C100045F2EC0645F2E805C0F60406C0F60405F8
:101C2000761B23F051FAB61008D0043D002455F875
:101C3000043F01349847A642F9D170BD70BD00BF82
:101C4000032A70B422D941EA00039B0713D0057818
:101C5000013A0C780023A54206D01BE010F8015F82
:101C600011F8014FA54215D1934203F10103F5D1BB
:101C7000002070BC70470C460346043104301E68D7
:101C80002568AE4208D1043A032AF4D8002ADED1EE
:101C90001046EEE7281BECE721461846002AD6D16D
:101CA000F6E700BF032A2DE9F00F09D82AB1002377
:101CB000CC5CC45401339342FAD1BDE8F00F7047B5
:101CC000830702440ED0441C4D1C15F8017C04F01F
:101CD0000306234601342946013504F8027C002E10
:101CE000F3D100E0034611F003046DD0D71A0D1BA9
:101CF000032F2E6819DDC4F1040C4FEAC4081C1D23
:101D00004FEACC0C55F8047FC4EB0209234604319A
:101D10000434B9F1030F26FA08FA07FA0CFB3E4621
:101D20004BEA0A0744F8087CECDC9A42C5D9013337
:101D30000131013211F8014C01330131934203F8B2
:101D4000024CF7D1B9E70C684033403143F8404CBE
:101D500051F83C4C43F83C4C51F8384C43F8384C63
:101D600051F8344C43F8344C51F8304C43F8304C73
:101D700051F82C4C43F82C4C51F8284C43F8284C83
:101D800051F8244C43F8244C51F8204C43F8204C93
:101D900051F81C4C43F81C4C51F8184C43F8184CA3
:101DA00051F8144C43F8144C51F8104C43F8104CB3
:101DB00051F80C4C43F80C4C51F8084C43F8084CC3
:101DC00051F8044C43F8044CD41A3F2CBBDC11E00E
:101DD0000C681033103143F8104C51F80C4C43F898
:101DE0000C4C51F8084C43F8084C51F8044C43F89B
:101DF000044CD41A0F2CEBDC032C96DD1C1D0D1D9E
:101E000055F8047C161B2346294604340435032E5A
:101E100044F8087CF4DC88E7032AC9B270B408D817
:101E20002AB10346121803F8011B9342FBD170BC80
:101E300070478307024409D0441C04F0030523467D
:101E400004F8011C0134002DF7D100E00346D51A37
:101E500001EB01243F2D04EB04442CDD1C604033D6
:101E6000D51A43F83C4C3F2D43F8384C43F8344CDA
:101E700043F8304C43F82C4C43F8284C43F8244C9E
:101E800043F8204C43F81C4C43F8184C43F8144CCE
:101E900043F8104C43F80C4C43F8084C43F8044CFE
:101EA000DCDC08E01C601033D51A43F80C4C43F816
:101EB000084C43F8044C0F2DF4DC032D08DD1D1DE8
:101EC000561B45F8044C032E2B4605F10405F7DCA0
:101ED0009A42ACD90133013203F8011C0133934219
:101EE000FAD1A4E7830770B5064614D10368A3F1BD
:101EF000013222EA030313F0803F0CD1031D1A467E
:101F000053F8044BA4F1013525EA040414F0803F92
:101F1000F5D0104600E0304603782BB1431C18463C
:101F200001330478002CFAD100F0F0F8304670BD8F
:101F300080EA010212F0030F40F03A8010F0030231
:101F400020F0030021F0030150F804CB08BF51F842
:101F5000043B0DD082F003024FEAC2026FF07F43D0
:101F600023FA02F251F8043B4CEA020C43EA020362
:101F7000ACF101329C4501BF22EA0C0212F0803F15
:101F800050F804CB51F8043BF2D04FEA0C604FEA12
:101F90001C2C012828BFB0EB036F08BF1B0AF4D02C
:101FA00003F0FF034FEA1060A0EB0300704700BF8F
:101FB00010F0030F0AD010F8012B11F8013B012A91
:101FC00028BF9A42F4D0A2EB030070474DF8045D9D
:101FD0004DF8044D4FF0010242EA022242EA024269
:101FE00001F0030C21F0030150F8044B51F8045B9D
:101FF000BCF1020F26D04BD824F07F4CBCEB152F40
:10200000A4EB020323EA04030DD113EAC21308BFB1
:1020100051F8045B0AD18CEA040CBCEB056F0CD1BF
:1020200050F8044BE8E74FEA15255CE033F07F43B6
:1020300052D10D784FEA146C55E04FEA146C05F05C
:10204000FF0550E04FEA044CA4EB02034FEA1C4C9E
:1020500023EA0403BCEB154F17D113EAC21308BFE0
:1020600051F8045B07D18CEA040CBCEB054F08D196
:1020700050F8044BE6E71B042ED10D884FEA144CB0
:1020800031E04FEA05454FEA144C4FEA15452AE086
:1020900004F0FF0CBCEB156FA4EB020323EA04036E
:1020A0000DD113EAC21308BF51F8045B0AD18CEAC0
:1020B000040CBCEB052F0AD150F8044BE8E74FEABB
:1020C000156510E014F0FF0F06D051F8045B4FEADD
:1020D000142C25F07F4506E04FF000005DF8044B1E
:1020E0005DF8045B70470CF0FF0205F0FF0001286B
:1020F00028BF904204BF4FEA1C2C2D0AF3D0A2EB5C
:1021000000005DF8044B5DF8045B704780EA010253
:10211000844612F0030F4FD111F0030F32D14DF866
:10212000044D11F0040F51F8043B0BD0A3F1013220
:102130009A4312F0803F04BF4CF8043B51F8043B33
:1021400016D100BF51F8044BA3F101329A4312F0AB
:10215000803FA4F101320BD14CF8043BA24312F0B2
:10216000803F04BF51F8043B4CF8044BEAD02346AF
:102170000CF8013B13F0FF0F4FEA3323F8D15DF861
:10218000044B704711F0010F06D011F8012B0CF829
:10219000012B002A08BF704711F0020FBFD031F8A1
:1021A000022B12F0FF0F16BF2CF8022B8CF8002028
:1021B00012F47F4FB3D1704711F8012B0CF8012BAB
:1021C000002AF9D1704700BF20F0030110F003008E
:1021D000C0F1000051F8043B00F1040C4FEACC0CB4
:1021E0006FF000021CBF22FA0CF213434FF0010CF7
:1021F0004CEA0C2C4CEA0C4CA3EB0C0222EA030236
:1022000012EACC1204BF51F8043B0430F4D013F0AE
:10221000FF0F1FBF013013F47F4F013013F47F0F06
:1022200018BF0130704700BF830770B413D1036833
:10223000A3F1013424EA030313F0803F0BD1031D03
:102240001D4653F8044BA4F1013626EA040414F0A9
:10225000803FF5D000E005462B782BB16B1C1D4666
:1022600001332C78002CFAD10139013D531E5AB1AB
:1022700011F8014F1A4605F8014F2CB1002BF5D18A
:102280006B70531E002AF3D170BC704770B4002AE3
:1022900045D041EA000313F0030329D1032A27D9CB
:1022A00005680C68A54223D1141F3AD0A5F101326C
:1022B00022EA050515F0803F0DD03AE05B686A68B8
:1022C000A3F10135934225EA03052ED1043C28D021
:1022D00015F0803F27D10D46034604310430032C0E
:1022E000ECD8661E2CB91C792A79A01A70BC7047EC
:1022F000561E04780A789442F7D1C6B18CB10136E3
:102300008B1C891904E08B4203F101030BD044B10B
:1023100013F8012C10F8014F9442F4D0E5E7104671
:10232000E4E72046E2E70020E0E7661EE1E730460A
:10233000DCE71846DAE700BF41EA000313F0030FB9
:10234000034670B425D0AAB10C78013A03F8014BCA
:102350004CB11C4672B111F8015F013A04F8015BFF
:102360002346002DF6D12AB19A18002103F8011B4B
:102370009342FBD170BC70470E4651F8044BA4F158
:10238000013525EA040515F0803F05D1043A43F8EC
:10239000044B032AF0D8D6E73146D4E7F0B40478EA
:1023A000002C21D00F7806463046AFB1A74219D095
:1023B0004B1C01E0944209D01D4613F8012B002A62
:1023C000F8D144780136002CEED12A78002A14BFC7
:1023D00030460020F0BC704744780D460136002C92
:1023E000E2D1F2E73A46F1E72046F3E72DE9F007BC
:1023F00001273C4600254FF0FF36631900EB060C21
:102400008B420DD21CF804C010F80380E0452ED298
:1024100001241D469F1B63198B4200EB060CF1D370
:102420004FF0010A002554464FF0FF3C1760631936
:1024300000EB0C0899420ED918F8048010F80390AC
:10244000C1451AD901241D46CCEB030A63199942F0
:1024500000EB0C08F0D80CF101000136B0423CBF93
:10246000BA463046C2F800A0BDE8F00770470BD06E
:1024700001272E463C46ED19BFE709D04FF0010A6F
:10248000AC4654465544D2E7BC4205D00134B4E7CB
:10249000544505D00134CAE727461D460124ACE760
:1024A000A2461D460124C2E72DE9F04FADF2244DAE
:1024B000164680460C461046194607AA1D46FFF7E9
:1024C00095FF07AB0DF21C42039043F8045F934263
:1024D000FBD16F1E002308A835B1F25CF91A013355
:1024E000AB4240F82210F8D107993046039A711890
:1024F000FFF7A6FB00287FD1DDF80CC022468246FC
:102500006F1E0CF1FF3CCDF808C0B444CDF814C0E8
:10251000DDF80CC004460195CCF1010CCDF810C0DB
:1025200009E034B1079A93423EBF04460199C2EBD9
:1025300001039A442A46019B08EB020000210AEBA2
:102540000305AA1A02F090FA00284FD1002D4DD0B1
:1025500008EB050308A913F8013C51F82330002BC0
:10256000DFD1039A944228BF2246BA4211D208EB27
:102570000A0316F802C0B118985C844506D02FE013
:1025800011F8010F13F802C0844529D10132BA4273
:10259000F6D3039B02989C4228BF184618D2DDF858
:1025A00008C008EB0A0316F80C1013F80C2091422F
:1025B00040F08580059A06EB040B06E013F801C095
:1025C00012F8019DE14503D10846411E5A45F5D157
:1025D0000134844275D8079C019BA2441C1BA9E7C7
:1025E000DDF810C00024E2449244A3E7002009B0C3
:1025F0000DF5806DBDE8F08FDDF80CC04FF0000ADE
:10260000DDF80CB00DF12009CCEB05036F1E63451E
:1026100038BF63462246013307930CF1FF33019321
:10262000039BB444CDF808C0C3F1010304930AEB43
:10263000050408EB02000021A21A02F015FA002896
:10264000D4D1002CD2D008EB040313F8013C59F884
:10265000233063BBBB4508EB0A0015D2DDF808C088
:1026600010F80B309CF800209A4218BF5B4621D12D
:10267000029A5B4605E012F8011F10F803C08C4572
:1026800018D10133BB42F6D3019B5A1CAFD0DDF801
:1026900004C016F80C1010F80C20914206D113F16A
:1026A000FF33A4D3F15CC25C9142F8D0079B9A44FB
:1026B0002246BCE7DDF810C0E2449A44F8E70398EC
:1026C00086E708EB0A0092E72DE9F04F8046037891
:1026D00087B00E46002B00F0F7800A789AB1844646
:1026E0000131012702E011F8012B5AB1934214BFC6
:1026F000002707F001071CF8013F0D46002BF2D11F
:102700002B7803BB1FB1404607B0BDE8F08F08F13E
:102710000100317802F092FEAD1B012D18BF002898
:10272000074608BF8046EED0A844404594BFC0EBA2
:10273000080401241F2D09D9214632462B46FFF7F4
:10274000B3FE8046DFE74FF00008DCE7294605AA24
:102750003046FFF74BFE0599711801903046019AFB
:10276000FFF76EFA002852D1019B83468046013B59
:102770000093F3180393019BC3F1010302932246D4
:1027800008EB0504B8180021A21A02F06DF9002820
:10279000D9D1002CD7D0019B9B4528BF5B469D42D9
:1027A00013D9F918F05CF21811F80810884240F0BB
:1027B000858007EB080C05E012F8011F1CF80300E8
:1027C00088427BD101339D42F6D89DE80A005B45E3
:1027D0007DD907EB0809725C19F801309A4276D16D
:1027E000039B06EB0B0A06E019F8020013F801CD73
:1027F000844503D111464A1E5345F5D10BF1010B17
:102800008B4566D8059B9844C3EB050BB7E7019849
:102810004FF0000B22462B1A06EB000900F1FF389F
:102820008246834238BF034639180133009105932D
:10283000C0F1010302930BEB0504B8180021A21AA2
:1028400002F012F900287FF47EAF002C3FF47BAF3A
:10285000554598BF07EB0B0014D9009899F8002054
:1028600010F80B309A4224D14A46534607EB0B002E
:1028700005E012F8011F10F803C08C451AD101338E
:102880009D42F6D8B8F1FF3F43463FF45AAF16F8E1
:10289000081010F80820914207D113F1FF33FFF41C
:1028A00050AFF15CC25C9142F7D0059B9B4422463D
:1028B000C1E75346029A93449B44F8E702994FF0CC
:1028C000000B884498445AE70D46012718E7019900
:1028D00094E7B84417E700BF2DE9F04F9DB08C4650
:1028E00083461092624600200021CDF85CC0CDE9FD
:1028F0000601114612F8013B2D2B00F24781DFE85B
:1029000013F03101450145014501450145014501EE
:1029100045014501640164016401640164014501EC
:102920004501450145014501450145014501450177
:102930004501450145014501450145014501450167
:102940004501640145014501450145014501450138
:1029500045014501450145012E0145012E00012596
:1029600012954E1C17964B7899469A46002B00F00C
:10297000FC80302B18BF4FF0000900F010812F2B86
:102980001D464FF0000A40F3F984392B00F3F6841A
:10299000721C5746544601E0392B18DC07EB8701BF
:1029A000082C03EB4101D8BFA1F1300707DD0AEB8A
:1029B0008A010F2C03EB4103D8BFA3F1300A179211
:1029C000904612F8013B01342F2B1D46E4DC58469B
:1029D000CDF810C001F05AFD01685846059101F08C
:1029E00055FD0068FFF7F0FB059902464046FFF7EA
:1029F0004DFCDDF810C08046002800F04281002028
:102A0000A0460146099025F02003452B40F0DF80C9
:102A100048EA000353EA090300F01D81DDF85CC0B9
:102A20000CF1010317939CF801502B2D00F0AB849F
:102A30002D2D00F03D8300220A92A5F13003092BD1
:102A400000F22C84302D06D1179B0133179313F815
:102A5000015B302DFAD0A5F13103082B00F2B780CD
:102A6000179A303D0D95531C179355780B922F2DC7
:102A700016DD392D14DC931C0C910D9A01E0392DD3
:102A80000BDC1793194602EB8202013305EB42027D
:102A900013F8015C303A2F2DF1DC0B460C990D92A6
:102AA0000B9A9B1A082BC8BF44F61F6205DC0D9ACF
:102AB00044F61F639A42A8BF1A460A9B03B15242CA
:102AC000B8F1000F00F08880099D3846002C08BF3F
:102AD00044460A94521B0992FDF738FDB8F1100FD5
:102AE000B4BFC1464FF01009B9F1090F02460B46B9
:102AF000CDE9062316DD48F62053C0F6030303EBA9
:102B0000C90353E91223FDF797FD044650460D46CD
:102B1000FDF71CFD02460B4620462946FDF7DAFB71
:102B2000CDE90601B8F10F0F00F3F280099C002CEB
:102B300000F0A28040F39185099D162D00F3458594
:102B400048F62051DDE90623C0F6030101EBC5017B
:102B5000D1E90001FDF770FD81468A4609E00024B5
:102B60001294FEE64FF00009CA460024CDF85CC07E
:102B70001294109C0CB1179B2360129D0DB10AF1A9
:102B8000004A484651461DB0BDE8F08F0025302B65
:102B90000E46129518BF4FF000097FF4F0AE73781F
:102BA000582B00F08383721C782B00F07F8316462D
:102BB000179212F8013B302BF9D04FF00109002B8E
:102BC0007FF4DDAE99469A46D3E7179291E600224C
:102BD000B8F1000F7FF478AF50EA09004CD100291A
:102BE00039D1493D252D36D8DFE815F06A02350088
:102BF000350035003500260035003500350035003C
:102C0000350035003500350035003500350035001C
:102C1000350035003500350035003500350035000C
:102C20003500350035003500350035006A023500C5
:102C300035003500350026005348179A10F8011F5B
:102C4000134669B15B780132402B02DD5A2BD8BFA5
:102C500020338B42F2D0DDF81890DDF81CA084E719
:102C6000531C17935378282B00F075850023069387
:102C70001C46CFF6F8740794DDF81890DDF81CA018
:102C800077E75846179D01F001FC0068FFF79CFAB2
:102C9000DDF810C02B1817932D5C002C40F09B81A1
:102CA000302D204605D10133179301301D78302D8A
:102CB000F9D0A5F13103082B00F29A81179E4FF04D
:102CC00000080990A5F1300101200A96002900F0C2
:102CD0006C83099A01280244099200F0328508EBBE
:102CE00000024346013ACDF82C80904603E06F0085
:102CF000434500F04B83013307EB87055A1E082A32
:102D0000F5DD0AEB8A02102BD8BF4FEA420AEFE743
:102D1000099DC9EB080905EB0904002C40F3DE838B
:102D200014F00F000DD048F62051DDE90623C0F65F
:102D3000030101EBC001D1E90001FDF77DFCCDE904
:102D4000060134F00F0440F05F81DDF81890DDF8E3
:102D50001CA00B940097584631460A9A434601F04E
:102D600067FF099D002D1190C0F2728400240D941C
:102D7000099D119C25EAE575CDF824900C340E953B
:102D80001394CDF828A073E0935004080F9B002BF8
:102D900000F0A8814FF000090025DDF81CC00024D8
:102DA000C3F6F075C3F6F079CDF830804FF0000827
:102DB0004346C7F6F078C7F6E0730CEA0808984572
:102DC00000F0C5810B9AB8F1D46F8CBF00230123AA
:102DD000002A08BF0023EBB10C98494688A3D3E929
:102DE0000023FDF7A5FE88B10C984946FDF7E6FEE5
:102DF000002800F04682FDF7A9FB89460C900F9C45
:102E000009F1004304B14B460C9C1D4605F1D66305
:102E1000C8EB030509980A9902F08AF902460B46A5
:102E200020462946FDF708FC02460B4609980A99F8
:102E3000FDF750FACDE90601079C09900A910B9D18
:102E400035B90023C7F6F0732340984500F0BC81E4
:102E50005846189901F08CFE5846514601F088FEFC
:102E60005846394601F084FE5846314601F080FE4E
:102E7000119C584616AD616801F044FE2369139910
:102E80009A1C920082460C30FEF70CFF099A0A9BAE
:102E900019A800950190584602F0C4F90121189034
:102EA000584601F05DFF169A199B6FF47F71002A56
:102EB000AABF0D9D0E9CAC180B9D0746B8BFC2EB78
:102EC0000400C5EB0202B8BF0D9C02EB0305A8BFCE
:102ED0000E988D420D99B4BF02F23343C3F136030D
:102EE000E618C3180B981D18A642B4BF33462346F4
:102EF000AB42A8BF2B46002BC2BFC3EB0606C3EBF9
:102F00000505C3EB040489B10A465846394601F069
:102F1000CFFF189A07465846394601F02BFF1899FB
:102F20008046584601F024FECDF86080002E05DD75
:102F300058461899324602F00DF818900E9A22B1B0
:102F40005146584601F0B4FF8246002D05DD51463A
:102F500058462A4601F0FEFF8246002C05DD394620
:102F60005846224601F0F6FF074618995246584641
:102F70004FF0000802F066F83946C4680646C0F80B
:102F80000C800F9402F040F84045C0F2138200F02C
:102F900061823046394602F0A3F900224FF08043A7
:102FA00004460D46FDF7C4FD00287FF4EFAE002374
:102FB0002046C3F6E07329460022FDF73DFB0F9C37
:102FC0000C90894601F1004304B10B460C9C1D4650
:102FD000DDF81CC0EAE64046A0460990A5F13001A4
:102FE000092903D8179A01300A926FE601210AE5F0
:102FF0004FF000080121CDF8248004E5AFF30080F4
:103000000000C0FFFFFFDF41B4F59A7F00F3588254
:10301000241148F6106A012C40F39883C0F6030A85
:10302000DDE906234FF00009554614F0010F104664
:1030300019464FEA640409F1010905D0D5E90023D6
:10304000FDF7FAFA02460B460835012CEDDC104676
:103050001946CDE9060107990AEBC909A1F1547196
:103060000791DDE90623D9E90001FDF7E5FA002320
:103070000022C7F6F073C7F6A042CDE90601079912
:103080000B40934200F21C820022C7F6904293420A
:1030900040F205834FF6FF724FF0FF3015460024D3
:1030A000C7F6EF750B94079581460690AA4651E640
:1030B00001230A930CF1020317939CF80250BCE41D
:1030C000AB48179A10F8011F1346002900F011832E
:1030D0005B780132402B02DD5A2BD8BF20338B4264
:1030E000F0D0B8E5069BDDF81CC0002B40F0A680B0
:1030F000CCF3130303BB0023204629460022C3F66A
:10310000F073CDF810C0FDF709FDDDF810C0002800
:1031100040F0468200230022C3F6E0732046294691
:10312000FDF78AFADDF810C08946024601F1004336
:103130000C9014461D4639E64FF000090025CDF8E5
:1031400030900024CBF6F075C3F6F0792EE6ACF1A2
:10315000547C099ACDF81CC00A9BDDE90601CDE933
:10316000024514461D46CDE9144501F0E1FF024633
:103170000B46DDE90201FDF75FFA02460B46DDE989
:103180000601FDF7A7F80023C7F6F0734FF6FF72AC
:10319000C7F69F42CDE90601079C2340934276D9AA
:1031A0004FF6FF73159DC7F6EF739D4200F07781D0
:1031B0004FF6FF714FF0FF330A460693C7F6EF72E2
:1031C000099307920A9243E649460C98FDF7CEFC14
:1031D000FDF7CCF902460B460C984946FDF778F806
:1031E0000F9D80468946002D37D1069A002A34D19A
:1031F000C4F31304002C30D157A3D3E90023FDF707
:103200008DFC00283FF424AE5446DDF82490DDF810
:1032100028A05846189901F0ABFC5846214601F009
:10322000A7FC5846394601F0A3FC5846119901F015
:103230009FFC5846314601F09BFC9AE4012B7FF439
:103240007BAF614600297FF477AF54464FF0000909
:10325000CA462223CBF80030DBE74046494640A36C
:10326000D3E90023FDF75AFC0028CDD1404649465A
:103270003DA3D3E90023FDF76FFC00283FF4E8AD40
:10328000C2E74FF000090C90C3F6F079B7E5069954
:1032900004F1547407940A940991D0E5CDF85CC008
:1032A0000022B8F1000F7FF40FAC95E4129D40F2BC
:1032B0000404C2F2000418AB58468DE8280017A990
:1032C000224619AB00F01CFD10F00707054604BFAD
:1032D000B946CA463FF44DAC062F00F06F81189AEC
:1032E0003AB121681AA802F045F85846189901F039
:1032F0003FFC199B062F0BD8DFE807F03C201B147E
:1033000004203C006FF000444FF0FF30079406901B
:103310002B077FF5B1AC0799DDF8189041F0004319
:103320009A4626E4002106910A46C7F6F0720792F3
:10333000EEE71A9B1B9C06930794E9E71A9803F2A1
:1033400033431B9A22F48012069042EA03520792FA
:10335000DEE700BFAFF300809535A094FFFFCF3FBD
:103360009535A094FFFFDF3F35E5AF350000E03F26
:1033700087500408002107910691C9E7B0465746D7
:103380005446FFF724BB00230A9393E6DDF82C8014
:1033900008EB0003013B082B03F1010800F37281E5
:1033A00007EB8707002001EB47070A9D6B1C17936B
:1033B0006D7813E60F9D54467DBB069868BB079A4F
:1033C000C2F313034BBB4346C7F6F0731340B3F18C
:1033D000D66F22D9736913B93369012B1DDD3146CC
:1033E0000122584601F0B6FD3946064601F00CFEB2
:1033F000002812DD0B9D002D40F09581079820F0EC
:1034000000431B0D1B05A3F580134FF0FF320692FE
:103410006FEA13536FEA035307930B9D002D00F0DF
:10342000C88000220023C3F6501214931592DDE9E0
:103430000601DDE91423FDF7FFF8CDE906018A4610
:103440000799814600297FF4E4AE069A002A7FF4AA
:10345000E0AEFEE60F9D5446DDF82490DDF828A08E
:10346000002D00F0D380079B4FF6FF72C0F20F02D1
:1034700023F07F4121F470019142069900F01981F7
:10348000CB07CAD54846514601F052FE02460B46CC
:1034900048465146FCF71EFFCDE90601BDE71498EA
:1034A00001307FF485AE0020544601462223C7F642
:1034B000F071CBF800300791814606908A46A8E665
:1034C000002300251C460695C7F6F07422230794B6
:1034D000A946CBF80030A246FFF74BBB3FF435AC12
:1034E000644214F00F020DD048F62053DDE90601C6
:1034F000C0F6030303EBC203D3E90023FDF7C6F9CB
:10350000CDE9060124113FF420AC1F2C40DC14F05F
:10351000100F14BF6A250025002C0B9517DD48F607
:10352000E845DDE90623C0F6030514F0010F104657
:10353000194605D0D5E90023FDF77EF802460B4673
:1035400008356410F1D110461946CDE906010B9CEF
:103550008CB1079AC2F30A53C3F16B03002B0ADD47
:103560001F2B40F30A810021342B069140F30D817B
:103570004FF05C720792069D0022079C00232846AC
:10358000A9462146A246FDF7BFFA00283FF4E2AB68
:103590004FF000092223CA46CBF80030FFF7E9BA02
:1035A0000F9A00239946CBF6E073C3F6E0790C92AC
:1035B000BFE5DDF81890DDF81CA02AE64FF0000901
:1035C0000136CA461796FFF7D4BA099CC8F12503FD
:1035D0009C423FF79DABC8F10F0848F62054C0F657
:1035E0000304DDE9062304EBC801D1E90001FDF77E
:1035F00023F8099DC8EB050804EBC804D4E90023AF
:10360000FDF71AF881468A46FFF7B3BA0799C1F366
:103610001303002B41D1069B002B3FF4EBAEDA07DE
:103620007FF5FBAE4846514601F082FD02460B464F
:1036300048465146FCF74CFE02460B46CDE90623B0
:1036400000220023FDF760FA00287FF4FFADE4E6D6
:10365000099D6D420D95FFF78BBB099C14F1160F68
:10366000FFF656AB48F62053DDE90601C0F603032A
:10367000A3EBC403D3E90023FDF708F981468A468A
:10368000FFF777BA0020B8F1100F3FF78EAE0AEBC4
:103690008A0A002001EB4A0A87E6069BBFE701F190
:1036A0005471002407918A460B94DDF81890FFF7B7
:1036B00051BB0B9DD5B10022C7F6F0721A40B2F192
:1036C000D46F13D8120D4FF0FF30C2F16B0200FA25
:1036D00002F291427FF4D4AE00220020C7F6F072CD
:1036E00006901A4002F58012079296E64FF0FF32DC
:1036F000EFE72A4C1146179214F8010F0B4610B34E
:103700005B780131402B02DD5A2BD8BF2033834236
:10371000F2D001321792002506952846C7F6F070C0
:103720000790FFF7A9BA079921F000431B0D1B056D
:10373000B3F1D66F3FF667AEB3F15C7F3FF671AE83
:1037400084E5434627E601311791E4E74FF000098D
:10375000C0F6030A7FE417A811491AAA00F07EFDFB
:1037600005287FF483AA1B9B1A9A43F0FF4343F476
:10377000E00307930692FFF77FBA4FF0FF32069CF3
:1037800002FA03F31C400694F5E64FF0FF31203BAC
:1037900001FA03F313400793EDE600BF8B500408D2
:1037A0001800002040F22C030A46C2F20003014632
:1037B0001868FFF791B800BF2DE9F84340F22C06D6
:1037C000C2F200060A4601464FF001083068FFF7D2
:1037D00083F80D460446FDF711FA00210746FDF770
:1037E000FFFC08B94FF000082046294600220023BC
:1037F0004FF00109FDF788F908B14FF0000908EA18
:10380000090818F0FF0F16D14FF6FF713846C7F6BA
:103810007F71FDF70DFDA0B938466FF40001FDF78B
:10382000E9FC58B1204629464FF0FF326FF480136F
:10383000FDF774F910B9336822221A603846BDE8E2
:10384000F8834FF6FF73204629464FF0FF32C7F644
:10385000EF73FDF781F90028EDD0DDE7AFF30080CD
:103860002DE9F04F40F20004C2F2000485B0994601
:103870000B46D4F80080029103901C4614F8015BBB
:1038800008EB05012346497801F00801C9B2002977
:10389000F3D12D2D7BD02B2D05BF24460B460B4697
:1038A00014F8015B39F0100112D1D9F1010038BFD1
:1038B0000020302D04D058B14FF00A09CB4608E063
:1038C000217801F0DF01582965D008B14FF00809CF
:1038D000CB46002B59460CBF6FF000464FF0004618
:1038E0008DE80C0030460027FEF764F930468A4622
:1038F0005946FEF731F8BC469DE80C0016E0303D15
:10390000A94525DD844594BF0021012151EAD777DF
:1039100029D15545D4BF00210121844518BF00217C
:1039200009BB0BFB0C5C012714F8015B08EB0501DC
:10393000497801F00406F6B2002EE0D111F003013F
:1039400006D0012914BF572137216D1AA945D9DCAA
:10395000791C0BD0C3B9604612B197B9029B1360B2
:1039600005B0BDE8F08F4FF0FF37DDE70399002B7E
:103970000CBF6FF000404FF0004022230B60002A84
:10398000EED0013C0294E9E7CCF1000CE3E714F837
:10399000015B012386E74FF010096578CB460234BE
:1039A00097E700BF30B440F22C04C2F200040D4689
:1039B000134601462A46206830BCFFF751BF00BFBE
:1039C000F8B540F29C14C2F200040F46054601F01F
:1039D00095F8A3685E6826F0030606F6EF73DF1B12
:1039E0003F0B013F3F03B7F5805F07DB002128460F
:1039F00001F010FDA3689B19984204D0284601F0FD
:103A00007FF80020F8BD7942284601F003FD01301F
:103A100010D040F6D423A168C2F20003F61B28465A
:103A200046F001061A684E60D71B1F6001F068F867
:103A30000120F8BD0021284601F0ECFCA368C21A61
:103A40000F2ADBDD40F2A45440F6D421C2F2000478
:103A5000C2F2000142F001025A602368C01A0860F5
:103A6000CCE700BF2DE9F0410E46804600295CD02E
:103A700001F044F840F29C1556F8041CC2F200050F
:103A8000A6F1080421F00103AF68E21897425068DC
:103A900020F0030067D011F00101506035D0002103
:103AA0001618766816F0010F06D11B1890680029C9
:103AB0004DD0D268C260906043F00102E350626072
:103AC000F1B9B3F5007F32D35A0A042A6CD89809A9
:103AD0003830410005EB810540F29C11C2F2000133
:103AE000AA68AA426BD0516821F003018B4202D22E
:103AF00092689542F7D1D368E360A260D4609C607D
:103B00004046BDE8F04100F0FBBF56F8086C05F1F7
:103B1000080CA41B9B19A668664543D0D4F80CC0BA
:103B2000C6F80CC0CCF80860BAE7BDE8F081DB0845
:103B30000121686805EBC3029B1001FA03F3E26000
:103B4000916818436860A160CC609460D8E7294E02
:103B5000B042AED16C6143F001022C61E060A06024
:103B60006260E350CCE7C018CB0707D456F8083C96
:103B7000E41AC018A268E368D3609A6040F2A852C1
:103B800040F00103C2F200026360AC601368984227
:103B9000B6D340F6D0234046C2F200031968FFF7BF
:103BA0000FFFADE701217BE702F15B004100142A22
:103BB00090D9542A0CD8180B6E3041008AE70126A0
:103BC0004D688010134606FA00F005434D6093E7F8
:103BD000B2F5AA7F03D8D80B773041007AE740F2DC
:103BE00054518A4203D8980C7C30410072E7FC2182
:103BF0007E206FE7A401002002694B112DE9F0013E
:103C0000934200F114072DDA043300EB82021432E0
:103C100011F01F0100EB830303F1040C29D05C6851
:103C20000CF104039A42C1F1200824FA01F438D9B6
:103C30003D461E6806FA08F6344345F8044B53F82F
:103C4000044B9A4224FA01F4F3D8CCEB0203053B6F
:103C500023F00303C31818331C60E4B10433DF1BE3
:103C6000BF101AE00023036100234361BDE8F001A7
:103C70007047624584BF63463946F3D953F8044B15
:103C80009A4241F8044BF9D86FEA0C039B1823F0D1
:103C90000303C3181833DF1BBF100761002FE5D1E2
:103CA000E2E73B46D8E700BF45F2A80043F67803B9
:103CB000C0F6040010213022C2F2010399540131F0
:103CC00010F8012FC9B2002AF8D145F2A0001A213C
:103CD000C0F6040061229954013110F8012FC9B2D5
:103CE000002AF8D145F298001A21C0F604004122BA
:103CF0009954013110F8012FC9B2002AF8D1704748
:103D00002DE9F04F8BB0884643F678060692C2F252
:103D100001060993079000F0B9FB00680290FEF7D6
:103D200053FA029B1A1896F83030039012F801AC3F
:103D3000002B00F00E81D8F800309D1C9A78302AB4
:103D400040F00082033300271D4613F8012B013792
:103D5000302AF9D016F802B043F67809C2F2010908
:103D6000BBF1000F00F0F8802B784FF0000B19F832
:103D70000340002C00F000826A1C144601322378B4
:103D8000F35C002BF9D1994620460299039AFEF77D
:103D90007DFAE8B12378BBF1000F00F0C181C4EBDC
:103DA0000B0B4FEA8B020592502B00F09B80702B7F
:103DB00000F098802246C8F80020B9F1000F0DD01D
:103DC000002F0CBF0627002738460BB0BDE8F08F48
:103DD000BBF1000F00F0BE812378E0E7631B49468A
:103DE000013B072B03DD5B100131072BFBDC079840
:103DF00000F088FEA54200F114030490089380F0BF
:103E0000DB819B46039B4FF000084746C3F1010C42
:103E10000FE0202F5FD03A46043714F8013C4C469F
:103E2000A542F35C03F00F0303FA02F348EA030828
:103E300019D214F8013C04F1FF395345E9D109EBDB
:103E40000C039D42E5D818460299039A0193CDF8D8
:103E500000C0FEF71BFA019BDDF800C00028D8D196
:103E60001C46A542E5D3089B40464BF8048B0499B9
:103E7000C3EB0B0B4FEAAB030B615D0100F024FFBA
:103E8000069A1468281AA04200F32581C0F24B81DB
:103E90000025069805998368994200F3F6800698F4
:103EA00005994368994280F200815E1AB44276DC3B
:103EB000C268022A00F06F81032A00F09881012A6B
:103EC00000F0868107985027049900F051FE14985D
:103ED0000023036078E74BF8048B4FF000080427B9
:103EE00042469AE763782B2B00F0F2802D2B00F0EE
:103EF000EA80601C4FF0000BF15C43F67803C2F2DD
:103F0000010300293FF456AF19293FF753AF90F84A
:103F100001C01039421C13F80C3093B1192B10DC7E
:103F2000023001E0192B0CDC024601EB810101306B
:103F300092F800C003EB4101103916F80C30002B49
:103F4000F0D1BBF1000F00D04942059B5B180593EF
:103F500031E7FFF7A9FEEEE628460299039AFEF73D
:103F600095F9002840F09A8003982C182B5C19F8DA
:103F70000320002A00F0E880302B40F00881631C09
:103F80001D4613F8012B302AFAD0B35C002B40F009
:103F9000FF804FF00109A3464F462C46F4E6771EFA
:103FA000002D40F0E780002F04DD0498394601F031
:103FB00005FA054608997B11012207F01F070498AE
:103FC000A41B51F8233002FA07F231461A4218BFF7
:103FD00045F00205FFF710FE069B02275B6805937C
:103FE000002D69D00698C368022B00F0EA80032BED
:103FF0005DD0012B5ED1AA075CD508990B682B43D5
:10400000DB0757D5049B002604991D69089B01EB2B
:1040100085001430194653F8042BB2F1FF3F40F0ED
:10402000EB80984243F8046CF4D8049A93689D425C
:10403000B8BF2B4680F2F980049901EB830201336B
:104040000B6101235361022F00F0D98004990B69A1
:104050009D420EDB14F01F0400F0AC80049B03EBC8
:104060008505286900F030FEC4F12003984280F2F3
:10407000A18004980121FFF7BFFD069A0598936877
:1040800001300590984240F395800798A327049942
:1040900000F06EFD149A0023136095E62B782C46F1
:1040A000CDF814B04FF001097EE6012798E7159B83
:1040B000002BA7D147F01007049B14980360059BC1
:1040C0000998036080E64FF0010BA378A01C13E76A
:1040D0004FF0000BF9E7061B0498314601F06EF92A
:1040E0000546A8B1731E0498012503F01F015A115B
:1040F00005FA01F100EB82025269114208D0AB428D
:1041000005DD0498B11E01F059F9032500B9022517
:1041100004983146FFF770FD059B9B190593B8E69F
:10412000CDF814B040E6251A04992A46079800F005
:1041300011FF059B5B1B00250593049000F1140300
:104140000893A6E6002705E605924FF001092BE645
:104150002C468146039904EB010B635CF25C002A58
:104160007AD00BF10102144612F8013BF15C0029F0
:10417000F9D114E601251DE728460299039AFEF7B6
:1041800085F80028E4D0A1462C46CB4602E6254619
:10419000A3460127F0E5159800287FF493AE099A0D
:1041A00062270498089913600123149A03610B6035
:1041B000106009E621277FE7DDF820B04FF0000806
:1041C00051E6159AC2F10103002B3FF473AF19E7D2
:1041D000A6427FF477AE012CE1DD0498611E01F068
:1041E000EDF800283FF46EAE069A5368D7E71599AC
:1041F00000293FF467AED2E701320A6023E7069A4E
:1042000022271368013BA3427FF456AF6311049841
:10421000012204F01F0400EB830302FA04F25B693D
:104220001A4214BF2127222746E751680798013117
:1042300000F068FC0646049800F10C01036906F1E1
:104240000C009A1C9200FDF72DFD04990798049626
:1042500000F08EFC3369EFE65C46A0E52DE9F04FF7
:1042600043F67808C2F2010885B00C46924698F8E9
:1042700030300290002B00F0AD8023685A1113F00B
:104280001F0303930AEB8202009201D004320092D2
:10429000009A002399460099CB464E4642F8043CCA
:1042A0000439029B0191DDF804C0196864464B781B
:1042B000002B33D018F80320002A6FD1202B00F2F6
:1042C00083805E4526DDB9F1070FCCBF00230123B3
:1042D000644528BF002393B1C9F108092268234629
:1042E0004FEA8909C9F12007586800FA07F5154314
:1042F00020FA09F21D6043F8042F9C45F4D8544578
:1043000098BF4FF0080905D90022043C2260B3464B
:10431000A446914601314B78002BCBD1002E55D0CD
:10432000B9F1070FCCBF00230123644528BF002348
:1043300093B1C9F10809226823464FEA8909C9F1F6
:104340002005596801FA05F0104321FA09F21860B6
:1043500043F8042F6345F4D3A2453ED20198524658
:1043600054F8041B1346A04243F8041B1A46F7D224
:104370000199002243F8042B9942FBD2009951F88D
:10438000043C4BB9019B9A4502D138E09A4537D09D
:1043900053F8042D002AF9D0052018E009F101098D
:1043A0000136B9F1080F07DC23681B0102F00F0288
:1043B00001311A432260AEE75445ABD90023043CD7
:1043C00023604FF00109F1E7292B1DD0042005B02F
:1043D000BDE8F08FFFF768FC4FE7039A002ACDD0C5
:1043E000009A039952F8043CC1F120024FF0FF31CA
:1043F00021FA02F21340009A42F8043CC1E7534606
:10440000012205201A60E2E7029B02311960002EAA
:1044100086D1DBE710B514463AB145F2B801104633
:10442000C0F60401FDF784FD20B945F2B400C0F6E2
:10443000040010BD45F2B4012046C0F60401FDF7AA
:1044400077FD0028F1D045F2C0012046C0F60401F6
:10445000FDF76EFD45F2B403C0F6040300280CBF5F
:104460001846002010BD00BF40F22010C2F200002C
:10447000704700BF40F22013C2F20003186A704771
:1044800000487047440100200020704700487047F2
:104490006401002040F22C030A46C2F200030146E8
:1044A0001868FFF7B7BF00BF0048704764010020DD
:1044B00040F22C030146C2F20003186800F008B86D
:1044C00040F22C030146C2F200031868FFF7CABA93
:1044D0002DE9F04F01F10B04162C83B0074630D9BB
:1044E00024F00704E30F8C422CBF194643F001016E
:1044F00000292FD1384600F001FBB4F5FC7F2ED205
:104500004FEAD40C40F29C16C2F2000606EBCC0235
:10451000D368934200F01182596803F10808DA6801
:10452000384621F0030499681B195C68CA6044F09E
:10453000010491605C6000F0E3FA404603B0BDE81E
:10454000F08F002310248C422CBF194643F0010148
:104550000029CFD00C234FF000083B60EDE75FEA65
:10456000542C04BF4FEAD40C4FEA4C0540F08F8026
:1045700040F29C16C2F2000606EB8505EB689D42F0
:1045800006D10DE0002A80F25581DB689D4207D0FC
:10459000596821F003010A1B0F2AF3DD0CF1FF3CDF
:1045A0000CF1010C40F29C123369C2F2000202F1DC
:1045B000080E734508BFD2F8049022D0586820F046
:1045C0000300011B0F2900F384810029C2F814E0C5
:1045D000C2F810E066DAB0F5007F80F04E81C108C5
:1045E0004FF0010802EBC100891008FA01F8516888
:1045F0008568D86048EA0109C2F804909D60EB60C4
:10460000836001224FEAAC0302FA03F34B4554D80E
:1046100019EA030F0DD193402CF0030C19EA030F94
:104620000CF1040C05D15B000CF1040C19EA030F2A
:10463000F9D006EBCC09E0464846C268904207D163
:104640005BE1002980F28381D268904200F05581BD
:10465000556825F00305291B0F29F2DD9046131933
:10466000D56844F0010058F8084F41F0010C506043
:104670003846C3F804C0E560AC6073613361C3F8C9
:104680000CE0C3F808E0595000F03AFA55E7BCF1E5
:10469000040F00F2DE804FEA941C0CF1380C4FEA54
:1046A0004C0565E71A1803F108083846536843F0CB
:1046B0000103536000F024FA3FE7B5686B6823F00C
:1046C000030A544504D8C4EB0A030F2B00F3A4805B
:1046D00040F6D029D6F80814C2F2000905EB0A0208
:1046E0000131D9F80030234408BF03F1100B06D084
:1046F00003F580530F3323F47F6323F00F0B384609
:104700005946019200F086FE019A411C804600F055
:104710006881824200F23181D9F8043042455B441D
:10472000C9F8043000F06681D6F8081440F29C10F5
:10473000C2F20000013117BFC2EB0802C0F80884C2
:104740009B18C9F8043018F0070338461FBFC3F19F
:104750000802C3F58053904403F1080208EB0B03F1
:1047600008BF4FF480521B051B0DC3EB020B5946CB
:1047700000F050FE431C00F04981C8EB0001594491
:1047800041F00101D9F80430B54240F6D022C6F814
:1047900008805B44C2F20002C8F80410C9F8043073
:1047A00018D0BAF10F0F40F20B81AAF10C00696822
:1047B00020F007004FF0050C05EB000E0F2801F06C
:1047C000010140EA01016960CEF804C0CEF808C0DA
:1047D00000F2208140F6D022D9F82C10C2F200025B
:1047E000B5688B42D9F8301088BFD36240F6D0222A
:1047F000C2F200028B4288BF13636A6822F0030290
:104800009442C4EB020301D80F2B05DC38464FF06D
:10481000000800F075F990E62A1943F0010344F00E
:10482000010438466C6005F108085360B26000F07E
:1048300067F982E65918DA689C6838464D6803F1D2
:10484000080845F00105E26094604D6000F058F9F9
:1048500073E6BCF1140F9CBF0CF15B0C4FEA4C05E6
:104860007FF686AEBCF1540F00F293804FEA143C01
:104870000CF16E0C4FEA4C057AE6420A042A75D90F
:10488000142A9CBF02F15B094FEA490508D9542A52
:1048900000F2C9804FEA103909F16E094FEA490563
:1048A00006EB850540F29C18C2F20008AA68AA42ED
:1048B00079D0516821F00301884202D29268954272
:1048C000F7D1D068D6F80490D8609A60D36083603E
:1048D00097E61D1941F00106556144F00104156188
:1048E00038465C6003F10808C5F80CE0C5F808E03C
:1048F0006E60695000F004F91FE608F10108083005
:1049000018F0030F7FF499AE4A461CF0030FA2F192
:1049100008010CF1FF3C00F09E8012688A42F4D03E
:1049200072685B0093423FF6C8AE002B3FF4C5AE01
:104930001A4200F09580C4467BE603F108025B69E9
:104940009A4208BF0CF1020C3FF42CAEE4E590460D
:104950005519D368384658F8082F6968D36041F074
:1049600001019A60696000F0CBF8E6E54FEA901922
:1049700009F138094FEA490592E7B54240F29C1324
:10498000C2F200033FF4C8AE9D686A6822F00302D9
:1049900036E7BCF5AA7F19D84FEAD43C0CF1770C66
:1049A0004FEA4C05E4E50125D8F804104FEAA909BF
:1049B000104605FA09F545EA0109C8F8049083E7AD
:1049C00001234546C8F80430002219E740F2545349
:1049D0009C450BD84FEA944C0CF17C0C4FEA4C05EB
:1049E000C6E5B5686A6822F0030209E7FC254FF0C6
:1049F0007E0CBDE51105090D00297FF495AEB26866
:104A00000BEB0A0141F001015160E3E601214FF097
:104A1000000BB7E6384605F108010192FFF722F8CE
:104A2000019A5368D6E6B2F5AA7F06D84FEAD03984
:104A300009F177094FEA490532E740F25451FC2564
:104A40008A424FF07E099EBF4FEA904909F17C09E6
:104A50004FEA490524E7726822EA0302726060E7C0
:104A60005B0008F1040863E78307C9B270B440D063
:104A7000541E002A3FD003788B4221D0431C04E00F
:104A800004B30278013C8A421AD013F0030F18468F
:104A900003F10103F4D1032C16D8651E94B10378F9
:104AA0008B420DD0421C002302E004788C4207D0D8
:104AB0009D42104603F1010302F10102F5D10020ED
:104AC00070BC70472046FBE741EA012646EA0646ED
:104AD0000246043013687340A3F1013525EA03034D
:104AE00013F0803F03D1043C032CF1D8D5E71046E6
:104AF000D3E71446CFE71046E2E700BF704700BF98
:104B0000704700BF70B50646446A0D465CB1E26866
:104B10009AB152F82500E0B1016842F82510002250
:104B20000261C26070BD1020FFF7C2FC0023044682
:104B30007062436083600360C360212230460421B9
:104B400000F0FCFC736AE060DA68002AE1D1002022
:104B500070BD01233046194603FA05F4621D920028
:104B600000F0ECFC0028F2D045608460D7E700BF7D
:104B700030B50446456A83B055B139B1636A4A68B5
:104B8000DB6853F82200086043F8221003B030BD00
:104B900010200191FFF78CFC0199606245608560EF
:104BA0000560C560E9E700BF2DE9F0478846D1F808
:104BB00010A082B0814601F1140500242F68013451
:104BC000BEB23F0C02FB063602FB07F303EB1643B3
:104BD000B6B206EB03461B0CA24545F8046BEDDCB0
:104BE00053B1D8F8082092450ADA08EB8A020AF194
:104BF0000101C8F810105361404602B0BDE8F087CB
:104C0000D8F80410484601930131FFF77BFFD8F82C
:104C1000102008F10C010232920004460C30FDF71E
:104C200041F841464846A046FFF7A2FF019BDCE75A
:104C30002DE9F84348F639651F46C3F6E305083306
:104C400006460C46904685FB0310DB17C3EB60005D
:104C5000012837DD012500216D000131A842FBDC70
:104C60003046FFF74FFF089B43610123B8F1090F5E
:104C70000146036122DD04F1090944444D4615F85B
:104C8000013B0A223046303BFFF78EFFA54201462A
:104C9000F5D109EB0804083C47450CDDC8EB0707D4
:104CA000E71914F8013B0A223046303BFFF77CFF3E
:104CB000BC420146F5D10846BDE8F8830A344FF0FE
:104CC0000908E9E70021CBE7034600201A0C01D1CF
:104CD0001B04102013F07F4F01D108301B0213F08A
:104CE000704F01D104301B0113F0404F01D102304D
:104CF0009B00002B02DB5B0001D4202070470130B9
:104D0000704700BF0368024613F0070007D0D907B9
:104D10001FD498071FD49B0802201360704799B2D4
:104D200009B91B0C102013F0FF0F01D108301B0A2A
:104D3000190701D104301B09990701D102309B08E2
:104D4000D90704D45B0801D12020704701301360DB
:104D50007047002070475B0801201360704700BF58
:104D600010B50C460121FFF7CDFE0122446102611E
:104D700010BD00BF2DE9F04F0C460E6985B01569D6
:104D80001746AE4204DA32463C462E460F461546DA
:104D9000A36806EB050861689845C8BF0131FFF7B5
:104DA000B1FE00EB880900F1140309F11409019028
:104DB00000204B4503D243F8040B9945FBD807EB81
:104DC000850504EB86061437143514341436AF42C7
:104DD00057D2019ACDF80890A946CDF80C8002F17F
:104DE000180CA04657F8044BA0B2F0B14246ACF103
:104DF0000403002452F8041B1D681FFA81FA090CF1
:104E00001FFA85FB2D0C00FB0ABA00FB015154442C
:104E100001EB1441A4B244EA01450C0C964243F85C
:104E2000045BE7D81C6057F8044C240C21D05CF8D4
:104E3000041C4246634600250846B2F800A0000C58
:104E400089B29B4604FB0A00451941EA054143F833
:104E5000041C53F8040B52F8041B1FFA80FA090CC7
:104E600004FB01A101EB15410D0C9642E5D8CBF8EE
:104E70000010B9450CF1040CB4D8DDF80890DDF849
:104E80000C80B8F1000F0BDD59F8043CA9F10409BE
:104E90001BB105E059F8043D13B9B8F10108F9D187
:104EA000019B1846C3F8108005B0BDE8F08F00BF25
:104EB00012F003032DE9F041144680460F4628D135
:104EC000A4101AD0D8F82450002D2ED0AE682EB9D8
:104ED00036E0641011D0356895B12E46E007F8D55C
:104EE000394632464046FFF745FF394605464046BB
:104EF000FFF73EFE64102F46EDD13846BDE8F08145
:104F0000314632464046FFF735FF306006460560C1
:104F1000E4E748F610525D1EC0F60302002352F883
:104F20002520FFF741FE0746CAE71020FFF7C0FA29
:104F300000230546C8F82400436083600360C36013
:104F4000404640F27121FFF70BFF0023A8600646A0
:104F50000360C3E72DE9F84F93460A690F464FEA0D
:104F60006B158B6805EB020A81460AF10106496858
:104F70009E4203DD5B0001319E42FBDC4846FFF7A9
:104F8000C1FD002D804600F114040ADD00231A46FD
:104F9000013344F8042BAB42FAD108EB830303F14D
:104FA0001404386907F1140507EB800014301BF076
:104FB0001F0B1CD0CBF120030022296801FA0BF152
:104FC0000A4344F8042B55F8042BA84222FA03F2B2
:104FD000F3D822600AB10AF102064846013E39467A
:104FE000C8F81060FFF7C4FD4046BDE8F88F55F8DB
:104FF000043BA84244F8043BEFD955F8043BA842CF
:1050000044F8043BF3D8E8E703460A69006930B482
:10501000801A0FD1043203F1140592009B188918ED
:105020000433043153F8042D51F8044DA24203D146
:105030009D42F7D330BC7047944294BF01204FF09B
:10504000FF30F7E72DE9F84F8B46044611465846E6
:105050009146FFF7D9FF051E61D0BCBF5B46CB462A
:105060002046B8BF9946DBF80410ACBF4FF00008EB
:105070004FF00108FFF746FDDBF8107009F1140549
:10508000D9F810300BF1140600240BEB870C09EB58
:1050900083090CF1140C09F1140900F1140AC0F889
:1050A0000C8056F8048B534655F804AB32461FFA71
:1050B00088F109191FFA8AFBCBEB01014FEA1A4468
:1050C000C4EB184404EB214489B241EA044124149E
:1050D000A94543F8041B9A46E3D8B445984614D929
:1050E00052F8045BA9B22D0C0C1905EB2445A4B2AF
:1050F00044EA05412C14944543F8041BF0D8F343CB
:10510000634423F0030304334344043B21B953F8BD
:10511000042D013F002AFAD00761BDE8F88F204630
:105120002946FFF7EFFC012345610361BDE8F88FD5
:105130000023C7F6F0730B40A3F15073002B02DD80
:105140001946002070475B4200211B15132B0BDD15
:10515000322B02DD0123184670470122C3F13303CD
:1051600002FA03F3184670474FF40022002042FA77
:1051700003F170472DE9F84300F1140806698946E8
:10518000043600EB86063446374654F8045B28465E
:10519000FFF79AFD0A28C0F12003C9F8003018DC97
:1051A000B045C0F10B0125FA01F738BF54F8084C9F
:1051B00047F07F5747F4401334BF24FA01F1002130
:1051C000153005FA00F541EA050210461946BDE81A
:1051D000F8830021B04502D254F8081C371FB0F103
:1051E0000B0418D005FA04F5C0F12B00474545F033
:1051F0007F5521FA00F645F4401545EA060388BFBD
:1052000057F8045C01FA04F18CBF25FA00F0002085
:1052100040EA0102D9E745F07F550A4645F44013BC
:10522000D3E700BF2DE9F04383B001211D461446AA
:105230000A9FFFF767FCC5F30A5625F07F43A9468E
:1052400023F4700380460EB143F480130193002CC5
:1052500024D002A840F8084D6846FFF753FD019B93
:10526000002831D1009AC8F81420002B0CBF01246B
:105270000224C8F81830C8F81040E6B908EB8403D7
:10528000A0F2324038601869FFF71EFD0B9BC0EB9F
:1052900044101860404603B0BDE8F08301A8FFF752
:1052A00031FD01231C46C8F81030019BC8F81430AA
:1052B0002030002EE2D00B9AA6F23349C0F135031C
:1052C000484438601360E5E7C0F12001009A03FA12
:1052D00001F123FA00F30A430193C8F81420C4E74C
:1052E0002DE9F04383B0884669460646FFF742FF42
:1052F0000D46044601A94046FFF73CFF2F460B46EA
:105300000246D8F810109946306926469046C1EBFF
:10531000000E9DE80300401A00EB4E110029C9BFA2
:1053200005EB0157A3EB015924463D46DCBF12466D
:105330004B4620462946FBF7A9FA03B0BDE8F083A7
:10534000172810B504460CDD00210020C3F6F071CB
:1053500000230022C4F22403FBF76EF9013CF7D1CD
:1053600010BD48F61053C0F6030303EBC003D3E9A6
:10537000040110BD70B40139156902F114034E1116
:10538000013602EB8505143500EB8606AB420CD2E4
:10539000014653F8044B9D4241F8044BF9D8AB1A2F
:1053A000153B23F003030433C018864204D90023BD
:1053B00040F8043B8642FBD870BC704730B44B11B8
:1053C000046900F114029C42B8BF234600DB11DCE3
:1053D000043300EB8300031D9A4218D253F8043CB7
:1053E0002BB9824213D250F8043D002BF9D0012092
:1053F00030BC704711F01F01EAD000EB83046469F0
:1054000024FA01F505FA01F1A142F0D1E0E700200C
:10541000EEE700BF38B543F67404C2F20104054656
:1054200008460023236013F097FB431C00D038BDCF
:105430002368002BFBD02B6038BD00BFC9B2F0B48D
:1054400000294BD083070FD00378002B73D09942EB
:1054500042D0431C05E013F8012B002A3BD09142B7
:105460003AD09A071846F6D1036841EA0127A3F11A
:10547000013247EA074722EA030212F0803F1CD1BB
:105480007B40A3F1013222EA030313F0803F14D1E1
:10549000021D02E014F0803F0FD1104652F8043B89
:1054A000A3F1013687EA030426EA0303A4F10135D8
:1054B00013F0803F25EA0404ECD00378002B3AD0A7
:1054C000994209D0431C01E0914205D0184613F8D7
:1054D000012B002AF8D11046F0BC704781070DD08F
:1054E0000378002BF8D0431C02E00278002AF3D0A6
:1054F00013F0030F184603F10103F6D10368A3F17B
:10550000013222EA030313F0803F0AD1021D104644
:1055100052F8041BA1F1013424EA010111F0803F8B
:10552000F5D00378002BD7D0431C184601330278FE
:10553000002AFAD1D0E71846CEE700BF10B501FB2C
:1055400002F1FEF7C5FF044670B150F8042C22F0BA
:105550000302043A242A1CD8132A98BF034605D80C
:1055600000221A605A609A60204610BD00211B2A52
:10557000016098BF00F108034160F1D9242A8160DD
:10558000C16011BF00F11003016100F11803416116
:10559000E6E70021FCF740FC204610BD21F0004169
:1055A000704700BF40F0BF60024B40F40030D8604D
:1055B000704700BF00ED00E0C3780BB3164B417895
:1055C000DB68DB43C3F30223C3F10402D2B201FA66
:1055D00002F20F2141FA03F38178D2B20B401A4351
:1055E000037803F1604303F56143120183F800235C
:1055F00003780122590903F01F0302FA03F307E0BD
:1056000003780122590903F01F0302FA03F3203142
:10561000024A42F82130704700ED00E000E100E06E
:1056200021F0604121F07F01014B084398607047F1
:1056300000ED00E0014B01229A607047003002400B
:1056400010B50023054C03E050F8232001332260FD
:105650008B42F9D1014B186810BD00BF00300240E9
:10566000044B1A69002A04DA034A5A6002F18832AC
:105670005A607047003C024023016745024B1A699B
:1056800042F000421A617047003C0240014BD86072
:10569000704700BF003C02400B4BDA68D0030DD4CA
:1056A000DA68D1060CD4DA6812F0EF0F0AD1DB68A1
:1056B00013F0020F0CBF082007207047012070472D
:1056C0000520704706207047003C024007B50823BC
:1056D0008DF80730FFF7E0FF8DF807009DF80730E1
:1056E000012BF7D09DF807000EBD000070B50546F0
:1056F0000E46FFF7EBFF082811D1094C236923F46C
:105700004073236123692361236943F0010323610B
:105710002E70FFF7DBFF236923F00103236170BDC7
:10572000003C024070B505460E46FFF7CFFF082843
:1057300013D10A4C236923F440732361236943F492
:1057400000732361236943F0010323612E60FFF797
:10575000BDFF236923F00103236170BD003C0240BB
:1057600070B5064641B1012908D0022914BF4FF493
:1057700040754FF4007503E00D4601E04FF480756D
:10578000FFF7A4FF08281ED10F4C236923F44073B0
:10579000236121690D432561236923F0F803236107
:1057A000236943F002031E432661236943F48033D7
:1057B0002361FFF78BFF236923F002032361236931
:1057C00023F0F803236170BD003C024008B52C4B68
:1057D000984205D10120014600F074F9012048E00B
:1057E000284B984205D10220012100F06BF90220DC
:1057F0003FE0254B984205D10420012100F062F9D9
:10580000042036E0214B984205D10820012100F008
:1058100059F908202DE01E4B984205D11020012196
:1058200000F050F9102024E01A4B984205D12020B6
:10583000012100F047F920201BE0174B984205D1C9
:105840004020012100F03EF9402012E0134B984225
:1058500005D18020012100F035F9802009E0104BAE
:1058600098420BD14FF48070012100F02BF94FF4D6
:1058700080700021BDE8084000F024B908BD00BFD9
:10588000000002400004024000080240000C0240F8
:10589000001002400014024000180240001C0240A8
:1058A000002002402DE9F0470F6800234FF0010C63
:1058B0004FF003080CFA03F202EA0705954231D1D2
:1058C0005A00066808FA02F4E443264006600E799E
:1058D000D0F8009006FA02FA013E4AEA0909012EC0
:1058E000C0F8009015D8866891F80590264086602B
:1058F000866809FA02F949EA06068660466826EAD9
:10590000050545608D79466805FA03F5ADB2354366
:105910004560C5682C40C460CD79C46805FA02F2C0
:105920002243C2600133102BC4D1BDE8F08701834C
:1059300070474183704701F00703C908083130B54B
:105940009B0050F821500F2404FA03F425EA0404C4
:1059500040F8214050F8214002FA03F2144340F885
:10596000214030BD014B1860704700BF20000E423F
:10597000064B002201281A701A7002D0042804D1A4
:1059800001E01870704705221A70704770380240A5
:10599000014B1860704700BF800E47421E4B9A684B
:1059A00002F00C02042A10B503D0082A03D01B4BC6
:1059B00018E01B4B16E059685A6811F4800F5968BB
:1059C00014BF174B154B02F03F02B3FBF2F3124A20
:1059D0005268C2F30142C1F3881101324B435200B5
:1059E000B3FBF2F30C4903608B680E4AC3F3031355
:1059F000D45C036823FA04F343608C68C4F3822404
:105A0000145D23FA04F484608968C1F34231525C66
:105A100023FA02F3C36010BD003802400024F400F2
:105A200040787D01AC05002000F44073B3F5407F61
:105A3000084B08D1996820F0704221F4F81122F443
:105A400040720A439A601A6F000542EA10501867C4
:105A5000704700BF00380240014B1860704700BF1C
:105A60003C0E4742044B1A6B09B1104301E022EA95
:105A700000001863704700BF00380240044B5A6BA7
:105A800009B1104301E022EA00005863704700BFEB
:105A900000380240044B1A6C09B1104301E022EABD
:105AA00000001864704700BF00380240044B5A6C75
:105AB00009B1104301E022EA00005864704700BFBA
:105AC00000380240044B1A6909B1104301E022EA90
:105AD00000001861704700BF00380240044B1A6A8A
:105AE00009B1104301E022EA00001862704700BFCC
:105AF00000380240044B5A6A09B1104301E022EA1F
:105B000000005862704700BF003802404309012B73
:105B1000074A01D1136803E0022B0CBF136F536FC8
:105B200000F01F0023FA00F000F00100704700BFF2
:105B300000380240044B1A6810B142F0040201E040
:105B400022F004021A60704700080650014B986862
:105B5000704700BF00080650002303E001330A38F5
:105B6000DBB2C0B20928F9D840EA0310C0B27047CE
:105B7000020900F00F030A2000FB0230C0B2704798
:105B800082B0002301930D4BDA68500613D44FF016
:105B9000FF32DA60DA680199013101910199B1F5BA
:105BA000803F02F0400201D0002AF3D0034BD868B6
:105BB000C0F3801000E0012002B0704700280040D0
:105BC000024BDA6822F08002DA6070470028004059
:105BD00038B50F4CCA236362532363620546FFF74F
:105BE000CFFF88B1A36823F04003A360A2682B68AD
:105BF0001343A360AB68236123696A6843EA0243E5
:105C00002361FFF7DDFF0120014BFF225A6238BDFF
:105C10000028004082B0002301930E4BCA225A6232
:105C200053225A62DA6822F0A002DA60D968019A37
:105C300001320192019AB2F5003F01F02001054ABC
:105C400001D00029F2D0D068FF235362C0F3401086
:105C500002B0704700280040F8B5244B0C469B6802
:105C600020B913F040032ED1CB702CE013F0400389
:105C70001ED1CB701CE01D4CCA23636253236362A8
:105C8000FFF77EFF80B105F07F3525F0FE452560EA
:105C9000FFF796FFA368990605D4FFF7BBFF003016
:105CA00018BF012000E00120104BFF225A62F8BD0E
:105CB000657823782D0245EA0345A3781D43E378F0
:105CC00045EA0345D7E72078FFF746FF07466078A7
:105CD000FFF742FF0646A078FFF73EFFE57840EA6F
:105CE000054040EA074545EA0625C4E7002800408C
:105CF0000F4B1B6870B5C3F30542C3F3062603F0D0
:105D00007F0503F480031B0C0C460A704E708D70E7
:105D1000CB7058B91046FFF72BFF20703046FFF7C5
:105D200027FF60702846FFF723FFA07070BD00BFFB
:105D300000280040F8B50C464B78002838D103F015
:105D40001002D2B20AB323F010030A334B701CE0E6
:105D50001C4CCA23636253236362FFF711FF80B1B7
:105D600025F07F4525F0C0056560FFF729FFA36892
:105D7000980605D4FFF74EFF003018BF012000E061
:105D80000120104BFF225A62F8BDE078FFF7E4FED5
:105D900007466078FFF7E0FE0646A078FFF7DCFED6
:105DA000257840EA453040EA074545EA0625CFE731
:105DB000CD788A781B0243EA05450B78154345EAFE
:105DC0004335C5E7002800400E4B5B6870B5C3F350
:105DD0000742C3F3042603F03F05C3F342330C46E6
:105DE000CA704E708D700B7058B91046FFF7C0FE28
:105DF000E0703046FFF7BCFE60702846FFF7B8FE43
:105E0000A07070BD0028004082B000230193054BB4
:105E10000193019B03EB80000190019B196002B08C
:105E2000704700BF5028004082B000230193054B0B
:105E30000193019B03EB80000190019B186802B065
:105E4000704700BF502800400A4B1A6C10B59C6880
:105E5000D96802F0040202EAD03200EA04031343D4
:105E600006D08BB213EA10130CBF0020012010BD26
:105E7000184610BD00280040054BDA68C0F30F102B
:105E800040F0800002F0800262EA0002DA607047AF
:105E900000280040014B1860704700BFDC0027421B
:105EA0001C4A038890429BB212D002F58062904255
:105EB0000ED0B0F1804F0BD0A2F58032904207D0C7
:105EC00002F58062904203D002F58062904203D1D5
:105ED0004A8823F0700313430F4A904208D002F51A
:105EE0008062904204D023F440730A899BB213432A
:105EF00003804B68C3620B880385064B984203D02E
:105F000003F58063984201D18B7A03860123838253
:105F1000704700BF0000014000100040038819B125
:105F20009BB243F0010303E023F001031B041B0CAD
:105F30000380704783899BB20AB1194301E023EAC9
:105F4000010181817047C9430182704708B5234B25
:105F5000984205D110200121FFF7CCFD102037E039
:105F60001F4B984207D14FF400300121FFF7B6FDD7
:105F70004FF4003009E01B4B98420BD14FF48020C6
:105F80000121FFF7ABFD4FF480200021BDE8084060
:105F9000FFF7A4BD144B984207D14FF40020012114
:105FA000FFF79CFD4FF40020EFE7104B984207D11C
:105FB0004FF480100121FFF791FD4FF48010E4E7CA
:105FC0000B4B984209D120200121FFF793FD20209F
:105FD0000021BDE80840FFF78DBD08BD001001405D
:105FE0000044004000480040004C00400050004089
:105FF00000140140038ACA889BB223F4405330B591
:1060000013430D46038283890989AA8823F4B05378
:106010000A43698923F00C031B040A431B0C92B248
:1060200013438381838AAA899BB223F44073134369
:1060300085B0838204466846FFF7B0FC194B9C424A
:1060400003D003F580639C4201D1039B00E0029BD7
:10605000A28912B2002A4FF019012A6801FB03F14C
:1060600001DA520000E092006423B1FBF2F1B1FBCF
:10607000F3F21201100903FB1011A08900B20028ED
:1060800006DAC9003231B1FBF3F303F0070305E090
:1060900009013231B1FBF3F303F00F031A432281FC
:1060A00005B030BD00100140838919B19BB243F4A3
:1060B000005303E023F400531B041B0C838170473F
:1060C000C1F3421310B5012401F01F01A34204FAE9
:1060D00001F101D10C3004E0022B01D1103000E0BD
:1060E000143003680AB1194301E023EA0101016099
:1060F00010BD10B5C1F34214012201F01F03012CA1
:1061000002FA03F201D1838903E0022C0CBF038A57
:10611000838A9BB21340028892B243B10123090AD9
:1061200003FA01F111420CBF0020012010BD1846F6
:1061300010BD090A012303FA01F3DB430380704712
:10614000354B1A6842F001021A6000229A60196801
:1061500021F0847121F48031196030495960196847
:1061600082B021F480211960DA60009201921A68ED
:1061700042F480321A601A6802F400320192009AE6
:1061800001320092019A1AB9009AB2F5A06FF2D1C9
:10619000214B1B6813F4003318BF01230193019BAB
:1061A000012B33D11C4B1A6C42F080521A641C4AEA
:1061B000116841F4804111609A689A609A6842F4CB
:1061C00000429A609A6842F4A0529A60154A5A6056
:1061D0001A6842F080721A6019680F4A8901FBD56B
:1061E000114B40F205611960936823F0030393603B
:1061F000936843F0020393609168074B01F00C0130
:106200000829F9D11A6842F400221A60074B4FF0AE
:1062100000629A6002B070470038024010300024DB
:106220000070004019544007003C024000ED00E0BF
:106230004B00DBB270B50324056804FA03F4E443B1
:1062400025400560066802F0030505FA03F53543AD
:1062500005604668012505FA01F526EA0505456051
:106260004568C2F3800606FA01F12943416081685E
:10627000214081608568C2F3011101FA03F12943CD
:106280008160C1680C40C460C168C2F3811202FA27
:1062900003F30B43C36070BD10B5134B03EBC00297
:1062A00053F830301279072A0ED892001C6AD2B205
:1062B0000F2000FA02F024EA00001862186A01FABE
:1062C00002F202431A6210BD083A92005C6AD2B22E
:1062D0000F2000FA02F024EA00005862586A01FA1E
:1062E00002F202435A6210BDC00500200E4B03EBC0
:1062F000C002D28802F0100292B20AB181F001010C
:10630000C20041B153F830109B1801221B7902FAE8
:1063100003F30B83704753F830109B1801221B794D
:1063200002FA03F34B837047C005002070B51E4E80
:1063300006EBC0050446E98801F400739BB23BB14B
:10634000890AFFF7A9FF56F834002979322205E0BF
:10635000CB0707D556F8300029793022BDE87040C8
:10636000FFF766BF01F002039BB223B156F830007D
:10637000297970220DE001F004039BB29BB101F07A
:1063800020018AB256F830002979002A0CBF312248
:106390003522FFF74DFFE9882046C1F3C001BDE873
:1063A0007040FFF7A3BF70BDC005002038B512488C
:1063B000124DFFF70BFA1248FFF708FA1148FFF7E2
:1063C00005FA1148FFF702FA1048FFF7FFF9104BE2
:1063D0001A6B42F01F021A63002405EBC403DB882A
:1063E00003F080039BB213B9E0B2FFF79FFF0134C3
:1063F000112CF2D138BD00BF00000240C0050020C2
:106400000004024000080240000C0240001002405C
:1064100000380240064A52F8303002EBC002596997
:106420001279012000FA02F24A405A61704700BF17
:10643000C00500200E4901EBC00210B5D38803F05F
:106440008004A4B294B951F830101279086901217E
:1064500001FA02F1014003F01003D1409BB20CBFDE
:10646000002001201BB180F0010010BD002010BDF4
:10647000C005002008B540200121FFF7FFFA0120E8
:10648000BDE80840FFF756BBFFF760BB2DE9F047BA
:10649000012903460E46C07937D11C7A5D7A93F8FC
:1064A00000800A22010900F00F0002FB010021090F
:1064B00004F00F0402FB01412C0905F00F0502FB5B
:1064C00004545D794FEA151C05F00F0502FB0C5CC6
:1064D0001D792F0905F00F0502FB07574FEA181524
:1064E00008F00F0802FB058593F806804FEA18199B
:1064F00008F00F0802FB0982C0B2C9B2E4B25FFA29
:106500008CFCFFB2EDB2D2B206E0197A5C7A93F855
:1065100005C01F791D789A79632C6CD800296AD040
:106520000C2968D8002866D014F0030F0AD104F5AE
:10653000FA694FF0640899FBF8FA08FB1A98B8F169
:10654000000F0CD104F5FA644FF4C87894FBF8F905
:1065500008FB1944D4F1010438BF002400E00124F1
:10656000DFF8A8804FF00C0909FB0484611811F8CA
:10657000011C81423FD3BCF1170F3CD83B2F3AD8C6
:106580003B2D38D8002A36D0072A34D85A791B4DEB
:106590001B4C2A701A791B486A701A78AA70DA792B
:1065A000A2701A7A62705A7A9B79E2701F220027D1
:1065B000426002F57872237007608260FFF708FB83
:1065C000012E05D130462946FFF746FB304604E050
:1065D00038462946FFF740FB38462146FFF7AAFB1D
:1065E000094B186840B1132044F22131FFF70CFC2D
:1065F0000020BDE8F0870120BDE8F0874CC80020EE
:106600005CC8002050C80020040B00204806002071
:1066100030B5002285B013460A2506E005FB0212BC
:10662000303A013302F0FF02DBB2C15CA1F1300469
:10663000092CF3D901338DF80720DBB200220A259B
:1066400006E005FB0212303A013302F0FF02DBB232
:10665000C15CA1F13004092CF3D901338DF8082075
:10666000DBB200220A2506E005FB0212303A0133B4
:1066700002F0FF02DBB2C15CA1F13004092CF3D9B6
:1066800001338DF80920DBB200220A2506E005FB64
:106690000212303A013302F0FF02DBB2C15CA1F119
:1066A0003004092CF3D901338DF80620DBB2002227
:1066B0000A2506E005FB0212303A013302F0FF0220
:1066C000DBB2C15CA1F13004092CF3D901338DF8A0
:1066D0000520DBB200220A2506E005FB0212303A53
:1066E000013302F0FF02DBB2C15CA1F13004092CDE
:1066F000F3D901338DF80420DBB200220A2506E02D
:1067000005FB0212303A013302F0FF02DBB2C15C3A
:10671000A1F13004092CF3D904A8002100F8102DB0
:106720006846FFF7B3FE05B030BD08B550B901208B
:10673000FFF72EF96120FFF7E9F90028FAD04FF4AE
:1067400000700AE001280AD1FFF712F94120FFF793
:10675000DDF90028FAD04FF48070FFF765F90120C9
:10676000FFF77AF9FFF756FA132041F23421BDE81A
:106770000840FFF749BB00002DE9F041427A40F2A2
:10678000B27302F5FA6200214FF4C87564269C07C3
:1067900008D1B3FBF6F406FB1434A4B214B14FF4E1
:1067A000B77408E0B3FBF5F405FB1434A4B2002C75
:1067B000F5D040F26D1401339BB293422144E6D3ED
:1067C0006423B2FBF3F703FB17239FB24FF4C873A4
:1067D000B2FBF3F403FB1424A4B2D4F1010438BFD8
:1067E0000024067ADFF858C0002302F003024FF0BD
:1067F0000C080CE022B9002F0CBF2546012500E053
:10680000254608FB053501331CF8055049195D1C68
:10681000ADB2B542EED3C3794479013B591803793F
:106820009A009B019A1A4FF4616303FB04230278D8
:1068300002489B1800FB0130BDE8F0818051010047
:106840004806002038B504460D4609B9084600E060
:1068500001201149FFF74CFA0F4B1A7862715A78F0
:106860009B78227123700D4B9B6A63800DB928467B
:1068700000E001200A49FFF7A7FA094BDA786272B3
:106880005A7822729A781B78E271A3712046FFF73A
:1068900073FFE06038BD00BF4CC8002000280040F6
:1068A0005CC80020F0B5012185B005464FF080504E
:1068B000FFF7F0F80120FFF755F81320FFF7B4FABF
:1068C00044F221339842254E13D1306015B9284641
:1068D000FFF72BFFFFF79EF94FF48040FFF7CCFA4C
:1068E0001F4B4FF480025A6168460021FFF7AAFF50
:1068F0002FE041F23427B8420FD1306015B9284655
:10690000FFF713FFFFF786F94FF48040FFF7B4FA63
:10691000134B4FF480025A611BE000242846346078
:10692000FFF703FF04A8012300F8104D2146684635
:106930008DF807308DF806308DF808308DF8094055
:106940008DF805408DF80440FFF7A0FD3760204624
:1069500001E0024B186805B0F0BD00BF040B002039
:10696000003C01403C23F0B5B1FBF3F4B4FBF3F27F
:10697000C16003FB1411017003FB12431821037162
:10698000B2FBF1F301FB13224271D91C0722B1FBC8
:10699000F2F402FB14120132827140F26D1540F2E2
:1069A000B2724FF4C871642412F0030605D1B2FB31
:1069B000F4F704FB1727BFB22FB9B2FBF1F701FBC5
:1069C0001727BFB227B9AB420BD9A3F5B77305E0C0
:1069D000B3F5B67F05D96FF4B6769B19013292B242
:1069E000E2E702F130014172002101726421B2FB41
:1069F000F1F701FB17218FB24FF4C871B2FBF1F42C
:106A000001FB142292B20C4C12E006B907B922B96C
:106A100065182D7BAB4200D307E0655CAB4204D226
:106A2000013101330172C371F0BD01315B1B017291
:106A3000017A0B29E9D9F3E748060020000000009D
:106A400010B588B0044600216846FFF7FBFE2046DB
:106A5000F9F79EFD08A3D3E90023F9F7EDFDFAF756
:106A600085F80399411804A8FFF77CFF04A80021CA
:106A7000FFF70CFD08B010BD000000000020AC4086
:106A80001FB501466846FFF76DFF68460021FFF716
:106A9000FDFC05B000BD70477047704708B54FF466
:106AA0008040FFF7D1F928B14FF48040FFF7E4F9B7
:106AB000FFF7F1FF024B4FF480025A6108BD00BF9F
:106AC000003C014008B54FF48050FFF7BDF928B1F4
:106AD0004FF48050FFF7D0F9FFF7DEFF4FF400507E
:106AE000FFF7B2F928B14FF40050FFF7C5F9FFF7EF
:106AF000D4FF024B4FF400325A6108BD003C014004
:106B000030B5002285B013460A2506E005FB0212C7
:106B1000303A013302F0FF02DBB2C15CA1F1300474
:106B2000092CF3D901338DF80720DBB200220A25A6
:106B300006E005FB0212303A013302F0FF02DBB23D
:106B4000C15CA1F13004092CF3D903338DF808207E
:106B5000DBB200220A2506E005FB0212303A0133BF
:106B600002F0FF02DBB2C15CA1F13004092CF3D9C1
:106B700002338DF80920DBB200220A2506E005FB6E
:106B80000212303A013302F0FF02DBB2C15CA1F124
:106B90003004092CF3D901338DF80520DBB2002233
:106BA0000A2506E005FB0212303A013302F0FF022B
:106BB000DBB2C15CA1F13004092CF3D900238DF8BC
:106BC00000309DF809308DF80420013368468DF8B7
:106BD0000930FFF7D1FD024B186005B030BD00BF92
:106BE0005028004007490A89064B02F0020292B27F
:106BF000002AF8D098811A89D207FCD5014B9889D0
:106C0000C0B270470038004010B50446C0F30740DA
:106C1000FFF7E8FFC4F30720FFF7E4FFE0B2BDE8A9
:106C20001040FFF7DFBF70B505460C460520002178
:106C30001646FFF75BFB5A20FFF7D4FF2846FFF705
:106C4000E3FF0020FFF7CEFFA61904E00020FFF7C6
:106C5000C9FF04F8010BB442F8D105200121FFF768
:106C600045FB002070BD052008B50021FFF73EFB65
:106C70000520FFF7B7FF0020FFF7B4FF00F0020088
:106C8000C0B20028F7D005200121BDE80840FFF779
:106C90002DBB052008B50021FFF728FB0520FFF7D5
:106CA000A1FF0020FFF79EFFC107FAD405200121B4
:106CB000BDE80840FFF71ABB70B505460C46052035
:106CC00000211646FFF712FB0320FFF78BFF284633
:106CD000FFF79AFFA61904E00020FFF783FF04F8EE
:106CE000010BB442F8D105200121FFF7FFFA4FF064
:106CF000FF3070BDC3B270B51446D218FF2A88BFEA
:106D0000C3F5807406460D4605200021FFF7EEFA14
:106D10000620FFF767FF05200121FFF7E7FAFFF7DD
:106D2000A2FF00210520FFF7E1FA0220FFF75AFF3A
:106D30003046FFF769FF2E1903E015F8010BFFF746
:106D400051FFB542F9D105200121FFF7CFFAFFF736
:106D5000A0FFA0B270BDF8B507460E461546002448
:106D6000381931192A1B0023FFF7C4FF2418A54244
:106D7000F6D10020F8BD10B5002104460520FFF72C
:106D8000B5FA0620FFF72EFF05200121FFF7AEFA26
:106D9000FFF769FF00210520FFF7A8FA2020FFF781
:106DA00021FF2046FFF730FF05200121FFF79EFA63
:106DB000FFF76FFF002010BD30B5484B002485B0B1
:106DC0001C70474B02941A6C42F480421A641A6A8F
:106DD00042F400421A621A6A22F400421A62A3F5CF
:106DE000003303AD1A8822F040021204120C1A80FC
:106DF0004FF441721A809C801A8892B242F040028D
:106E00001A80204604222946FFF70DFF9DF80C301A
:106E1000532B01D000205EE09DF80D30462BF9D1B8
:106E20009DF80E30442BF5D19DF80F30502BF1D149
:106E3000062029460122FFF7F6FE08231AE00198F2
:106E400029460122FFF7EFFE9DF80C307BB904A91B
:106E5000032251F80C0D0430FFF7E5FE01980422DF
:106E6000043002A9FFF7DFFE002809DAD2E7019B10
:106E70000134083301939DF80C309C42DFD9E6E7DA
:106E8000029B002BC6D00024254601988DF80C509B
:106E90001C300222001903A9FFF7C5FE002811DBF0
:106EA0009DF80C2072B10D4B012101FA02F15960DD
:106EB0009DF80D10197202990332013121FA02F284
:106EC0005A8102E00234082CDFD1044B5A68002AB0
:106ED000A0D00120187005B030BD00BF7CC80020D4
:106EE0000038024000F00700C0F10703021D042B28
:106EF00028BF0423062A01D9033800E0002001221C
:106F000002FA03F3013B03F0050303FA00F07047B4
:106F100070B5344DBDF810602B81092A0CBF4FF4B9
:106F2000805200220C23EE80002604466B812960EB
:106F3000AA80AE81FFF70AF82B4B9C4211D103F5D2
:106F400094335A6C42F010025A64284BD868C0F34C
:106F50000220FFF7C7FF264B000183F825032022FC
:106F600028E0244B9C4211D103F5FA331A6C42F409
:106F700000321A641D4BD868C0F30220FFF7B2FF3D
:106F80001B4B000183F82603402213E01A4B9C425E
:106F900027D103F5F8331A6C42F480221A64134B9C
:106FA000D868C0F30220FFF79DFF114B000183F862
:106FB000270380225A6020462946FFF71BF8204607
:106FC0000121FFF771F82046012240F22551FFF719
:106FD00077F8204640F227713246BDE87040FFF74F
:106FE0006FB870BDC8CB00200010014000ED00E07C
:106FF00000E100E0004400400048004007B50021E7
:10700000642003F0B3FF0A4B0A49186064220A485F
:1070100002F0A6FB64220948094902F0A1FB002303
:10702000009308484FF416610822FFF771FF0EBD68
:10703000D8CB002098C80020B8CB002088C80020FA
:1070400028CA0020004400400F4A938923F080039F
:107050001B041B0C70B506460D469381002408E006
:107060000A4802F083FB30B9315D0848013402F070
:107070009EFBAC42F4DB044B9A8992B242F0800250
:107080009A81204670BD00BF00440040B8CB00206C
:10709000094B07B50021024618680B4604F0BCF8FE
:1070A000019028B1054801A902F06CFB019801E0AC
:1070B0004FF0FF300EBD00BFD8CB002088C80020A5
:1070C00013B500230193264B1A8802F0080292B2EE
:1070D00012B19B889BB20193214C40F2277120464C
:1070E000FFF707F8C0B11F4801A902F04BFB18B128
:1070F000BDF80430A3800AE0A38923F080031B04B9
:107100001B0CA381A3899BB243F02003A3811448E5
:1071100040F22771FFF70DF8114C40F2255120463F
:10712000FEF7E7FFD8B1A3880F489BB2019302F0A6
:107130001DFB18B90C48019902F039FB08480B4CAB
:1071400040F22551FEF7F5FF094B2146186804F07F
:1071500031F823681BB1074B4FF080521A601CBDF9
:1071600000440040B8CB002088C80020080B002055
:10717000D8CB002004ED00E07047FFF7A1BF7047B7
:107180001FB5FFF73BFF02F0B1FA01F06FFD01F010
:10719000CFFF38B101F02CFC01F014FD032037497A
:1071A00002F0B8FF002401F01FFF8022234634497B
:1071B0000094019402940394324804F037F901F0EA
:1071C0006FFF802223463049009401940294039477
:1071D0002E4804F02BF90120FFF764FB80222346A0
:1071E0002B4900940194029403942A4804F01EF958
:1071F000FFF740F911F030F810F040FA05F078F997
:1072000010F0ECFD80222346009401940294039434
:107210002149224804F00AF92346214900944FF4F9
:10722000C0720194029403941E4804F0FFF810F019
:1072300071FE1D4B009401930294234603941B4955
:107240001B484FF4807204F0F1F81A4900944FF48F
:1072500080722346019402940394174804F0E6F8E0
:107260004FF47A6004F07CFB01F034FD204604F01A
:10727000B5F904B0BDE8104004F0D2BD388E030863
:107280005B8E03080D900208658E03081D910208AD
:107290006D8E0308C99E0208798E0308757B03086A
:1072A000878E0308D57C03080C0B0020948E0308FE
:1072B000E17F0308A38E0308997F03081FB5224CC2
:1072C00000212046FEF72AFE20460121FEF73BFE64
:1072D00072B64FF000604FF40031FEF7A1F91B4A7F
:1072E000D1684FF6FF030B4043F0BF6343F4003314
:1072F000D3604FF44070FEF755F962B601214FF4A8
:107300008050FEF7AFFB4020FEF7C0F98020FEF76B
:10731000BDF90024FFF74AF801F01CFEFFF74CFD11
:10732000002002F02FFE0A4900944FF47A7223469F
:10733000019402940394074804F078F804F0A8F943
:10734000204604B010BD00BF001C004000ED00E06E
:10735000B68E030881710208704700002DE9F74FCF
:1073600090E80808D0F808A0D0F80C90D0F8108069
:1073700047698669C56901930446164800F0C0FB59
:10738000154800F0BDFB1548214600F0B9FB019BF4
:107390001348194600F0B4FB1248594600F0B0FB00
:1073A0001148514600F0ACFB1048494600F0A8FBDC
:1073B0000F48414600F0A4FB0E48394600F0A0FB00
:1073C0000D48314600F09CFB0C48294600F098FB24
:1073D000FEE700BFBF8E0308CC8E0308DB8E0308D8
:1073E000F18E0308078F03081D8F0308338F0308EE
:1073F000498F03085F8F0308758F03088B8F03087D
:107400001EF0040F0CBFEFF30880EFF30980DFF8E4
:10741000041008475D730208FEE7FEE7FEE77047C9
:107420007047000007B500234020019311F0B2F926
:10743000012804D1094B01A9186803F0BBFE4020C4
:1074400011F0BEF94FF4803011F0BAF9019B1BB175
:10745000034B4FF080521A600EBD00BF0CC80020D5
:1074600004ED00E02DE9F84FD368D2F810B0814662
:107470008A4690461E4600270124002506E004FBAC
:1074800007F306FB0533A4FB06455D194846514644
:1074900022462B46F9F7D6FEB94208BFB042EED2DB
:1074A00000262DE022462B4648465146F9F7CAFEF3
:1074B000514622462B4607464846F9F7C3FE20466A
:1074C000294691469A46D8F80C200023F9F7BAFECF
:1074D00004460D4626B9002F02DC54EA0503E1D12B
:1074E000092FFAB207DD98F8003013F0040F0CBF33
:1074F0005723372300E030239B180BF8013B01365C
:1075000054EA0503CED100238BF80030BDE8F88F94
:1075100070B5CA680C69012300E05343B0FBF3F572
:107520009542FAD200251AE0CE68B0FBF3F203FBD5
:107530001200B3FBF6F31DB9002A01DC002BF3D1D6
:10754000092AD6B206DD0A7812F0040F0CBF5722C2
:10755000372200E03022921904F8012B0135002B6C
:10756000E2D1237070BD70B5CA680C69012300E0D8
:107570005343B0FBF3F59542FAD200251AE0CE68EA
:10758000B0FBF3F203FB1200B3FBF6F31DB9002AC4
:1075900001DC002BF3D1092AD6B206DD0A7812F0FD
:1075A000040F0CBF5722372200E03022921904F852
:1075B000012B0135002BE2D1237070BD2DE9F04184
:1075C0001369546806460F46154600E0013C13F85F
:1075D000012B12B92B7A1BB903E0002CF6DCF9E77A
:1075E000013C2B78990707D5EB68102B01D1023CA1
:1075F00002E0082B08BF013C2B7813F0090F0DD1D6
:10760000A04604E030462021B84708F1FF38B8F121
:10761000000FF7DC631E24EAE4741C1B297A09B10D
:107620003046B8472B789A0712D5EB68102B0AD151
:1076300030213046B8472B7813F0040F30460CBF8A
:107640007821582103E0082B02D130463021B84779
:107650002B78DB070DD5A04604E030463021B84733
:1076600008F1FF38B8F1000FF7DC631E24EAE47478
:107670001C1BD5F8108001E03046B84718F8011BF4
:107680000029F9D12B7803F00903082B06D103E078
:1076900030462021B847013C002CF9DCBDE8F081E0
:1076A0008368026893423CBF4268D15483680133C7
:1076B0008360704790E80C00D154013343607047F9
:1076C0002DE9F04F9BB0174604AA05460E461C460E
:1076D0000E9208E2252900D03AE19DF828200023E7
:1076E00002F0FC0263F3C3028DF828200221D2B21B
:1076F00002F0010CC2F340000B938DF830308DF88E
:107700003C10C2F3C00212E02D290FD004D8232967
:1077100008D02B290FD107E0302900D00BE04FF023
:10772000010C04E0012002E0012300E0012217F82F
:10773000011B0029E8D19DF828808DF830306CF3CA
:107740000008C44660F3410C6046A1F1300362F3C7
:10775000C300092B8DF828001DD804E000FB02327D
:1077600017F8011B01E000220A20A1F130035FFAA3
:1077700083FCBCF1090FF1D9A1F16103052B02D8FB
:10778000A1F15703B5E1A1F14103052B02D8A1F105
:107790003703AEE10B922E290ED13A78303AD2B2AD
:1077A0007B1C092A98BF8DF83C2013F8011BA1F11E
:1077B0003002092A1F46F8D97A2902D117F8011B8D
:1077C00005E06C2909D139786C2902D001370123F1
:1077D00004E079780223023700E00023692936D0DB
:1077E00016D8632900F0A1800CD8462900F0B38098
:1077F00006D8002900F08181252940F07481A7E096
:10780000582912E0642922D0662940F06C81A2E058
:10781000732900F0908005D86F2978D0702940F046
:10782000628140E0752903D0782940F05C8141E015
:107830000A22022B0D9207D1073424F0070303F12B
:107840000804D3E9000117E020680AA94FE00A22E2
:10785000022B0D9212D1073424F00703D3E9000163
:1078600003F10804002871F1000305DA2D234042DA
:1078700061EB41018DF830300AAA33E0012B20681A
:1078800004F1040807D1002803DA2D2340428DF8C3
:1078900030300AA92FE0002803DA2D2340428DF86A
:1078A00030300AA92AE09DF8283043F002038DF811
:1078B000283000231022B1F1580EDEF100019DF8AE
:1078C00028000D9251EB0E011AAA61F38200022BDF
:1078D00002F8400D09D1073424F00703D3E9000171
:1078E00003F10804FFF7BEFD0BE020681146012BF1
:1078F00004F1040802D1FFF70BFE01E0FFF733FEAD
:107900004446284631460AAAFFF758FEEBE0082312
:1079100020680D930AA9FFF726FE284631460AAAD9
:1079200004F10408FFF74AFE10E02846217804F12C
:107930000408B0470AE023680AAA284631460E9395
:10794000FFF73CFE04AA04F104080E924446CAE084
:107950002846B047C7E0073424F0070303F10804C2
:1079600093E8040400921046514600220023F9F7E0
:10797000D5F838B10B9B013B0B930AF1004A4FF04D
:10798000010B09E09DF830302BB10B9B013B0B93B1
:107990004FF0020B00E09B4651460098F9F7E6F8DD
:1079A0000022019080460A2108E098FBF1F010AB1C
:1079B00001FB108843F8228001328046B8F1000FA5
:1079C000F3D102F1FF3912B90B9A013A0B929DF8EB
:1079D0002820D0071BD5BBF1010F02D128462D214D
:1079E00007E0BBF1020F05D128462B2101E0284614
:1079F0003021B0479DF83C200B9B4A440232591E6F
:107A000093420B91F3DC17E028462021B0479DF804
:107A10003C100B9A49440231501E8A420B90F3DC11
:107A2000BBF1010F02D128462D2104E0BBF1020F6A
:107A300002D128462B21B047B9F1FF3F02D1284699
:107A4000302107E010AB284653F82910303109F1F6
:107A5000FF39C9B2B047B9F1FF3FF3D128462E2113
:107A6000B0474FF001091DE00A23019803FB09F913
:107A7000F8F77CFD02460B4600985146F8F728FCC3
:107A8000CDE902014846F8F771FD02460B46DDE9F3
:107A90000201F8F7D1FDF9F769F8804610B92846D8
:107AA0003021B0479DF83C305A1E8DF83C20002B09
:107AB000DAD10A2208E098FBF2F110A802FB118843
:107AC00040F8238001338846B8F1000FF3D198467F
:107AD00006E010AB284653F828103031C9B2B04741
:107AE00018F1FF38F5D217F8011B00297FF4F2AD29
:107AF00003E00A2B7FF732AE4CE61BB0BDE8F08FF7
:107B00000FB407B5064904AB0868064953F8042BBF
:107B100009680193FFF7D4FDBDE80E4004B070473B
:107B2000140B0020100B00201FB5002481B1013977
:107B30000290019101A808490394FFF7C1FD039940
:107B4000019B029A994234BF5454D454039800E0E4
:107B5000084604B010BD00BFA17602080CB407B5FA
:107B600004AB53F8042B0193FFF7DEFFBDE80E4092
:107B700002B0704737B50D461346009000246846A2
:107B80002A4604490194FFF79BFD9DE80C00D4545C
:107B900001983EBDB57602080EB403B503AA52F8AB
:107BA000041B0192FFF7E6FFBDE80C4003B07047ED
:107BB00038B5084B044618680D46F8F7E9FC02464C
:107BC0000B4620460449FFF7E7FF2046FAF7FCFA88
:107BD000287038BDA0CF0020A18F030838B5084B0E
:107BE000044618680D46F8F7D3FC02460B462046BB
:107BF0000449FFF7D1FF2046FAF7E6FA287038BDAE
:107C0000A0CF0020A18F030838B5084B0446586860
:107C10000D46F8F7BDFC02460B4620460449FFF727
:107C2000BBFF2046FAF7D0FA287038BDA0CF00205D
:107C3000A18F030838B5084B044698680D46F8F73D
:107C4000A7FC02460B4620460449FFF7A5FF204645
:107C5000FAF7BAFA287038BDA0CF0020A18F030828
:107C600038B5064B05460C461A7C0549FFF794FFCC
:107C70002846FAF7A9FA207038BD00BFA0CF00202F
:107C8000A78F030838B5064B05460C465A7C0549B4
:107C9000FFF782FF2846FAF797FA207038BD00BF39
:107CA000A0CF0020A78F030838B5064B05460C4629
:107CB0009A7C0549FFF770FF2846FAF785FA20708D
:107CC00038BD00BFA0CF0020A78F030838B5084BF0
:107CD0000446D8680D46F8F75BFC02460B46204682
:107CE0000449FFF759FF2046FAF76EFA287038BDAD
:107CF000A0CF0020A18F030838B5064B05460C46DF
:107D00001A7D0549FFF748FF2846FAF75DFA20700B
:107D100038BD00BFA0CF0020A78F030838B5084B9F
:107D200093F82D3005460C460BB1064900E0064994
:107D3000FAF7ECF92846FAF747FA207038BD00BF89
:107D4000A0CF002053900308DF92030838B5064BFC
:107D500005460C46DA7C0549FFF71EFF2846FAF770
:107D600033FA207038BD00BFA0CF0020A78F0308D2
:107D700030B587B004460D4602A80021FEF762FD2B
:107D80009DF80F109DF811209DF81030009102F51C
:107D9000FA6205492046FFF7FFFE2046FAF714FA7B
:107DA000287007B030BD00BFAA8F030830B585B07A
:107DB00004460D4668460021FEF744FD06499DF83D
:107DC00005209DF804302046FFF7E6FE2046FAF72E
:107DD000FBF9287005B030BDF08F030830B585B0D1
:107DE00004460D4668460021FEF72CFD0549039A1E
:107DF0002046FFF7D1FE2046FAF7E6F9287005B0D5
:107E000030BD00BFA78F030838B5084B93F8403347
:107E10000C46054606490BB1064A00E0064AFFF744
:107E2000BBFE2846FAF7D0F9207038BDDCCB002025
:107E30002C040408DF9203085390030838B5054A60
:107E400005460C460449FFF7A7FE2846FAF7BCF999
:107E5000207038BD1DCF00202C04040838B5094B14
:107E60000446D3F870030D46F8F792FB02460B4622
:107E700020460549FFF790FE2046FAF7A5F928703D
:107E800038BD00BFDCCB0020A18F030838B5054A00
:107E900005460C460449FFF77FFE2846FAF794F999
:107EA000207038BD2DCF00202C04040838B5074BB6
:107EB0009A1805460C4692F876230549FFF76CFEA2
:107EC0002846FAF781F9207038BD00BFDCCB0020CE
:107ED000A78F0308063238B50446D0B20D4601F02C
:107EE0002AF9054902462046FFF756FE2046FAF7D2
:107EF0006BF9287038BD00BFA78F030838B504465A
:107F000006200D4601F017F9044902462046FFF706
:107F100043FE2046FAF758F9287038BDA78F0308AA
:107F200038B5074B9A1805460C4692F87423054954
:107F3000FFF732FE2846FAF747F9207038BD00BF38
:107F4000DCCB0020A78F0308073238B50446D0B237
:107F50000D4601F0F0F8054902462046FFF71CFEE9
:107F60002046FAF731F9287038BD00BFA78F030803
:107F700038B5044607200D4601F0DDF804490246F5
:107F80002046FFF709FE2046FAF71EF9287038BD93
:107F9000A78F030838B5044608200D4601F0CBF83A
:107FA000044902462046FFF7F7FD2046FAF70CF990
:107FB000287038BDA78F03087FB5044603A80E4676
:107FC0000CF0BEF803980C4B0C4DB0FBF3F203FB26
:107FD0001200B0FBF5F305FB130041F27071039042
:107FE000B0FBF1F0009006492046FFF7D5FD204692
:107FF000FAF7EAF830707FBD00D68300407E0500B6
:10800000B98F030870B5074C054620460E46FAF7AF
:10801000DBF80246307021462846D2B2BDE87040F7
:10802000FAF78AB907CE002070B5074C05462046FE
:108030000E46FAF7C9F80246307021462846D2B2F9
:10804000BDE87040FAF778B940CC002070B5074C15
:10805000054620460E46FAF7B7F80246307021462C
:108060002846D2B2BDE87040FAF766B9D48F03084B
:1080700070B5074C054620460E46FAF7A5F80246AD
:10808000307021462846D2B2BDE87040FAF754B9A4
:1080900068CC002070B5074C054620460E46FAF71E
:1080A00093F80246307021462846D2B2BDE87040AF
:1080B000FAF742B97ACC002070B5074C0546204645
:1080C0000E46FAF781F80246307021462846D2B2B1
:1080D000BDE87040FAF730B9D5CD002070B5074C37
:1080E000054620460E46FAF76FF8024630702146E4
:1080F0002846D2B2BDE87040FAF71EB91BCE002068
:1081000070B5074C054620460E46FAF75DF8024664
:10811000307021462846D2B2BDE87040FAF70CB95B
:108120008ACC002070B5074C054620460E46FAF76B
:108130004BF80246307021462846D2B2BDE8704066
:10814000FAF7FAB8B5CF002070B5074C05462046BF
:108150000E46FAF739F80246307021462846D2B268
:10816000BDE87040FAF7E8B8C0CF002038B5084B3A
:108170001546172202FB00320C460846023205491A
:10818000FFF70AFD2046FAF71FF8287038BD00BF38
:10819000ECCE00202C04040838B5084B15461722F5
:1081A00002FB00320C46084605320549FFF7F4FC95
:1081B0002046FAF709F8287038BD00BFF4CE002039
:1081C0002C040408034B172202FB003090F81133F3
:1081D0000B707047DCCB0020084A38B592F820318C
:1081E0000C46054606490BB1333200E00232FFF778
:1081F000D3FC2846F9F7E8FF207038BDDCCB00201F
:108200002C040408084A38B592F820310C4605467B
:1082100006490BB1433200E01232FFF7BDFC28469D
:10822000F9F7D2FF207038BDDCCB00202C04040805
:10823000084A38B592F820310C46054606490BB17C
:10824000533200E02232FFF7A7FC2846F9F7BCFFC3
:10825000207038BDDCCB00202C040408084B93F8B8
:10826000202112B193F8633001E093F832300BB162
:10827000312300E03023037001230B70704700BFEF
:10828000DCCB002038B5054A05460C460449FFF70B
:1082900083FC2846F9F798FF207038BDADCD00204B
:1082A0002C04040838B5054A05460C460449FFF776
:1082B00073FC2846F9F788FF207038BDC1CD002037
:1082C0002C04040838B5054A05460C460449FFF756
:1082D00063FC2846F9F778FF207038BD89CE00206E
:1082E0002C04040838B5054A05460C460449FFF736
:1082F00053FC2846F9F768FF207038BD9DCE00205A
:108300002C04040838B5054A05460C460449FFF715
:1083100043FC2846F9F758FF207038BDB1CE002045
:108320002C04040838B5054A05460C460449FFF7F5
:1083300033FC2846F9F748FF207038BDC5CE002031
:108340002C04040838B5054A05460C460449FFF7D5
:1083500023FC2846F9F738FF207038BDD9CE00201D
:108360002C04040838B5054A05460C460449FFF7B5
:1083700013FC2846F9F728FF207038BD55CF0020A0
:108380002C04040838B5064B05460C46D3F89C234C
:108390000449FFF701FC2846F9F716FF207038BDA5
:1083A000DCCB0020A78F030838B5064B05460C46EA
:1083B000D3F8A0230449FFF7EFFB2846F9F704FFA1
:1083C000207038BDDCCB0020A78F030838B5054AE4
:1083D00005460C460449FFF7DFFB2846F9F7F4FE93
:1083E000207038BD65CF00202C040408054B93F89D
:1083F0009A330BB1312300E03023037001230B705B
:10840000704700BFDCCB0020054B93F878330BB1ED
:10841000312300E03023037001230B70704700BF4D
:10842000DCCB002038B5084B93F820310C460546CC
:1084300006490BB1064A00E0064AFFF7ADFB2846A5
:10844000F9F7C2FE207038BDDCCB00202C040408F4
:10845000DE8F0308E38F0308012008B50146FDF70E
:10846000D3FC02200021BDE80840FDF7CDBC000090
:10847000014B83F820017047DCCB0020014B012227
:108480001A707047180B002001460148F9F73EBEEC
:108490000FCC002001460148F9F738BE1FCC002060
:1084A00001460148F9F732BE2FCC002008B5064935
:1084B0000222F9F7EBFE054B08B9012200E0002289
:1084C00083F8632008BD00BFE98F0308DCCB0020E0
:1084D00001460148F9F71ABEADCD0020014601481A
:1084E000F9F714BEC1CD002010B5054C0146204659
:1084F000F9F70CFE2046BDE810400FF0DDBB00BFD1
:1085000089CE002010B5054C01462046F9F7FEFD46
:108510002046BDE810400FF0CFBB00BF9DCE00202D
:1085200010B5054C01462046F9F7F0FD2046BDE8A0
:1085300010400FF0C1BB00BFB1CE002010B5054CFC
:1085400001462046F9F7E2FD2046BDE810400FF055
:10855000B3BB00BFC5CE002010B5054C0146204678
:10856000F9F7D4FD2046BDE810400FF0A5BB00BFD1
:10857000D9CE002010B5064C01462046F9F7C6FDBD
:1085800020460FF06FFBBDE810400FF021BB00BF8D
:10859000D5CD002010B5054C01462046F9F7B6FDB3
:1085A0002046BDE810400FF079BB00BF1BCE002075
:1085B00001460148F9F7AABD8ACC002001460148CE
:1085C000F9F7A4BD55CF002008B5F9F705FB024B1C
:1085D000C3F89C0308BD00BFDCCB002008B5F9F749
:1085E000FBFA024BC3F8A00308BD00BFDCCB0020A0
:1085F00001460148F9F78ABD65CF002008B5064954
:108600000222F9F743FE054B08B9012200E00022DF
:1086100083F89A2308BD00BFE98F0308DCCB002054
:1086200008B506490222F9F731FE054B08B90122C7
:1086300000E0002283F8782308BD00BFE98F03081B
:10864000DCCB002010B58CB004460021122207A814
:10865000F9F7E2FB002109226846F9F7DDFB04F196
:108660000801022207A8F9F767FE211D042207A8C6
:10867000F9F7DAFD0222A11C07A8F9F7D5FD03A836
:108680000021FEF7DFF89DF811209DF81030084911
:108690006846FFF781FA6846F9F796FD6946C2B267
:1086A00007A8F9F7C1FD07A8FDF7B2FF0CB010BD90
:1086B000EC8F030810B590B00446002112220BA8DD
:1086C000F9F7AAFB0E22002103A8F9F7A5FB07A8DA
:1086D0000021FEF7B7F89DF825109DF824309DF88D
:1086E0002320009103A80A49FFF756FA03A8F9F7D7
:1086F0006BFD03A9C2B20BA8F9F796FD0BA82146A2
:108700000522F9F791FD0BA8FDF782FF10B010BD0F
:10871000FA8F030838B50D4C0D4994F840530122E7
:10872000F9F7B4FD48B9012084F8400365B90FF0AA
:10873000BFFBBDE838400FF0FDBB002084F84003CC
:10874000BDE838400FF0B4BB38BD00BFDCCB002023
:10875000DF92030801460148F9F7D8BC1DCF00207D
:1087600070B5F9F735FAF8F749FA274BD3F87043A3
:10877000064600212046F8F75BFD00B133E02046B5
:108780000021F8F737FD002832D030460021F8F7F5
:1087900045FD70B12046F7F7FBFEFCF7FFFE0446EF
:1087A0000D463046F7F7F4FE22462B46F7F792FDCA
:1087B00016E030462146F8F731FDA0B12046F7F724
:1087C000E7FEFCF7EBFE044630460D46F7F7E0FE09
:1087D000FCF7E4FE02460B4620462946F7F778FDF3
:1087E000F8F70CFA0AE030462146F8F75BFA05E0A4
:1087F00020460021F8F7F4FC10B13046FEF720F9CE
:10880000014BC3F8706370BDDCCB002010B50C4683
:10881000F9F7E2F90249091981F8760310BD00BFA2
:10882000DCCB002010B50C46F9F7D6F9E31DC1B238
:10883000D8B2BDE8104000F080BC03460731C8B292
:10884000194600F07ABC000010B50C46F9F7C4F9DF
:10885000044B1B19214683F874030020BDE8104027
:10886000FFF7EBBFDCCB0020024B00221A705A70DE
:10887000704700BFDCCB002010B5094C09492046E9
:10888000F9F744FC084904F11000F9F73FFC04F142
:1088900020000649F9F73AFC012284F8302010BD87
:1088A000DECB00200D9003081990030825900308E3
:1088B00010B5094C09492046F9F728FC084904F18C
:1088C0001000F9F723FC04F120000649F9F71EFC1B
:1088D000012284F8302010BDDECB00203390030845
:1088E000199003082590030870B51E4C1E4D1F4EAD
:1088F00029462046F9F70AFC314604F1A000F9F7B1
:1089000005FC314604F1B400F9F700FC294604F1F6
:10891000C800F9F7FBFB04F1FA001549F9F7F6FB7B
:108920002946144D04F58770F9F7F0FB294604F544
:10893000BE70F9F7EBFB294604F5C870F9F7E6FBC2
:10894000294604F5D270F9F7E1FB294604F5DC70FD
:10895000F9F7DCFB04F5E6702946BDE87040F9F74D
:10896000D5BB00BF0DCD0020F90604083F900308D9
:10897000469003084D90030810B5502003F072FB99
:10898000044698B100F074FA21461148F9F7BEFB8D
:1089900004F112010F48F9F7B9FB04F132010E4856
:1089A000F9F7B4FB204603F0E3FB0BE00B490A4860
:1089B000F9F7ACFB0A490648F9F7A8FB054809494D
:1089C000F9F7A4FB08480949BDE81040F9F79EBB38
:1089D00068CC00207ACC002040CC002055900308C1
:1089E00060900308729003088ACC0020F9060408FE
:1089F0002DE9F041144D002417274FF0010814F021
:108A0000FF0308D11149124885F81133F9F77EFBAD
:108A10001048114910E007FB04F6AB1906F5447045
:108A200028180E4983F81183023006F54676F9F7C7
:108A30006DFBA8190A4905300134F9F767FB022CD0
:108A4000DDD1BDE8F08100BFDCCB00207A900308C7
:108A5000EECE0020F9CE0020809003088690030817
:108A60008B90030810B5084C08490948012384F885
:108A70004033F9F74BFB074B07480849C4F87033FC
:108A8000BDE81040F9F742BBDCCB00209090030812
:108A90001DCF0020000040402DCF00209F900308F4
:108AA000044B0122032183F8742383F8751383F8A0
:108AB00076237047DCCB002010B50B4C0B490C48DB
:108AC000012384F8783384F89A33F9F71FFB40F2D6
:108AD000147308480849C4F89C337B23C4F8A033B6
:108AE000BDE81040F9F712BBDCCB00204D90030825
:108AF00055CF002065CF002080900308002306E0BA
:108B000003F1006202F580421268C25401338B42C5
:108B1000F6D1704708200221FCF722BE08B5FCF709
:108B200089FD0348E921BDE80840FCF789BD00BF85
:108B3000DCCB00202DE9F84F06468A46FFF7EEFF12
:108B4000174C80460327FCF78BFD3546FFF7E2FF05
:108B500004EB0A0B0AE015F8011B2046FCF7C6FDE2
:108B600004F1010908282E464C4602D15C452E46E8
:108B7000F1D141460B48FCF7D5FDFCF77FFD0A48D3
:108B80004FF46A71FFF7BAFFFFF7C8FF404504D002
:108B9000013F17F0FF07D6D1FEE7BDE8F88F00BF11
:108BA000004000089C5F0008DCCB002008B5FCF703
:108BB00041FD03484721BDE80840FCF741BD00BF27
:108BC000DCCB002008B5FFF7F1FF054B4FF46A71CD
:108BD000C3F81C011846BDE80840FFF7ABBF00BF53
:108BE000DCCB002010B50D4CFFF746FEFFF760FE12
:108BF000FFF77AFEFFF738FE002384F82031FFF7F5
:108C000031FFFFF74DFFFFF757FFFFF7CFFF044B93
:108C1000C4F81C01C4F8A43310BD00BFDCCB002095
:108C200015CD5B0710B50F4CFFF71EFEFFF724FEB6
:108C3000FFF73EFEFFF758FEFFF79EFE002384F885
:108C40002031FFF7D5FEFFF70DFFFFF729FFFFF7F4
:108C500033FFFFF7ABFF044BC4F81C01C4F8A43387
:108C600010BD00BFDCCB002015CD5B0710B5094857
:108C70004FF46A71FFF742FF074B1C68FFF74EFF86
:108C8000844205D0FFF7CEFFBDE81040FFF79ABF42
:108C900010BD00BFDCCB00209C5F000810B50B4C62
:108CA000FFF7E2FDFFF720FE002384F82031FFF7F5
:108CB000D9FEFFF7F5FEFFF7FFFEFFF777FF044B46
:108CC000C4F81C01C4F8A43310BD00BFDCCB0020E5
:108CD00015CD5B07022008B5FDF7A6F810F0FF0FD1
:108CE00014D002200021FDF78FF80320FDF79CF837
:108CF00060B102200EF04CFF0220054901F00AFA93
:108D000003200021BDE80840FDF77EB808BD00BF84
:108D1000A490030873B50A4E451E002431198C3106
:108D2000022201A8F9F708FB0021102201A8FAF796
:108D300039FE0334122C05F8010FEFD17CBD00BFC2
:108D4000DCCB002070B5074C06460D4628220021DA
:108D50002046F9F761F8204631462A46BDE87040C2
:108D6000F8F7A0BF40CC002010B502460C460648DC
:108D70001221FEF7F3FE102122460448FEF7EEFE14
:108D8000034B0120187010BD190B00202B0B002085
:108D90003D0B0020094B1B7810B504465BB1122136
:108DA000074AFEF7DBFE04F112001021054AFEF728
:108DB000D5FE012010BD184610BD00BF3D0B0020A0
:108DC000190B00202B0B002070B5044658B3164D2C
:108DD000D5F81C61FFF7EAFE864205D105F18C004B
:108DE00005F19E01FFF7C0FF2046FFF7D3FF50B902
:108DF00012210E4A2046FEF7B1FE04F112001021A6
:108E00000B4AFEF7ABFE102104F12200094AFEF7DF
:108E1000A5FE04F132001421074AFEF79FFE074B1E
:108E20000120A36470BD70BDDCCB002060900308FE
:108E300072900308B8900308BE90030815CD5B0735
:108E400010B50446FCF7F6FB20461321BDE81040A0
:108E5000FCF7F6BB10B5044640B1FFF7F1FF502117
:108E60000246204600F034F8012010BD10BD00007D
:108E700038B5044678B150210B4A00F01BF80B4B73
:108E800020461D68FFF7DCFF854205D1A36C084A28
:108E9000934201D106E038BD2046FFF795FF2046FA
:108EA000FFF7D8FF012038BD008000089CBF0008F4
:108EB00015CD5B075118801A02E013688354013204
:108EC0008A42FAD1704710200221FCF749BC000009
:108ED0002DE9F84F1B4C8A46904606460327FCF7BF
:108EE000BFFB3546FFF7EFFF04EB0A0B0AE015F86E
:108EF000011B2046FCF7FAFB04F1010908282E4665
:108F00004C4602D15C452E46F1D141460E48FCF755
:108F100009FCFCF7B3FB0B48FFF792FF40450FD06D
:108F2000013F17F0FF07DAD1BFF34F8F074A084B15
:108F3000D16801F4E0610B43D360BFF34F8FFEE7CC
:108F4000BDE8F88F008000089CBF000800ED00E03D
:108F50000400FA0530B5012185B08020FCF79AFDA8
:108F60002C23002401258DF80030684606238DF857
:108F700001308DF802408DF80350FCF71DFB0F4BBC
:108F8000202283F82C23ADF80C40ADF806400C4CA1
:108F900041F26F73ADF8043020464FF47A7301A9A3
:108FA0000293FCF77DFF20462946FCF7B7FF2046D9
:108FB00029462A46FCF7BEFF05B030BD00E100E0BF
:108FC000001C004008B504480121FCF7BCFF10203C
:108FD000BDE80840FDF71EBA001C00400121FDF766
:108FE00085B90021FDF782B908B50920FFF7F9FF1F
:108FF0000A20FFF7F6FF0B20FFF7F3FF0C20FFF727
:10900000F0FF0D20BDE80840FFF7EBBF70B50E4E36
:109010000E4D0023F47CE40909D0A34202D00A20BB
:10902000FFF7DFFF0A20FDF7F5F9092005E0A3426D
:1090300002D00920FFF7D5FF0A20FDF7EBF92888B9
:1090400002F08EFC2346E5E7A0CF0020600600205A
:10905000FDF7E0B9014B1880704700BF60060020A3
:109060007047000008B503200EF092FD0949012069
:1090700001F050F84FF4FA7002F072FCFFF7B2FD05
:10908000FFF7A0FD40F2F23002F06AFCBDE80840B4
:1090900000F046BBC79003080078FDF7CBB900008D
:1090A00010B5094C0F23237005236380074BA36081
:1090B000074B2822E3602046002363612283A376C6
:1090C000FFF7EAFFA07110BD84CF00206190020875
:1090D0006590020810B504460078FDF7ABF96369A6
:1090E00050B9228BA07601339342636114D9642076
:1090F000BDE81040FFF7AEBF228B93420AD9A37E92
:1091000043B90123A3764FF47A70FFF7A3FFE36816
:10911000984710BD0023636110BD000008B50348E7
:10912000FFF7D8FF642002F01BFCF8E784CF002093
:109130000E20FDF77FB9FDF77DB9003118BF012181
:10914000FDF7D4B838B5104C0025002329460B2272
:1091500004F1150023606360A360E3602574657407
:10916000A574E574257584F82C5084F82E5084F885
:109170002D50F8F751FE04F1200029460B22BDE8DE
:109180003840F8F749BE00BFA0CF002030B5032813
:1091900087B0364D0CD100210A2203A8F8F73CFE17
:1091A000334B3449EA681B8803A8FEF7F5FC37E027
:1091B00005283BD1002103A80A22F8F72DFE2E4BEB
:1091C0001C684FF07E512046F8F728F860B1204621
:1091D0002A49F8F70FF838B12046F7F7D9F9CDE961
:1091E000000103A8264918E020464FF07E51F8F709
:1091F00001F81E4D50B121492046F7F75DFEF7F703
:10920000C7F9CDE9000103A81E4906E02046F7F79B
:10921000BFF9CDE900011C4903A86A69FEF7BCFC4F
:1092200003A8F8F7D1FFC1B203A81AE0062811D1AC
:1092300000210A2203A8F8F7EFFDAA690C4B134995
:109240001B880092124A128803A801926A69FEF7ED
:10925000A3FCE5E755F820402046F8F7B5FFC1B27A
:109260002046FDF7F1FE07B030BD00BF64060020C8
:10927000780B0020FB900308740B002000002041B5
:10928000E2900308E9900308F0900308F6900308C1
:109290003E0B002010B50E4C002060860DE04FF410
:1092A000FA70FDF7F5FE002803DA094B00225A8612
:1092B00008E0638EE05401336386638E312B01D85E
:1092C0000D28ECD1024B588E003018BF012010BD84
:1092D000400B0020000000002DE9FF410378282BFF
:1092E000044640F0E480784B012283F82D2083F877
:1092F0002E20002283F82C20744B197811B11A709B
:1093000000F01EFF01340A22002101A8F8F784FDB5
:1093100020466F49F9F742F8001BC6B23246214693
:1093200001A8F9F709F801A8F8F752FCF7F766FC6D
:109330000136A619644C0A226060002101A8F8F7E2
:109340006BFD30466249F9F729F8801BC5B23146FA
:109350002A4601A80135F8F7EFFF75190A22002106
:1093600001A8F8F759FD28465949F9F717F8401BA5
:109370005FFA80F84246294601A8F8F7DDFF01A808
:10938000F8F726FCF7F73AFC08F10108A8440A228E
:10939000A060002101A8F8F73FFD4D494046F8F7CD
:1093A000FDFFC8EB0000C7B23A46414601A8F8F7F6
:1093B000C3FF01A8F8F710FC013747440A222074C4
:1093C000002101A8F8F728FD41493846F8F7E6FFE3
:1093D000C01BC6B23246394601A8F8F7ADFF01A856
:1093E000F8F7F6FBF7F70AFC0136BE1920600A22EF
:1093F000002101A8F8F710FD30463549F8F7CEFFF7
:10940000801BC5B22A46314601A8F8F795FF01A88E
:10941000F8F7DEFB28A3D3E90023F6F759FF002273
:109420002C4BF7F709F926A3D3E90023F7F72EFA17
:10943000F7F7C4FB0135751960740A22002101A8F1
:10944000F8F7EAFC28462249F8F7A8FF401BC6B205
:109450003246294601A8F8F76FFF01A8F8F7B8FBD4
:10946000F7F7CCFB0136AD19E0600A22002101A814
:10947000F8F7D2FC18492846F8F790FF401BC4B211
:10948000294601A82246F8F757FF0023194609E0AC
:1094900001AAC3F107009A5C303A02FA00F21143C4
:1094A000C9B20133DAB2A242F2D3074BD974BDE894
:1094B000FF8100BFAFF300809A9999999999F93F7C
:1094C000666666666666E63FA0CF0020E80B002071
:1094D000019103080000594085500408AFF3008053
:1094E00010B50378232B37D11C4B012283F82D2094
:1094F00083F82E201130002283F82C2003461C46CE
:109500001A1A217801332029D2B2F8D013480E2A32
:10951000437D00F1150008D821460A2213B9F8F757
:109520000BFF06E0F8F708FF08E00D4923B9F8F74C
:10953000EDFD0EF04DFB01E0F8F7E8FD0B342146A0
:1095400008220848F8F7F8FE074804F1080102224B
:10955000BDE81040F8F7F0BE10BD00BFA0CF00205E
:1095600003910308C3CF0020C0CF002030B503789B
:10957000282B85B005461BD10E4C012300210A2261
:1095800001A884F82D3084F82E3084F82C10F8F7D8
:1095900043FC691C01A8F8F7B9FDE37CDB0906D0A0
:1095A00001A8F8F715FBF7F709FBA07400E0A37416
:1095B00005B030BDA0CF002070B52E4C2E4D00263A
:1095C00094F82D30CBB194F82E10B1B994F82C301A
:1095D000022B03D0013384F82C300EE0274826609C
:1095E0000B226660A660E66021746174A174E17468
:1095F000217584F82D10F8F70FFC2B786BB1002043
:10960000287084F82E00FFF7C1FDFFF743FE10B16C
:109610001B48FFF761FE01232B702B789BB10021C3
:1096200032221748F8F7F8FB00230B202B7084F840
:109630002E30FFF7ABFDFFF72DFE10B11048FFF7FE
:1096400095FF01232B702B7873B1002309202B7019
:1096500084F82E30FFF79AFDFFF71CFE10B1084882
:10966000FFF73EFF01232B704FF47A7002F078F978
:10967000A6E700BFA0CF002062060020C0CF0020D8
:10968000400B002070B50646144C02E0322002F078
:1096900067F92378114D002BF8D0002330462B704A
:1096A000FFF774FDFFF7F6FD90B101240C480D495A
:1096B0002C700322F8F7EAFD68B10B490848032231
:1096C000F8F7E4FD002814BF4FF0FF30002070BD14
:1096D0004FF0FF3070BD204670BD00BF6206002015
:1096E000400B00200B9103080F9103081FB5FFF7F3
:1096F00029FD084B08490948012283F82D20002341
:1097000000930193029303934FF4807201F08EFE55
:1097100005B000BDA0CF002013910308B995020841
:1097200008B504200EF034FA0A49002000F0F2FCDB
:1097300040F2F23002F014F900F00EFCBFF34F8F4C
:10974000054A064BD16801F4E0610B43D360BFF3D7
:109750004F8FFEE7C790030800ED00E00400FA0514
:10976000002380E806008360C36070474268C368D6
:109770008068511E8B4208BF1018C01A421E50420A
:10978000504170478368C268934205D102E00023CC
:1097900083600AE000207047026852F823200A60C4
:1097A0004268013393428360F1D00120704738B59D
:1097B00004460D46FFF7DAFF50B9E368226842F825
:1097C0002350626801339342E36003D1E06001E01B
:1097D000002038BD012038BD084B1B681B185B7882
:1097E00003F00402D2B20AB1303805E003F00303FB
:1097F000012B08BF20305738C0B27047000000204E
:109800002DE9F04707460E46044615464FF020095D
:109810001EE0252B12D16878C0B195F80280B8F10E
:10982000000F13D0FFF7D8FF82464046FFF7D4FF62
:1098300040EA0A1004F8010B023507E02B2B04F173
:1098400001020CBF84F80090237014460135013EDC
:109850002B780BB1012EDCD8002323703846BDE8ED
:10986000F087000038B50620FFF765FC1C4B93F825
:1098700076431C4B60401A7DC4B284F0010102F0B3
:109880000F0242EA01121A75174A184B117869B98A
:10989000012515701C7014BB0820154900F03AFC16
:1098A00006200EF075F9134B1D7038BD14B9124A1D
:1098B000012111701B78A3420FD00E4D082024B156
:1098C0000E4900F027FC052003E0094900F022FCC6
:1098D00006200EF05DF901232B70044B1C7038BD7F
:1098E000DCCB0020A0CF0020810B00207F0B0020CC
:1098F00042910308E80B0020830B00204F910308DE
:10990000F0B589B0002168461E22F8F785FA454B6C
:1099100093F8745393F87573434B1C78434B197841
:1099200029BB01221A70424B1C70424B1D70424BE6
:1099300095421F700AD14CB12846FEF77EFF0720E2
:109940000EF026F909203D4900F0E4FB3A4B187867
:10995000012865D1002C63D00146FEF76EFF082078
:109960000EF016F90A20354900F0D4FB58E054B146
:10997000334B93F82D300B2013B1FFF769FB05E053
:10998000FFF72CFB02E00B20FFF72BFB284B1B788B
:10999000A3423FD0274B1E78012E1BD168460021E1
:1099A0001E22F8F739FA34B130460021FEF745FFA0
:1099B0006846224905E020462146FEF73EFF214940
:1099C0006846F8F78FFA07200EF0E2F8092069469A
:1099D00000F0A0FB184B1E78012E1BD16846002119
:1099E0001E22F8F719FA34B130463146FEF725FF4A
:1099F0006846124905E020463146FEF71EFF114930
:109A00006846F8F76FFA08200EF0C2F80A20694697
:109A100000F080FB074B1D70074B1F70044B1C7040
:109A200009B0F0BDDCCB0020830B0020820B0020AE
:109A30008C0B00207A0B00207E0B00205A9103082B
:109A4000A0CF00206B910308F0B589B000211E2241
:109A50006846F8F7E1F93D4F3D4B397893F8745378
:109A600093F875633B4B3C4A1C783C4B19BB1D700B
:109A70003B4B14700120022D38701E7009D144B187
:109A8000FEF7DBFE07200EF083F80920354900F0D1
:109A900041FB334B1B78022B55D1002C53D00120B6
:109AA0000146FEF7CAFE08200EF072F80A202D4982
:109AB00000F030FB47E01278A2423ED01B78022B28
:109AC0001BD1684600211E22F8F7A6F934B1012007
:109AD0000021FEF7B2FE6846224905E020462146F5
:109AE000FEF7ABFE20496846F8F7FCF907200EF0B8
:109AF0004FF80920694600F00DFB194B1B78022B2B
:109B00001BD1684600211E22F8F786F934B10120E6
:109B10000146FEF792FE6846134905E02046012102
:109B2000FEF78BFE0F496846F8F7DCF908200EF0C7
:109B30002FF80A20694600F0EDFA084B1D70084B1B
:109B40001E70054B1C7009B0F0BD00BF870B0020D4
:109B5000DCCB00208B0B0020850B0020890B002024
:109B60008A0B00205A9103086B91030838B5174AF5
:109B7000174B1178DC7C174BE40969B90125157086
:109B80001C7014B30C20144900F0C4FA0B200DF023
:109B9000FFFF124B1D7038BD14B1114A0121117025
:109BA0001B78A3420FD00D4D0C2024B10A4900F0C0
:109BB000B1FA0B2003E00B4900F0ACFA0C200DF0D9
:109BC000E7FF01232B70034B1C7038BD840B002072
:109BD000A0CF0020800B002042910308E80B00205A
:109BE000830B00204F91030838B5194B194ADB7CD1
:109BF0001178DC0918BFC3F38014174B69B901252C
:109C000015701C701CB30D20144900F083FA0D2050
:109C10000DF0BEFF124B1D7038BD14B1114A012169
:109C200011701B78A34210D00D4D2CB10D200DF0FA
:109C3000AFFF0D20094904E00E200DF0A9FF0A49ED
:109C40000D2000F067FA01232B70034B1C7038BD08
:109C5000A0CF00208D0B00207B0B00204291030839
:109C6000E80B00208B0B00204F91030838B5224CE5
:109C7000207CF7F7C9F821490546F7F7D9FAD8B19A
:109C80001F4B01251D70237D03F00E032B4323750D
:109C90001C4C237873BB0D20FFF7A0F90C20FFF7B5
:109CA0009DF90E201849257000F034FA0F200DF0B0
:109CB0006FFF164B1D7038BD28461549F7F79AFA05
:109CC000C0B1237D0F4D03F00E0323752C78012CBA
:109CD00010D10D20FFF785F90C20FFF782F9002342
:109CE0000E200C492B7000F015FA10200DF050FFDB
:109CF000064B1C7038BD00BFA0CF002000008C4276
:109D0000830B00207D0B002042910308E80B00200C
:109D100000008A424F91030838B51B4C1B49E56887
:109D20002846F7F785FAB0B1194B01251D70237D40
:109D300003F00D0343F002032375164B1A7812BB90
:109D40000B2015491D7000F0E5F90A200DF020FFE9
:109D5000124B1D7038BD28461149F7F74BFA90B1E8
:109D6000237D03F00D0323750A4B1C78012C0AD1C7
:109D700000220B200B491A7000F0CCF909200DF0DD
:109D800007FF064B1C7038BDA0CF0020000020420A
:109D9000830B00208F0B002042910308E80B00206A
:109DA00000001C424F91030838B51B4B1A7D93F8F5
:109DB0002D4002F00B0284F0010142EA81021A7583
:109DC000164A174B117869B9012515701C7014BB20
:109DD0000F20144900F09EF911200DF0D9FE124B0E
:109DE0001D7038BD14B9114A012111701B78A342AE
:109DF0000FD00D4D0F2024B10D4900F08BF912202A
:109E000003E0084900F086F911200DF0C1FE01239E
:109E10002B70034B1C7038BDA0CF00207C0B0020A2
:109E2000860B002042910308E80B0020830B0020E2
:109E30004F91030838B51D4BDC7CE2091A7D08BF41
:109E4000C4F3801402F0070218BF002442EAC402DF
:109E50001A75174A174B117869B9012515701C70CE
:109E600014B31020144900F055F913200DF090FEA2
:109E7000124B1D7038BD14B1114A012111701B78AD
:109E8000A3420FD00D4D102024B90E4900F042F925
:109E9000142003E0084900F03DF913200DF078FE8E
:109EA00001232B70034B1C7038BD00BFA0CF0020D6
:109EB0008E0B0020880B002042910308E80B002045
:109EC000830B00204F91030870B541F2883001F0F8
:109ED00047FD104D104E0024104B2C7093F82D3080
:109EE00034704BB1FFF742FEFFF77EFEFFF7BEFE78
:109EF000FFF712FFFFF79EFFFFF756FFFFF7B2FCD9
:109F0000FFF7FEFCFFF7A0FD4FF47A7001F028FD8B
:109F1000E2E700BF830B00208B0B0020A0CF0020C6
:109F2000084611461A460023FCF7C6BE08461146ED
:109F30001A460023FCF70FBF08460021FCF71BBFA1
:109F400008B5034C01250348257001F009FDFAE727
:109F5000E80B0020C027090008B5084B1B785BB14F
:109F6000074B0021186842F210720B4601F054F9B9
:109F7000431E5842584108BD012008BDF00B002087
:109F8000EC0B00201FB5224B1A780446002A3ED065
:109F90005A685B891F4920480A605B08043B8B6054
:109FA0000122382300F0A1FB1CB11B4800F0A7FBE5
:109FB00004E0194800F085FC0028F6D1144B17493D
:109FC0005A685B890A605B08043B8B601448012275
:109FD000382300F08AFB1CB1114800F090FB04E02C
:109FE0000F4800F06EFC0028F6D10E4B01201870CF
:109FF00001F06CF80C4B0D4918600023009301939D
:10A00000029303930A484FF4807201F00FFA1FBDC8
:10A010007CC80020AC060020BC0B00209406002069
:10A02000900B0020F00B0020EC0B00208091030827
:10A03000419F020830B5124B002185B004464FF015
:10A04000FF3218680B4601F0E7F80546A8B1216811
:10A0500021B96846FCF7F6FB039B23602379112B9B
:10A060000CBF08480848214600F07CFB044B002147
:10A0700018680A460B4600F08FFF284605B030BD31
:10A08000EC0B0020BC0B0020900B002070B50D4E97
:10A090000A46002105460B46306801F0BDF804462B
:10A0A00070B12B79112B0CBF07480848294600F0E6
:10A0B000C3FB002104460A4630680B4600F06CFFE3
:10A0C000204670BDEC0B0020BC0B0020900B002044
:10A0D00070B50D4D0A46002106460B46286801F072
:10A0E0009BF8044668B13379112B0CBF0748084828
:10A0F00000F0DCFB002104460A4628680B4600F00D
:10A100004BFF204670BD00BFEC0B0020BC0B0020B5
:10A11000900B002000B58FB0002300936B448DF8A6
:10A1200004003122581DF8F707F9044B1B7813B1CE
:10A130006846FFF77FFF0FB000BD00BFF00B0020A7
:10A1400030B58FB005460021322201A8F7F764FE32
:10A150002846F8F739F8C4B2294601A82246F8F78C
:10A16000EBF822238DF804303B21002305E001AAFF
:10A17000985C202808BF99540133DAB2A242F6D382
:10A180000EAB1C193B2304F8353C044B1B781BB168
:10A19000112001A9FFF7BEFF0FB030BDF00B00206A
:10A1A000014B1878704700BFF00B002008B5044839
:10A1B00000F0C6FA0A2390FBF3F0013008BD00BF9F
:10A1C000BC0B0020014800F0BBBA00BFBC0B002054
:10A1D0002DE9F0439DB00D460646FFF7F3FF002141
:10A1E0000446142209A86FF00908F7F715FE08FBCA
:10A1F00005482A4C08F1090800250DF13D07C5EB7B
:10A200000803002BA36246DBD4F80C902069216878
:10A2100093FBF9F202EB000E88689EFBF0FC00FB5A
:10A220001CE009FB1233206263624FF0FF311123FF
:10A230000EA88DF83C30FFF729FF002338468DF833
:10A240006E30F7F7C1FF394602463046F7F7ECFFAC
:10A2500005A80E99FCF786FB9DF81D109DF81B20A4
:10A2600000919DF819109DF81C3001919DF818106F
:10A2700002919DF8141009A803910949FDF78CFC7F
:10A2800009A93046F7F72EFE013530460549F7F7A4
:10A2900029FE0A2DB3D11DB0BDE8F083BC0B002010
:10A2A00089910308A79103082DE9F0419CB09046DD
:10A2B000112205460C468DF83C2023B10EA84FF024
:10A2C000FF31FFF705FF2C4B402095FBF0F01E6897
:10A2D000DD681F69B668986290FBF5F1CF1997FBAE
:10A2E000F6F206FB127605FB11001E6258624FEA79
:10A2F000981700250DF13D0635E011234FF0FF3191
:10A300000EA88DF83C30FFF7C1FE002330468DF8D3
:10A310006E30F7F759FF0DF13E01421E2046F7F768
:10A3200083FF05A80E99FCF71DFB9DF81D109DF8F5
:10A330001B2000919DF819109DF81C3001919DF88B
:10A34000181002919DF8141009A803910B49FDF70C
:10A3500023FC09A92046F7F7C5FD20460849F7F771
:10A36000C1FD0135EDB2BD42C7D32046F7F72CFF42
:10A370001CB0BDE8F08100BFBC0B00208991030830
:10A38000F806040808B5044800F0DAF90A2390FB3F
:10A39000F3F0013008BD00BF900B0020014800F031
:10A3A000CFB900BF900B00202DE9F0439DB00E46C1
:10A3B0000446FFF7F3FF00210546142209A86FF0B9
:10A3C0000909F7F729FD09FB0659384D09F1090973
:10A3D00000260DF13D07C6EB0903002BAB6261DBE4
:10A3E000334AD1682A6993FBF1F189182A68926887
:10A3F00091FBF2F002FB10122A62EA6893FBF2F181
:10A4000002FB11336B624FF0FF3105230EA88DF86C
:10A410003C30FFF73BFE27492046F7F763FD264B0C
:10A420009DF83C2053F822804046F7F7CDFE414688
:10A4300002462046F7F7F8FE20492046F7F752FD7E
:10A44000002338468DF86E30F7F7BEFE39460246D7
:10A450002046F7F7E9FE19492046F7F743FD05A81E
:10A460000E99FCF77FFA9DF81D109DF81B200091B6
:10A470009DF819109DF81C3001919DF8181002915B
:10A480009DF8141009A803910D49FDF785FB09A952
:10A490002046F7F727FD013620460A49F7F722FD47
:10A4A0000A2E98D11DB0BDE8F08300BF900B0020AC
:10A4B000BC0B00206F420408C4060020AA910308C8
:10A4C00089910308A79103082DE9F041ADF58B6D43
:10A4D0009046052204460D468DF83C2023B10EA877
:10A4E0004FF0FF31FFF7F4FD434B6421DE681F6935
:10A4F00094FBF1F494FBF6F000EB070E1F689C62EE
:10A50000BF689EFBF7F206FB104407FB12E75C6294
:10A510001F62B8FBF1F800240DF13D0662E06422F1
:10A5200000211CA8F7F778FC4FF0FF310EA8FFF7C9
:10A53000ADFD324B9DF83C2053F822703846F7F7BA
:10A5400043FE394602461CA8F7F76EFE2C491CA8AC
:10A55000F7F7C8FC002330468DF86E30F7F734FE6D
:10A56000314602461CA8F7F75FFE25491CA8F7F7FD
:10A57000B9FC05A80E99FCF7F5F99DF81D109DF89A
:10A580001C3000919DF819109DF81B2001919DF839
:10A59000181002919DF8141009A803911949FDF7AC
:10A5A000FBFA09A91CA8F7F79DFC1CA8F7F70CFEFD
:10A5B00083B2632B0CD81A461CAB98182021C2F129
:10A5C0006302F7F729FC1CA80F49F7F78BFC02E0A0
:10A5D0000A238DF8AF3028461CA96422F7F724FE21
:10A5E0000134E4B244459AD32846F7F7EDFD16B09E
:10A5F0000DF5806DBDE8F081900B0020C4060020B1
:10A60000AA91030889910308F806040803680A68F8
:10A6100010B55C68A2181C6883684868043343431B
:10A6200004FB0230083010BD70B504681646FFF711
:10A63000EDFF65690146324620460423A84770BDF8
:10A6400073B502AC056844F8042DFFF7DFFF2E69EF
:10A650000146224628460423B0477CBD0068436873
:10A66000CB18016810B5594344690423A04710BDB5
:10A6700013B5006802AB046943F8042D42688A18D8
:10A68000016851431A460423A0471CBDF8B503686E
:10A6900028CB04464D194FF07F425D430E46FFF72D
:10A6A000E7FF20682946C36898472246291D52F8CB
:10A6B000040B04230769B847204631466FF0FF02B8
:10A6C000FFF7D6FF0020F8BD4B68C2680133934204
:10A6D0004B6009DB00680A6880680132002382420F
:10A6E00081E80C00A8BF0B60704780E80E000A6884
:10A6F0000433083AB2FBF3F3C3600020704738B567
:10A700000446002505E0294620460022FFF7B0FF59
:10A71000013523689B689D42F5DB002504E029464E
:10A720002046FFF7B3FF013523689B689D42F6DBA7
:10A73000002020616061A061E0612062606238BD3C
:10A740000368816902699B688A1AD21892FBF3F147
:10A7500003FB112310B5C169C468406904FB0311F0
:10A76000081A10BD0368F7B585699B68013595FB2C
:10A77000F3F203FB12550F4601AA29460446FFF7E0
:10A780006DFF019B13F5807F1BD02369AB4208D17D
:10A79000216889686A1C00238A4222616361A8BF1C
:10A7A0002361236AAB4208D1216889686A1C0023AF
:10A7B0008A4222626362A8BF236220462946FFF7CD
:10A7C00065FF2046A16901AAFFF748FF019B13F529
:10A7D000807F05D12046A169154AFFF749FF08E0AF
:10A7E00013F5803F05D01348FDF78AF94FF0FF308D
:10A7F0001DE004F118056FF0FF0229462046FFF71F
:10A800001FFF29462046FFF701FF2668A368D6F8F8
:10A8100010C0011D3A463046E0472946044A20460A
:10A82000FFF70EFF20462946FFF74EFF0020FEBD32
:10A830000000FFFFD79303082DE9F3410446884643
:10A8400000F1200521E02046294601AAFFF7ECFE91
:10A85000019B13F5803F14D129462046FFF7D6FE11
:10A860002768A368D7F814C0011D42463846E04760
:10A8700020462946FFF728FFA36A0133A36230462A
:10A8800012E020462946FFF71FFF226AA3699A4279
:10A8900005D1666AE369F11A4E424E4100E0002696
:10A8A000002ED0D04FF0FF30BDE8FC8100F1100148
:10A8B000034600F1200203C982E8030000209862E9
:10A8C00070472DE9F04F03689E68002585B0044667
:10A8D000013EAA46A846A9466FF0FF0731E043684B
:10A8E000D0F814C005EB030B036803FB0BFB5946C0
:10A8F000082302AAE047029B002B6BD0B3F17F4FE5
:10A9000001D0013306D120465946FFF7BFFE6FF054
:10A91000FF030293029B13F5807F02D013F5803F63
:10A9200058D162680399914254D113F5807F5BD06E
:10A9300013F5803F03D150E06E1E4FF00108013542
:10A940001F46206883689D42C9DBB8F1000F41D0E3
:10A95000BAF1000F08BF00260023A661E36104F1ED
:10A9600018050BE02046294601AAFFF75DFE019B72
:10A97000013306D020462946FFF7A6FEA369B3425D
:10A98000F0D00023C4F81090636104F110050CE0CE
:10A990002046294601AAFFF747FE019B13F5803F99
:10A9A00013D020462946FFF78FFE2269A3699A42F9
:10A9B00008D1E3696269B2EB030EDEF1000353EBE9
:10A9C0000E0300E00023002BE2D02046FFF76EFFCD
:10A9D00000200DE04FF0FF300AE017F5807F08BF40
:10A9E000A9464FF0010AAAE717F5803FA4D0A4E7D3
:10A9F00005B0BDE8F08F0000F8B50F4C01F024FA67
:10AA00002568ADB90D4F0E4E384600F097F9304627
:10AA100000F094F90B4B1F600B4B0A200C212A46C7
:10AA20001E6000F07CFA206010B901F005FAFEE724
:10AA3000BDE8F84001F034BA240C0020F80B0020E7
:10AA40000C0C0020F40B0020280C002010B504464C
:10AA500091424160206105D88169D21A8A420CD2A4
:10AA6000074B04E09A4201D2994206D2054B18687E
:10AA7000211D00F07DF9002010BD012010BD00BF98
:10AA8000280C0020F40B00201FB5FFF7B5FF0B4B7F
:10AA90001B6813B901F0D0F90DE0022300930023E5
:10AAA000019302930393064806494FF4807200F025
:10AAB000BDFC08B9EEE7FEE705B000BD240C0020A0
:10AAC000C1AB0208FD9303082DE9F041804617460B
:10AAD0001E460D4691B12C2001F0C4FA044680B107
:10AAE000FFF78AFF069BC4F80080A561E761266234
:10AAF0006362201D00F02DF903E0FEE701F09CF9F0
:10AB0000FBE72046BDE8F08130B50F4C05462068D4
:10AB100085B0B8B105290191029203950DDC01F0D1
:10AB2000A9F8022801A9206802D1089A002301E0AF
:10AB30000022134600F030FA04E01A4601A900236F
:10AB400000F0EEFA05B030BD240C00202DE9F341F1
:10AB5000194E4FF0000823E0DB68DC681D68271DF4
:10AB6000384600F01DF9636A20469847E369012BD7
:10AB700016D1A369EB18AB4206D963602461306833
:10AB8000394600F0F5F80BE00021CDF800802046B2
:10AB90002A460B46FFF7B8FF10B901F04DF9FEE762
:10ABA00033681A68002AD7D1044A03481168136031
:10ABB0000160BDE8FC8100BFF40B0020280C0020E0
:10ABC0002DE9F043DFF86C8187B0C146574B1B6815
:10ABD0001F68D7F1010738BF002717B9DB681D6868
:10ABE00000E0002500F082FD00F088FDD8F800307C
:10ABF0009842064603D2FFF7A9FF012300E0002395
:10AC0000C9F80060002B32D12FBBB54223D800F029
:10AC100009FE464B1B68DB68DC68201D00F0C0F8AD
:10AC2000E369012B13D1A1692046691832462B46EE
:10AC3000FFF70CFF01280AD10097204639462A4623
:10AC40003B46FFF761FF10B901F0F6F8FEE7636AD3
:10AC5000204698475FE0364BA91B186800F08EFB32
:10AC600000F0E0FD002856D101F0DAF853E000F0E2
:10AC7000D9FD50E0039B002B4EDB059C636913B1AB
:10AC8000201D00F08DF800F039FDD8F80030984212
:10AC9000054601D2FFF75AFF039BC9F80050092B64
:10ACA0003AD84FF004629A4024D44FF063429A405D
:10ACB00004D44FF080629A4029D42DE0049BA1690E
:10ACC000204659182A46FFF7C1FE012824D1636A9D
:10ACD00020469847E369012B1ED1A269049B0021FD
:10ACE000D218009120460B46FFF70EFFA0B901F0E5
:10ACF000A3F8FEE70499A16111B901F09DF8FEE700
:10AD0000204669182A462B46FFF7A0FE04E020469D
:10AD100001F02EFA00E0064E0022306803A9134627
:10AD200000F07AFA0028A5D150E700BFF40B00200C
:10AD3000240C0020200C0020006A704700F108035A
:10AD400043604FF0FF32C360036100238260036001
:10AD50007047002303617047436808619A684B603D
:10AD60008A609A6899600368516001330360704794
:10AD70000A68531C30B501D1036907E000F10803EC
:10AD800000E023465C6825689542FAD95A68086154
:10AD90004A60916059608B6003680133036030BD85
:10ADA0004168826803698A6082685160596881429B
:10ADB00008BF5A60002202611868013818607047A5
:10ADC00038B5044604F1240501F03EF80AE0636A50
:10ADD0005BB1284600F0CEFE08B100F045FFA36C41
:10ADE000013BA364A36C002BF1DC4FF0FF33A364A1
:10ADF00001F056F804F1100501F026F80AE0236985
:10AE00005BB1284600F0B6FE08B100F02DFF636C80
:10AE1000013B6364636C002BF1DC4FF0FF33636430
:10AE2000BDE8384001F03CB8026C30B503466AB169
:10AE3000C4684568A418AC42C46024BF0468C460F8
:10AE40000846D968BDE83040F6F72CBF30BD38B5AC
:10AE50001546026C04463AB9056805B128E0406819
:10AE600000F064FF656024E06DB98068F6F71AFFB2
:10AE7000A268236CD3186268A360934218D3236836
:10AE80002846A36015E0C068F6F70CFF236CE26863
:10AE900021685B42D2188A42E26002D26268D3180B
:10AEA000E360022D04D1A36B13B1A36B013BA36339
:10AEB0000020A36B0133A36338BD38B50D460446AB
:10AEC00010B900F0B9FFFEE700F0BEFF2368E06BA9
:10AED000226CA36000FB0231013802FB0033616089
:10AEE000E36000214FF0FF33A1636364A36455B9AD
:10AEF000236983B104F1100000F03CFE01280AD15F
:10AF000000F08EFF07E004F11000FFF717FF04F1D7
:10AF10002400FFF713FF00F0C3FF012038BDF8B590
:10AF20000D461746064610B900F086FFFEE711B140
:10AF30004843013000E00846543001F093F80446DD
:10AF400038B10DB9206007E000F15403036003E05D
:10AF5000FEE700F071FFFBE7E66325642046012170
:10AF6000FFF7ABFF84F850702046F8BD10B50C46D3
:10AF700010B900F061FFFEE7814202D900F05CFFEA
:10AF8000FEE700210222FFF7CAFF10B1846310BD63
:10AF9000FEE700F051FFFBE72DE9F04385B00F46D7
:10AFA00001921D46044610B900F046FFFEE7002955
:10AFB0007BD1036C002B78D074E0FEE7E36B012BB0
:10AFC00076D178E0FEE7019E26B179E0FEE7012622
:10AFD00002E000264FF0000800F036FFA26BE36BA2
:10AFE0009A4201D3022D15D1204639462A46FFF751
:10AFF0002EFF636A43B104F1240000F0BBFD012879
:10B0000004D100F00DFF01E00028FAD100F048FF64
:10B01000012058E0DDF80490B9F1000F02D100F0F2
:10B020003FFF3DE016B902A800F0E0FD00F038FF58
:10B0300000F05CFB00F008FF636C013308BFC4F84C
:10B040004480A36C013308BFC4F8488000F028FF97
:10B0500002A801A900F0DAFDE8B900F0F5FED4F885
:10B060003890E66B00F01CFFB1450ED104F11000E2
:10B07000019900F023FD2046FFF7A2FE00F0D2FB6D
:10B080000028A4D100F0CCFEA1E72046FFF798FEEF
:10B0900000F0C8FB9BE72046FFF792FE00F0C2FBE2
:10B0A000002010E000F0C8FE87E7022D03D185E7FD
:10B0B00000F0C2FE86E700F0DDFD002889D182E7BE
:10B0C00000F0BAFE82E705B0BDE8F08370B5064631
:10B0D000542000F0C7FF044608B103E0FEE700F08B
:10B0E000ABFEFBE701230025C3634FF0FF3385630D
:10B0F00045604364056083648560C560056480F8CD
:10B1000050601030FFF71AFE04F12400FFF716FE1E
:10B11000204629462A462B46FFF73EFF204670BDB3
:10B120002DE9F0410F4616461D46044610B900F0C1
:10B1300083FEFEE741BB036C33B322E0FEE7E36B23
:10B14000012B24D126E0FEE7022D18D120463946F6
:10B150002A46FFF77CFEA36C01330BD1636A03B967
:10B160000BE004F1240000F005FD30B12EB1012404
:10B17000346019E0A36C0133A364012414E00024BB
:10B1800012E000F059FED9E7022D03D1D7E700F015
:10B1900053FED8E700F020FF00F04EFEA26BE36BF9
:10B1A0009A428046D0D2D1E7404600F075FE204654
:10B1B000BDE8F081F8B50D46044610B900F03CFE3C
:10B1C000FEE7066C16B100F037FEFEE700F004FF64
:10B1D00000F032FEA26BE36B9A42074616D2A36BD5
:10B1E0000133A363A36C01330BD1636A03B90BE092
:10B1F00004F1240000F0BEFC30B12DB101242C601C
:10B2000005E0A36C0133A364012400E03446384612
:10B2100000F042FE2046F8BD2DE9F04385B00E4611
:10B2200001929946044610B900F006FEFEE7002997
:10B2300040F08980036C002B00F0858080E0FEE701
:10B24000019D25B185E0FEE7012501E000250027ED
:10B2500000F0FAFDA36B3BB320463146E568FFF7EB
:10B26000E3FDB9F1000F12D1A36B013BA363236887
:10B2700013B900F099FD606023698BB104F11000EF
:10B2800000F078FC01280BD100F0CAFD08E0636AE9
:10B29000E5602BB104F1240000F06CFC0028F3D130
:10B2A00000F0FEFD012057E0DDF80480B8F1000F4A
:10B2B00002D100F0F5FD41E015B902A800F096FCBE
:10B2C00000F0EEFD00F012FA00F0BEFD636C0133F9
:10B2D00008BF6764A36C013308BFA76400F0E0FDFA
:10B2E00002A801A900F092FC18BB00F0ADFDA56B0F
:10B2F00000F0D6FDBDB9236833B900F0A5FD606844
:10B3000000F0C8FC00F0CCFD04F12400019900F02D
:10B31000D5FB2046FFF754FD00F084FA002893D1B6
:10B3200000F07EFD90E72046FFF74AFD00F07AFA34
:10B330008AE72046FFF744FD00F074FA00200BE096
:10B3400000F07AFD7BE700F095FC00287FF47EAFEB
:10B3500076E700F071FD76E705B0BDE8F08310B543
:10B36000044610B900F068FDFEE700F06DFDA36B28
:10B37000E46BE41A00F094FD204610BD38B5044695
:10B380000D4600F061FD636C013301D1002363645D
:10B39000A36C013301D10023A36400F081FDA36BF2
:10B3A00023B904F12400294600F0BCFB2046BDE887
:10B3B0003840FFF705BD0000064A13681968064BC0
:10B3C00011B94FF0FF3203E01268D268D2685268B8
:10B3D0001A607047300C0020080700200E4B1A68D6
:10B3E00010B550600D4A12689042044607D20C4ACC
:10B3F000106819680431BDE81040FFF7B9BC094A6C
:10B40000106819680431FFF7B3FC074B1A689442BF
:10B4100038BF1C6010BD00BFE00C0020FC0C0020F9
:10B42000000D0020300C0020080700202DE9F84F07
:10B430000A9DDDF82C800C9E0F4693469A46814665
:10B4400010B900F0F9FCFEE7042D02D900F0F4FC7D
:10B45000FEE736B9900000F005FE0646002800F031
:10B460009E805C2000F0FEFD044678B106634FEA42
:10B470008B023046A521F6F7CFFC236B0BF1FF3B87
:10B4800003EB8B0B2BF0070B002603E0304600F09C
:10B490006FFE84E0A319BA5D83F83420BB5D13B15D
:10B4A0000136102EF6D10026271D384684F8436059
:10B4B000E562E5642665FFF74CFC04F11800FFF730
:10B4C00048FCC5F1050366652461A361646284F8E4
:10B4D000586058464946524600F082FC2060B8F158
:10B4E000000F01D0C8F8004000F0AEFC2E4A1368EF
:10B4F000013313602D4B1E6836BB1C601368012B93
:10B500002AD1DFF8D0804FF0140909FB06800136FC
:10B51000FFF714FC052EF8D1DFF8BC80244E40461E
:10B52000FFF70CFC3046FFF709FC2248FFF706FC4A
:10B530002148FFF703FC2148FFF700FC204BC3F82C
:10B540000080204B1E6007E01F4A126822B91A686B
:10B55000D26AAA4298BF1C601C4A13680133136068
:10B560001B4A6364E36A1168012404FA03F001438F
:10B570001160184A142000FB03203946FFF7ECFB4A
:10B5800000F08EFC104B1B6833B1084B1B68DB6A64
:10B59000AB4201D200F044FC2046BDE8F88F4FF0EA
:10B5A000FF30BDE8F88F00BF080D0020E00C002040
:10B5B000500C0020E40C0020CC0C00200C0D0020CE
:10B5C000300C0020000D0020340C0020040D002061
:10B5D000200D0020680C00203C0C002038B50446EB
:10B5E00000F032FC0CB9224B1C68251D2846FFF7E1
:10B5F000D7FB68B9E26A1F4914235343CB583BB9C0
:10B600001D4B0120196800FA02F221EA02021A60B9
:10B61000A36A1BB104F11800FFF7C2FB17482946C3
:10B62000FFF79AFB164B1A6801321A60154B1A681D
:10B6300001321A6000F034FC134B1B68002B15D04C
:10B640000B4B1B689C4209D1104B1B6813B100F0D7
:10B65000F3FBFEE7BDE8384000F0E2BB00F0F4FB8E
:10B66000FFF7AAFEBDE8384000F01ABC38BD00BFA5
:10B67000E00C0020680C0020200D0020CC0C0020E5
:10B68000380C0020040D0020340C0020F80C0020A1
:10B6900030B585B000248022009401940294039474
:10B6A0000E480F492346FFF7C1FE012805460FD17A
:10B6B000FFF7EAF9012805460AD100F0BDFB094B66
:10B6C0001D60094B1C6005B0BDE8304000F040BC77
:10B6D00015B900F0B1FBFEE705B030BDFDB80208BA
:10B6E00005940308340C0020FC0C0020024B1A685F
:10B6F00001321A60704700BFF80C0020014B186837
:10B70000704700BFFC0C00203B4B1B682DE9F04745
:10B71000002B5BD1394B1A6801321A601E688EB952
:10B72000374B1A68126812B100F086FBFEE7354A03
:10B73000196810681860344B11601A6801321A6079
:10B74000FFF73AFE314B1B6800249E4200D232E0E4
:10B750002B4FDFF8CC80DFF8BCA03B681B68002BC8
:10B760003AD12A4B4FF0FF321A6024E0274A136087
:10B7700021E005F104094846FFF712FBAB6A1BB153
:10B7800005F11800FFF70CFBEB6AD8F80010012256
:10B7900002FA03F214200A4300FB03A04946C8F84A
:10B7A0000020FFF7D9FA1A4BEA6A1B68DB6A9A4253
:10B7B00028BF0124D1E7164B1B68DB6A14225343D0
:10B7C000144AD358012B88BF01240CE0124B1A688D
:10B7D00001321A60002406E03B68DB68DD686B68B4
:10B7E0009E42C6D2C2E70D4B1B68002B18BF012436
:10B7F0002046BDE8F08700BFF80C0020FC0C0020BC
:10B80000300C0020000D00202C0C00200807002028
:10B81000E00C0020680C0020640C0020240D0020A7
:10B82000200D00202DE9F8432C4C236813B900F0BB
:10B8300003FBFEE700F008FB2368013B236023685D
:10B840000BB1002444E0264B1B680BBBF9E7F368FF
:10B85000DC6804F1040804F11800FFF7A1FA40467F
:10B86000FFF79EFAE36A2A68012707FA03F114201A
:10B870000A4300FB039041462A60FFF76DFA194B1B
:10B88000E26A1B68DB6A9A4206D3174B1F6003E02B
:10B89000164E174DDFF860903368002BD7D1154C4A
:10B8A00023686BB9104B1C68012CCAD10EE0FFF75E
:10B8B0002BFF08B1012333602B68013B2B6001E0B3
:10B8C000094E25462368002BF1D1EBE700F0A8FADA
:10B8D00000F0E6FA2046BDE8F88300BFF80C00202F
:10B8E000080D0020E00C0020240D0020E40C0020B6
:10B8F000200D0020640C0020680C0020F8B5144CCA
:10B90000144E154F2368E3B1FFF7F0FE3568FFF7DB
:10B9100089FF002DF6D000F097FAF368DD68281D46
:10B92000FFF73EFA3B68013B3B602368013B236025
:10B9300000F0B6FA286B00F01BFC284600F018FC5B
:10B94000E0E7064B1B68012BDCD900F069FAD9E768
:10B95000380C0020CC0C0020080D0020680C0020C2
:10B9600038B5044618B9BDE8384000F059BA114B53
:10B970001B6813B100F060FAFEE7FFF7B7FE0E4B4D
:10B980001D6865190D4C20680430FFF709FA48B9A5
:10B990000B4B19682268D26A012000FA02F221EAF0
:10B9A00002021A602846FFF719FDFFF73BFF002847
:10B9B000D9D038BDF80C0020FC0C0020E00C002091
:10B9C000200D002070B50C46054610B900F034FA81
:10B9D000FEE711B900F030FAFEE71C4B1E6816B105
:10B9E00000F02AFAFEE7FFF781FE194B2A68186873
:10B9F0009042144402D2944207D201E0944206D30A
:10BA0000844294BF0023012302E0334600E0012377
:10BA10002C6093B10F4D28680430FFF7C1F948B985
:10BA20000D4B19682A68D26A012000FA02F221EA55
:10BA300002021A602046FFF7D1FCFFF7F3FE18B9A7
:10BA4000BDE8704000F0ECB970BD00BFF80C0020FC
:10BA5000FC0C0020E00C0020200D002008B5124B4B
:10BA60001A68124B0AB101221CE01A60104B1A68C6
:10BA7000B2FA82F2D2B21423C2F11F020D495A4324
:10BA80008B188A5812B900F0D7F9FEE75A68526845
:10BA900003F108018A425A6004BF52685A605B6829
:10BAA000DA68054B1A6008BDF80C0020240D002050
:10BAB000200D0020680C0020E00C002038B50D4659
:10BAC00010B900F0B9F9FEE7124C21681831FFF700
:10BAD0004FF920680430FFF763F948B90E4B196835
:10BAE0002268D26A012000FA02F221EA02021A60F8
:10BAF000691C07D1074B094819680431BDE8384073
:10BB0000FFF72AB9064B18682818BDE83840FFF738
:10BB100065BC00BFE00C0020200D00200C0D0020B3
:10BB2000FC0C002038B50D4610B900F085F9FEE791
:10BB30000D4C21681831FFF70FF920680430FFF72A
:10BB40002FF948B9094B19682268D26A012000FA16
:10BB500002F221EA02021A60054B18682818BDE8B3
:10BB60003840FFF73BBC00BFE00C0020200D002058
:10BB7000FC0C002038B5C368DC6814B900F05CF92F
:10BB8000FEE704F118052846FFF70AF9114B1B6878
:10BB900083B9251D2846FFF703F90F4AE36A1068A9
:10BBA000012101FA03F1014311600C4A142000FB4A
:10BBB000032000E00A482946FFF7CEF8094BE26A65
:10BBC0001B68DB6A9A4203D9074B0120186038BD15
:10BBD000002038BDF80C0020200D0020680C00204B
:10BBE000E40C0020E00C0020240D002008B510B962
:10BBF00000F022F9FEE7034B1B680360024B1B6851
:10BC0000436008BD2C0C0020FC0C002038B50D460C
:10BC1000044610B900F010F9FEE711B900F00CF974
:10BC2000FEE700F011F90E4B1A682B68591C10D072
:10BC30000C49086821688842616801D08A420AD2AA
:10BC4000501A984207D28A1AD3182B602046FFF761
:10BC5000CDFF002400E0012400F022F9204638BD89
:10BC6000FC0C00202C0C0020014B01221A607047B4
:10BC7000240D0020054B1B6833B1054B18680028C4
:10BC80000CBF02200020704701207047340C0020B8
:10BC9000F80C0020F8B50446002840D0204AC36ABA
:10BCA0001168C96A8B423AD28169002904DB1268A3
:10BCB000D26AC2F1050282611A4E6269142707FB3B
:10BCC00003639A4227D11FE0E26A5743F3593BB915
:10BCD000154B0120196800FA02F221EA02021A60EB
:10BCE0000F4B114A1B681068DB6A012101FA03F14E
:10BCF000014311600B4AE362142000FB0320294634
:10BD0000BDE8F840FFF728B8251D2846FFF748F89A
:10BD10000028D9D0E4E7024B1B68DB6AE362F8BD78
:10BD2000E00C0020680C0020200D002038B50446EF
:10BD300008B9002038BD036D13B900F07DF8FEE7A7
:10BD4000C16AC26C013B91420365F2D0002BF0D175
:10BD5000051D2846FFF724F868B9E26A1049142344
:10BD60005343CB583BB90F4B0120196800FA02F23C
:10BD700021EA02021A60E36CC3F10502A261094ADA
:10BD8000E3621168012404FA03F001431160044ADC
:10BD9000142000FB03202946FEF7DEFF204638BDB5
:10BDA000680C0020200D0020044B1A681AB11A6894
:10BDB000116D013111651868704700BFE00C00205B
:10BDC00006480068006880F3088862B661B6BFF371
:10BDD0004F8FBFF36F8F00DF00BF000008ED00E062
:10BDE0004FF0807300E90A00034B40F8202C40F824
:10BDF0000C3C4038704700BF7DBE0208074B1968F5
:10BE00000868B0E8F00F80F30988BFF36F8F4FF038
:10BE1000000080F311884EF00D0E7047E00C0020FA
:10BE2000044B4FF080521A60BFF34F8FBFF36F8FF8
:10BE3000704700BF04ED00E0EFF311804FF05001B8
:10BE400081F311887047002008B5FFF7F5FF094A14
:10BE5000136801331360BFF34F8FBFF36F8F012B54
:10BE600007D1054B1B6813F0FF0F02D0FFF7E4FF6B
:10BE7000FEE708BD0C07002004ED00E008B5054B07
:10BE80001B68013302D0FFF7D7FFFEE7FFF7D4FFAF
:10BE9000FEE700BF0C07002080F311887047000008
:10BEA00008B5074B186810B9FFF7C6FFFEE7013861
:10BEB000186018B9BDE80840FFF7EEBF08BD00BF25
:10BEC0000C070020EFF30980BFF36F8F0D4B1A684A
:10BED00020E9F00F10602DE908404FF0500080F38A
:10BEE0001188FFF7BBFD4FF0000080F31188BDE81B
:10BEF000084019680868B0E8F00F80F30988BFF3BC
:10BF00006F8F7047E00C002008B5FFF795FFFFF733
:10BF1000FBFB18B1044B4FF080521A600020BDE8C3
:10BF20000840FFF7B9BF00BF04ED00E0064B1A68F8
:10BF30004FF47A73B2FBF3F2044B013A1A60072212
:10BF400043F8042C704700BFBC05002014E000E05B
:10BF500007B51D4B1A780192FF221A701B788DF8D5
:10BF600003309DF80320194B02F050021A70184A52
:10BF70000723136005E09DF803305B008DF8033064
:10BF80000B469DF80320591E1206F4D4104A1B02DA
:10BF900003F4E06313600C4B019A1A70D3F8202964
:10BFA00042F47002C3F82029D3F8202942F07042ED
:10BFB000C3F82029FFF7BAFF064B00221A60FFF7EB
:10BFC000FFFEFFF75BFF00BF00E400E0280D00204C
:10BFD0002C0D00200C07002008B5EFF305830F2B74
:10BFE00008D90A4A9B5C0A4A12789A4202D9FFF79A
:10BFF00023FFFEE7074B1A68074B1B6802F4E06259
:10C000009A4202D9FFF718FFFEE708BDF0E300E00F
:10C01000280D00200CED00E02C0D002010B50F4B7A
:10C0200000E013461A688242FBD359685C188442C8
:10C0300003D1406841185960184641684418944239
:10C0400006D1074C2468A24202D014CA611841608C
:10C050008342026018BF186010BD00BF380D002079
:10C06000340D0020F8B50546FFF740FB3A4B1B683E
:10C070001BBB3A4A560707D0D31D23F0070302F52E
:10C080007042D11A1A4601E04FF470415118083934
:10C0900021F007013248002380E80C000B604B6060
:10C0A0008B1A82E80A002F4A2B4813602E4A01603F
:10C0B00013602E4B4FF000421A602C4B1E68354225
:10C0C00040D1002D3FD005F1080358071CBF23F0D5
:10C0D00007030833002B33D0234A1768BB4231D8FB
:10C0E0001F4A146801E0224604466168994204D35D
:10C0F00019480068844204D124E020680028F2D165
:10C10000F6E7206815681060CA1A0835102A09D9A0
:10C11000E018410702D0FFF78FFEFEE74260636040
:10C12000FFF77CFF62681049BB1A0B600D49086875
:10C13000834238BF0B601643002384E8480002E0C6
:10C140001D4600E00025FFF76DFB6B0702D0FFF7EF
:10C1500073FEFEE72846F8BD340D002000000010F5
:10C16000380D0020400D0020300D0020440D00202F
:10C1700010B5044610B3124A50F8043C12681A4233
:10C1800002D1FFF759FEFEE750F8081C11B1FFF786
:10C1900053FEFEE723EA020340F8043CFFF7A6FA49
:10C1A000084B54F8041C1A68A4F108008A181A6095
:10C1B000FFF734FFBDE81040FFF734BB10BD00BFF0
:10C1C000440D0020300D0020014B00221A707047F2
:10C1D000580D00201B4B73B5002405460E461C600D
:10C1E0000AE0281918491022F6F750F818B9154B2B
:10C1F00010341C6002E00134B442F2D1114B1A68D1
:10C2000018460AB900201BE0AD18002302E00DF823
:10C2100003100133E95C0D2903EB0204F7D104603C
:10C22000002BEFD0013B012200200A2106E01DF87F
:10C230000340303C02FB0400013B4A43002BF6DA8A
:10C240007CBD00BF540D00205AB90308074B1422CF
:10C2500013B502FB00300469FFF750FA00230246D1
:10C26000009320460121FEF74FFC1CBD68E2002030
:10C2700070B5094C06460D4630466168F5F758FE24
:10C2800028B9A3682B60E36801206B6070BD246847
:10C29000002CF1D1204670BDC407040838B5082031
:10C2A0000C4603F09FFA0146A0B1002505604560E9
:10C2B000204603F005FF2046084903F003FF20460F
:10C2C000074903F003FF204606490A2203F003FF53
:10C2D000284600E0FF2040B238BD00BFE9D2020886
:10C2E0002BC3020813C3020838B54B68B0F8665078
:10C2F0009D4228BF9DB20C462A460968002305F0DE
:10C3000044FA28B923685B19236063685D1B656084
:10C3100038BD08B50346084613B904F06FF902E0CA
:10C320001946FFF7E1FF002008BD03F093B938B5C7
:10C3300004460D46002103F0C3FE2046002103F011
:10C34000C3FE2046002103F0BDFE284603F082F91B
:10C350002046BDE8384004F051B908B50346084608
:10C360005A68194612B1FFF7BFFF01E0FFF7DFFF80
:10C37000002008BD70B5456804460E4625B1084644
:10C380002146FFF7B1FF36E04FF47A721B48294689
:10C39000F5F742FD1A4B18681A4B1A6800F520731E
:10C3A0009342194B03D815494FF4207203E0904291
:10C3B00005D21249121A1B78FDF776FF0546104B7D
:10C3C0001A68AA181A60104B00221A7045B9012287
:10C3D000304621461A70FFF7AAFF0C4B1D700AE089
:10C3E000064B3046214684E82800FFF77DFF3046A3
:10C3F000074903F069FE002070BD00BFD0CF0020C8
:10C400004C0D0020640D002011070020580D002065
:10C4100075C3020870B5456804460E4625B1084646
:10C420002146FFF761FF36E04FF47A721B48294638
:10C43000F5F7F2FC1A4B18681A4B1A6800F57A7374
:10C440009342194B03D815494FF47A7203E0904296
:10C4500005D21249121A1B78FEF736F80546104B22
:10C460001A68AA181A60104B00221A7045B90122E6
:10C47000304621461A70FFF75AFF0C4B1D700AE038
:10C48000064B3046214684E82800FFF72DFF304652
:10C49000074903F019FE002070BD00BFD0CF002077
:10C4A0004C0D0020640D002012070020580D0020C4
:10C4B00015C402081FB5FEF73FFC0A4B93F878330A
:10C4C000044673B1F9F7E0FF074902466846FBF7F7
:10C4D00063FB064BE0B2142200FB02306946F5F71D
:10C4E00015FE1FBDDCCB002076FF030868E20020AC
:10C4F000F0B587B004F0B0F9502204461349144F48
:10C50000144E03F00BFD2046FF2103F03FFD1249BE
:10C5100003F0DFFD0024F9F7B7FF1425024605FB01
:10C5200004750E4902A8FBF737FB02A92846F5F768
:10C53000EDFD00222346009609480A49FEF7C4FA99
:10C540000134022C2861E6D107B0F0BD784504081B
:10C5500068E20020B5C402089DC2020876FF030805
:10C5600079FF030840771B0070B5024688B00C467F
:10C57000684611461E221E46F5F7DEFE68460B4948
:10C58000F5F70CFF0546012075B929464FF4FA620C
:10C590002046F5F741FC204601F016FD2046F5F750
:10C5A00013FE30802846FFE708B070BD83FF030804
:10C5B00070B5024688B00C46684611461E221E46DB
:10C5C000F5F7BAFE68460B49F5F7E8FE0546012087
:10C5D00075B929464FF4FA622046F5F71DFC20464E
:10C5E00001F0E4FE2046F5F7EFFD30802846FFE736
:10C5F00008B070BD83FF030800B593B00146322236
:10C6000005A8F5F799FE684600211422F5F704FC09
:10C61000012002F0B7F813B000BD000030B593B0B0
:10C6200004460D46002002A90DF10702FBF79EFD0E
:10C630000021322205A8F5F7EFFB1B4B01221A70EF
:10C64000F9F722FF1949024605A8FBF7A5FA05A943
:10C650001748F5F75BFD0020FFF7F8FD1549204668
:10C66000F5F754FD02A92046F5F73CFC1249204697
:10C67000F5F738FC05A92046F5F734FC0F492046AC
:10C68000F5F730FC0E492046F5F72CFC0D49204605
:10C69000F5F728FC0C492046F5F724FC2046F5F771
:10C6A00093FD288013B030BD4B0D002076FF0308AA
:10C6B00068E2002085FF0308C1FF0308D3FF0308D9
:10C6C000E8FF0308F5060408FDFF03082DE9F04123
:10C6D00090461F46F5F7F8FF0546E0B10F49F5F71C
:10C6E0005DFE0F4906462846F5F758FE044620B978
:10C6F00028460C49F5F752FE0446A51B013D40466D
:10C70000711C2A46F5F718FE302323700120337080
:10C710003D70BDE8F0813870BDE8F08196030408F3
:10C720006900040801910308F0B5A9B00446142279
:10C730000D4607A800211F46F5F76EFB00211422C5
:10C740000CA8F5F769FB002132221BA8F5F764FB62
:10C75000312221461BA8F5F7EFFD0DF103064149F3
:10C760001BA8F5F7BFFB1BA83F4907AA3346FFF7F5
:10C77000ADFF20B93D4B00221A70012070E01BA8CC
:10C780003B490CAA3346FFF7A1FF0028F2D0002452
:10C79000204604A93246FBF7E9FC204601A93246AF
:10C7A000FBF7FAFC04A807A90B22F5F76FFD002898
:10C7B00051D101A80CA90B22F5F768FD00284AD138
:10C7C0002A4B01221A70F9F75FFE2A4902461BA87C
:10C7D000FBF7E2F9284B142000FB04301BA9F5F706
:10C7E00095FC2046FFF732FD24492846F5F78EFCDC
:10C7F00004A92846F5F776FB21492846F5F772FB90
:10C800001BA92846F5F76EFB22461E491BA8FBF71D
:10C81000C3F91D492846F5F765FB1BA92846F5F71E
:10C8200061FB1A492846F5F75DFB19492846F5F7DB
:10C8300059FB2846F5F7C8FC2821012C14BF154ADE
:10C84000154A388011A8FBF789F9052011A9FDF7D1
:10C8500061FC002004E00134E4B2022C8AD097E7A6
:10C8600029B0F0BD019103086B0004084B0D0020B6
:10C870007200040876FF030868E2002085FF0308C1
:10C88000C1FF0308A78F03087C000408F50604080D
:10C89000FDFF0308C79003089000040870B59CB022
:10C8A000322206460C4602A800211D468DF80710CC
:10C8B000F5F7B2FA28492046F5F728FC2749304613
:10C8C00002AA0DF10703FFF701FF02A82449F5F7BB
:10C8D0002FFB78B90720FCF7D5FE40B2012806D11E
:10C8E00007202049FDF716FC20461F492BE0204673
:10C8F0001E4928E01E4902A80522F5F7C7FC01469B
:10C9000038BB32220FA8F5F787FA0FAA0DF10703FB
:10C9100018493046FFF7DAFE0FA8F5F759F9F4F792
:10C920006DF9154B18600520FCF7ACFE40B20128EC
:10C93000204607D11149F5F7D5FA07201049FDF730
:10C94000E9FB02E00F49F5F7CDFA2046F5F73CFC8C
:10C9500028801CB070BD00BF5C170408A900040843
:10C96000AF000408B6000408E10004082001040830
:10C970007301040877010408740B00207E01040889
:10C98000C7900308AC010408F0B500268DB0074637
:10C990000C461422314602A81D468DF80760F5F7B3
:10C9A0003BFA1422314607A8F5F736FA2B49204600
:10C9B000F5F7ACFB2A49384602AA0DF10703FFF749
:10C9C00085FE02A82749F5F7B3FA98B90820FCF7C5
:10C9D00059FEC6B2012E07D823492046F5F782FA40
:10C9E00006202249FDF796FB76B2721C30D1204614
:10C9F0001F492BE002A81F49F5F79AFA08B902204F
:10CA000012E002A81C490622F5F740FC20BB0DF1FC
:10CA100007031A4907AA3846FFF758FE07A8F5F793
:10CA2000DBF8174B18800320FCF72CFEC6B2012E52
:10CA300007D814492046F5F755FA06201249FDF7A4
:10CA400069FB76B2731C03D110492046F5F74AFA08
:10CA50002046F5F7B9FB28800DB0F0BD5C1704083F
:10CA6000A9000408EE010408F3010408B600040854
:10CA70001202040845020408C502040896030408CB
:10CA8000780B00204F02040868020408940204088E
:10CA900030B50024BBB0054621466E2202A88DF8B1
:10CAA0000740F5F7B9F90DF1070302AA28461E4918
:10CAB000FFF70CFE6E2102AA1EA8FCF7A1FE1EA81D
:10CAC000FBF758FD21466E2202A8F5F7A5F90DF1F6
:10CAD000070302AA28461549FFF7F8FD6E2102AAAE
:10CAE0001EA8FCF78DFE1EA8FBF754FD21466E2202
:10CAF00002A8F5F791F90DF1070302AA28460C499F
:10CB0000FFF7E4FD6E2102AA1EA8FCF779FE1EA81D
:10CB1000FBF74EFD21466E2202A8F5F77DF901F0E4
:10CB2000FBFD3BB030BD00BFCA020408D1020408BF
:10CB3000DE02040830B50025A3B004464022294691
:10CB400002A88DF80750F5F767F94022294612A888
:10CB5000F5F762F90DF10703B54902AA2046FFF780
:10CB6000B5FD02A8FBF7B4FC4022294602A8F5F760
:10CB700053F90DF10703AF4902AA2046FFF7A6FDBE
:10CB800002A8FBF7ABFC4022294602A8F5F744F9BE
:10CB90000DF10703A84902AA2046FFF797FD02A856
:10CBA000FBF7A2FC4022294602A8F5F735F90DF162
:10CBB0000703A24902AA2046FFF788FD02A8FBF757
:10CBC000A1FC4022294602A8F5F726F90DF107033A
:10CBD0009B4902AA2046FFF779FD02A8FBF7A0FCBB
:10CBE0004022294602A8F5F717F90DF107039549E8
:10CBF00002AA2046FFF76AFD02A8FBF79FFC40222D
:10CC0000294602A8F5F708F90DF107038E4902AA93
:10CC10002046FFF75BFD02A8FBF79EFC4022294659
:10CC200002A8F5F7F9F8894902AA0DF10703204691
:10CC3000FFF74CFD02A8FBF739FC02A88449022249
:10CC4000F5F724FB002831D02946402202A8F5F749
:10CC5000E3F80DF107037F4902AA2046FFF736FDEE
:10CC600002A8FBF711FC2946402202A8F5F7D4F8E8
:10CC70000DF10703784902AA2046FFF727FD02A815
:10CC8000FBF708FC2946402202A8F5F7C5F87349CE
:10CC900002AA0DF107032046FFF718FD02A8FBF7D3
:10CCA000FFFB02A829464022F5F7B6F800214022F2
:10CCB00002A8F5F7B1F86A4902AA0DF10703204668
:10CCC000FFF704FD02A8FBF7ABFC614902A80222B2
:10CCD000F5F7DCFA0146002856D1402202A8F5F704
:10CCE0009BF8604902AA0DF107032046FFF7EEFC0E
:10CCF00002A8FBF783FC02A855490222F5F7C6FA01
:10CD00000546002840D12946402202A8F5F784F8BC
:10CD10000DF10703544902AA2046FFF7D7FC02A8E9
:10CD2000FBF74CFC2946402202A8F5F775F80DF1F7
:10CD300007034E4902AA2046FFF7C8FC02A8FBF7EA
:10CD400043FC2946402202A8F5F766F80DF10703D7
:10CD5000474902AA2046FFF7B9FC02A8FBF748FCA6
:10CD60002946402202A8F5F757F8424902AA0DF1D8
:10CD700007032046FFF7AAFC02A8FBF72FFC02A836
:10CD800029464022F5F748F80021402202A8F5F78D
:10CD900043F80DF1070302AA37492046FFF796FC36
:10CDA00002A80021FBF732FD0021402202A8F5F77E
:10CDB00033F80DF1070302AA30492046FFF786FC3D
:10CDC00002A80021FBF740FD0021402202A8F5F750
:10CDD00023F80DF1070302AA29492046FFF776FC44
:10CDE00002A80121FBF730FD0021402202A8F5F73F
:10CDF00013F8244902AA0DF107032046FFF766FC49
:10CE000002A8FBF787FC02A81F490122F5F73EFAAA
:10CE1000054602A8002D3FD129464022F4F7FCFF29
:10CE200020461A4902AA0DF10703FFF74FFC2FE035
:10CE3000E7020408F70204080803040813030408BF
:10CE40001F0304082B0304083703040843030408E2
:10CE5000E98F030849030408510304085503040833
:10CE60005B030408630304086F0304087A030408DF
:10CE7000830304088B03040893030408980304083D
:10CE80009D030408A2030408DF920308A703040813
:10CE900002A8FBF75FFC23E024490122F5F7F6F92D
:10CEA000054610BB0DF10703214902AA2046FFF7F2
:10CEB0000DFC02A8FBF7C6FB2946402202A8F4F7A6
:10CEC000ABFF1C4902AA0DF107032046FFF7FEFB4A
:10CED00012A8402102AAFCF793FC12A8FBF7EAFB78
:10CEE00002A829464022F4F797FF134902AA0DF140
:10CEF00007032046FFF7EAFB02A8FBF731FC0021FD
:10CF0000402202A8F4F788FF0AF074FC50B1012017
:10CF1000FBF7AEFA01F000FC40F2F230FEF720FD24
:10CF2000FCF7FEFB01F0F8FB23B030BD5390030883
:10CF3000C5030408B2030408B80304082DE9F0414E
:10CF400090461F46F5F7C0FB0546E0B10F49F5F7DF
:10CF500025FA0F4906462846F5F720FA044620B977
:10CF600028460C49F5F71AFA0446A51B013D404630
:10CF7000711C2A46F5F7E0F9302323700120337045
:10CF80003D70BDE8F0813870BDE8F081960304087B
:10CF9000AA910308F806040810B508490446F5F7F5
:10CFA00093FB48B1021B92B2C2F5BB62002103326F
:10CFB000BDE81040F4F730BF10BD00BFBD0304084A
:10CFC000F0B5002587B006460C464FF4FA620846D5
:10CFD00029461F468DF80350F4F71EFF3046FFF731
:10CFE000DBFF2946142201A8F4F716FF01AA0DF170
:10CFF00003030B493046FFF769FB9DF8031001A8B6
:10D00000FBF7A0FE01A8F9F77BFD06492046F5F7DE
:10D010007DF82046F5F7D8F8388007B0F0BD00BF9E
:10D02000C2030408CB030408F0B5002587B0074607
:10D030004FF47A7208460C4629461E468DF8035076
:10D04000F4F7EAFE3846FFF7A7FF2946142201A8A5
:10D05000F4F7E2FE1D49384601AA0DF10303FFF77C
:10D0600035FB01A81A49F4F763FFE8B9FDF798F812
:10D0700008B9012028E0174D2B78002BF9D1164A6A
:10D080001360FDF79FF8154B15498001C21C1A600B
:10D090002046144BFAF780FD2046F5F795F801235A
:10D0A00030802B7002200FE0FDF77AF80028E0D0E6
:10D0B00001A8F4F791FD0146204601F0B7FA204699
:10D0C000F5F782F83080284607B0F0BDFB0304086E
:10D0D00001040408580D00204C0D0020640D0020B0
:10D0E0000504040894B90308F0B5002587B0074685
:10D0F0004FF47A7208460C4629461E468DF80350B6
:10D10000F4F78AFE3846FFF747FF2946142201A8A4
:10D11000F4F782FE1E49384601AA0DF10303FFF71A
:10D12000D5FA01A81B49F4F703FFF0B9FDF738F869
:10D1300008B9012029E0184D2B78002BF9D1174AA6
:10D140001360FDF72BF964225043154B1549C21C9F
:10D150001A602046144BFAF71FFD2046F5F734F805
:10D16000012330802B7002200FE0FDF719F8002812
:10D17000DFD001A8F4F730FD0146204601F0F4F9B4
:10D180002046F5F721F83080284607B0F0BD00BFF3
:10D19000FB03040801040408580D00204C0D002076
:10D1A000640D00200504040894B903082DE9F0413A
:10D1B000B0B005460C46142200210AA81E46F4F71A
:10D1C0002BFE002114220FA8F4F726FE05AF002144
:10D1D000322214A8F4F720FE002114223846F4F776
:10D1E0001BFE2846FFF7D8FE6E22294614A8F5F745
:10D1F000A3F80DF1060833492046F4F787FF14A879
:10D2000031490AAA4346FFF761FA00284ED014A814
:10D210002E490FAA4346FFF759FA002846D00025A9
:10D22000002114223846F4F7F7FD00210B2202A852
:10D23000F4F7F2FD284602A94246FAF797FF28467E
:10D2400039460DF10702FAF7A7FF02A80AA90B2237
:10D25000F5F71CF818BB39460FA80B22F4F7F0FCC1
:10D260000146E0B914220FA8F4F7D6FD14A8184916
:10D270000FAA4346FFF72AFAC0B1164B172202FB4A
:10D2800005300FA90B220530F4F70CFD01F044FA2C
:10D2900003201149FCF73EFF2046104908E0013504
:10D2A000EDB2022DBCD120460D4901E00D492046CA
:10D2B000F4F718FE2046F4F787FF3080002030B0E6
:10D2C000BDE8F0815C1704082F0404083904040841
:10D2D00042040408F4CE0020C79003084B0404085D
:10D2E000AC040408760404082DE9F04F9BB01746FF
:10D2F000002204460D468DF80A208DF80B2003927B
:10D300000492002B40F02B85002F00F02885084662
:10D31000398902F0A3FED4F80090B9F1000F40F073
:10D320001B85DFF8E8B27E683A89DFF8DCA2584650
:10D330003146AAF80020F4F7B5FCBAF80030A0494D
:10D340000BF803905846F5F7BFF90DF1340A014682
:10D3500032225046F4F7F0FF4946102205A8F4F7B0
:10D360005BFD0DF10A0305AA95495046FFF7E6FD5E
:10D3700058469449F5F7A8F90DF1240B01463222DD
:10D380005046F4F7D9FF494610225846F4F744FDB9
:10D390000DF10B0350468B495A46FFF7CFFD8A4BE0
:10D3A0001B68002B34D1894B1B68002B30D1884A75
:10D3B000FF219946874B1170142202FB09328649DE
:10D3C00001935046FAF7E8FB5046F4F7FDFE02469B
:10D3D0008DF80B00D2B258465146F4F757FF5FFA6A
:10D3E00089F87E4A019B40B9404679490192FAF793
:10D3F000E9FE019A012313700AE00021117009F17E
:10D400000109734AFF21B9F1020F1170D4D1C84646
:10D410006D4B1A68714B02B102E06C4A12680AB196
:10D4200001221A701B78002B40F014816C4B93F88A
:10D43000783343B9DFF8E8816A4E40463146FFF75A
:10D44000EDF800F072BC304667490D22F4F71EFF7C
:10D4500000B905E1304665490E22F4F717FF00B91F
:10D4600006E1304662491022F4F710FF00B907E1E7
:10D47000304660490C22F4F709FF00B910E130464C
:10D480005D490F22F4F702FF18B15C4B1B68002BBB
:10D490007ED030463989DFF88081FEF79BFEFF2879
:10D4A000C8F800006BD85648DFF85C9100214FF4B3
:10D4B0008072F4F7B1FC4FF000080BE006EB0800B7
:10D4C00050490422F4F7E2FE10B908F1040807E01D
:10D4D00008F10108B9F800309845EFD34FF0000883
:10D4E000494BB3F800A0B8F1000F2BD0DFF828911A
:10D4F0004348D9F80020C8EB0A0A92450CD2434BA6
:10D50000354A5146FAF72AFBD9F80030CAEB030333
:10D51000C9F8003000F020BC06EB0801F4F784FEE7
:10D520003748DFF8FC802F4EF4F74EFE414682B2BA
:10D5300033463348FFF7F8F8002873D1C4F8008069
:10D54000338876E02D4E33680133012B336040F28F
:10D55000038403A92E48FEF78BFE039B2360049BE4
:10D56000284663602146FEF7BFFE2846294902F09F
:10D57000ABFD294BC6F80080C3F80080ECE32748D8
:10D58000FAF7BEFA1D4A0023C8F8003013605FE0C6
:10D59000214B1A68002A5BD031461948F4F744FE43
:10D5A0001748F4F711FE1E490E4B82B21448FFF7DC
:10D5B000BBF8B8BB1A4B23600A4B1B8839E000BF8D
:10D5C000BAFF0308CFFF03085C0D0020700D002098
:10D5D0001007002068E200202C0404084B0D0020F6
:10D5E000DCCB0020480D0020D8040408E604040821
:10D5F000F5040408060504081305040864E2002085
:10D6000064E10020F5060408740D002088DB00208A
:10D61000230504085BC3020890E200202F050408DC
:10D62000B8D300208F4803A9FEF722FE039B236096
:10D63000049B636028462146FEF756FE28468A4929
:10D6400002F042FD894A00231360894A136083E394
:10D65000844872E3304687490D22F4F717FE08B973
:10D6600085486AE3304685490E22F4F70FFE08B973
:10D67000834862E3304683491022F4F707FE08B975
:10D6800081485AE3304681490C22F4F7FFFD08B97E
:10D690007F4852E330467F490C22F4F7F7FD08B982
:10D6A0007D484AE330467D491222F4F7EFFD40B948
:10D6B0004046FEF7CBFD7A4B1B78002B40F03C83B5
:10D6C000EBE2304677490E22F4F7E0FD20B9404600
:10D6D000FEF7BCFD744830E3304674491122F4F77C
:10D6E000D5FD20B94046FEF7B1FD714825E330462F
:10D6F00070491522F4F7CAFD20B94046FEF7A6FD91
:10D700006D481AE330466D491022F4F7BFFD40B969
:10D710006B4E304600F050FB26603046F4F754FD67
:10D7200031E1304667491122F4F7B0FD90B95C4B06
:10D730001B78002B40F01083634BDFF88481634E2D
:10D74000634802221A70634B41461A883346FEF73B
:10D750000BFF2AE1304660491222F4F797FD20B111
:10D760005E4B1B68002B00F010814D4B1A78002A8D
:10D7700040F0F282594BD3F80080B8F1000F2FD15E
:10D78000574B4F48C3F80080564BDFF84891C3F819
:10D790000080F4F719FD414602464948F4F73CFB86
:10D7A00030463989FEF716FD4F4B186008E006EB4E
:10D7B00008004E490822F4F769FD38B108F1010864
:10D7C000B9F800309845F2D3444B2DE1B8F1000F81
:10D7D000FAD0404B1A88434BC8EB02021A6000E0B3
:10D7E00090463E4B1A68012A03D13D4A1268012A2D
:10D7F00006D01B68002B7DD1394B1B68002B79D1DB
:10D80000364B19681A4619B93549096801B922E039
:10D810001368012B22D1324B1B68012B1ED109E06A
:10D8200006EB090031490822F4F730FD58B109F13F
:10D83000010903E0DFF89CA04FF00009BAF80030BE
:10D840009945EDD300E0C846264B224A11881A6854
:10D850008A181A60214B1A6801321A600022244B80
:10D860004DE000BF230504085BC3020890E20020DE
:10D8700064E20020D8040408DC040408E604040878
:10D88000EA040408F5040408F90404084805040837
:10D890004C050408060504080A0504085505040893
:10D8A000100700207405040878050408830504089F
:10D8B000870504089505040899050408AB050408C4
:10D8C000B8D30020BC0504084A0D0020480D0020F4
:10D8D00088DB0020740D0020CE050408700D0020A8
:10D8E000500D0020680D00206C0D0020E10504089B
:10D8F000600D0020994A9A4B11881A688A181A609C
:10D90000964B1A8806EB0801C8EB02081FFA88F24A
:10D910001A80944BDFF884821868101818609048B9
:10D92000D8F800300068984240F010818E4E3046A2
:10D93000F4F77AFC01228D493046F4F775FC304645
:10D94000F4F742FC81B23046FFF7F4F8884B00212F
:10D950001960884BD8F8002019603046F4F75CFA5B
:10D9600085493046F4F7D2FB84493046F4F7BAFAD9
:10D9700083493046F4F7B6FA3046F4F725FC814B7C
:10D980001880266080B26060DEE130467E490D225C
:10D99000F4F77CFC68B9714BDFF8CC81794E1A88BA
:10D9A0007A4841463346FEF703FE002840F0D48112
:10D9B000BBE1304676490E22F4F768FC20B1754B86
:10D9C0001B68002B00F0F080734B1A78002A40F09F
:10D9D000C381704BD3F80080B8F1000F35D1654B8F
:10D9E0006148C3F800805E4BDFF87091C3F8008097
:10D9F000F4F7EAFB414602465B48F4F70DFA30467D
:10DA00003989FEF7E7FB654B186008E006EB080074
:10DA100063490522F4F73AFC68B108F10108B9F846
:10DA200000309845F2D35B4B1A6801321A60514BB3
:10DA300001221A6090E1B8F1000FF4D0474B1A8828
:10DA4000474BC8EB02021A6000E09046514B1A683F
:10DA5000012A03D1474A1268012A06D01B68002B0D
:10DA600034D1444B1B68002B30D14A4B19681A46FD
:10DA700019B94049096801B922E01368012B22D184
:10DA80003C4B1B68012B1ED109E006EB0900444901
:10DA90000522F4F7FBFB58B109F1010903E0DFF8B7
:10DAA000BCA04FF00009BAF800309945EDD300E072
:10DAB000C8462B4B294A11881A688A181A60354BB8
:10DAC0001A6801321A600022264B04E0234A244BD4
:10DAD00011881A688A181A60204B1A8806EB080108
:10DAE000C8EB02081FFA88F21A801E4BDFF8AC80E0
:10DAF0001868101818601A48D8F800300068984262
:10DB000024D1194E3046F4F78FFB012217493046D5
:10DB1000F4F78AFB3046F4F757FB81B23046FEF744
:10DB2000B7FF1C4B00211960124BD8F80020196078
:10DB30003046F4F771F910493046F4F7E7FA0F4927
:10DB40003046F4F7CFF93046164913E7002A00F0C3
:10DB500003810548F4F768FBFEE000BF740D002068
:10DB6000680D0020600D0020B8D30020019103084B
:10DB7000700D0020500D0020EB050408F506040888
:10DB8000FD050408480D00206C06040888DB002011
:10DB90007A0604085C0D0020100700206C0D0020A0
:10DBA000890604088F06040830466F491022F4F7EE
:10DBB0006DFBE8B96D4E6E4BDFF8C4811A886D4875
:10DBC00033464146FFF790FA022833460AD133889C
:10DBD000C4F80080284621466360FEF785FB28468E
:10DBE00065491FE0002840F0B780C4F8008026E0B7
:10DBF000304662491322F4F749FB10BB5C4B5D4889
:10DC00001A885F49594BFFF70FFA022811D15C4B74
:10DC10002360564B1B88284621466360FEF764FB51
:10DC20005849284602F050FA2846574902F04EFA61
:10DC300092E0002840F09080514B23604B4B1B88B2
:10DC400081E0304651491122F4F720FB50B9DFF84A
:10DC50003081464E464B47481A8841463346FEF7C8
:10DC600093FE62E030464A491222F4F70FFB50B9A6
:10DC7000DFF80C813D4E3E4B3E481A884146334604
:10DC8000FEF70CFE51E0304642490E22F4F7FEFA50
:10DC900028B900F02DFD00F03FFD3F484DE0304633
:10DCA0003E490F22F4F7F2FA10B900F061FD53E09B
:10DCB00030463B491022F4F7E9FA20B9FAF7D8FBCD
:10DCC000FAF7DCFB38E0304636491222F4F7DEFA88
:10DCD00050B9DFF8AC80254E254B26481A884146BE
:10DCE0003346FEF789FC20E030462F491222F4F734
:10DCF000CDFA50B9DFF888801C4E1D4B1D481A889C
:10DD000041463346FFF752FA0FE0304627491322C7
:10DD1000F4F7BCFA68B9164BDFF86480134E1A8822
:10DD2000144841463346FFF74BF9C4F80080338866
:10DD300009E04046FEF78AFA1D4803A9FEF798FA63
:10DD4000039B2360049B636028462146FEF7CCFAC0
:10DD50002846184902F0B8F9384601F0EDFE0020D7
:10DD60001BB0BDE8F08F00BFFA060408480D002084
:10DD7000740D002088DB002015C402080B0704087E
:10DD8000B8D3002075C30208C9C1020820070408DF
:10DD90003207040845070408590504085407040815
:10DDA0006407040875070408880704089B0704082B
:10DDB000680504085BC3020810B54FF47A728CB092
:10DDC00004460021F4F728F820466F49F4F79EF93D
:10DDD00002A80DF10701F9F717FF20466B49F4F788
:10DDE00081F89DF8072002A92046F4F71DFA02A841
:10DDF0000DF10701F9F71EFF20466549F4F772F8A7
:10DE00009DF8072002A92046F4F70EFA02A80DF1AA
:10DE10000701F9F7CDFE20465E49F4F763F89DF857
:10DE2000072002A92046F4F7FFF902A80DF1070127
:10DE3000F9F7D4FE20465849F4F754F89DF8072026
:10DE400002A92046F4F7F0F902A80DF10701F9F74D
:10DE500007FF20465149F4F745F89DF8072002A92D
:10DE60002046F4F7E1F902A80DF10701F9F70AFFDE
:10DE700020464B49F4F736F89DF8072002A92046C2
:10DE8000F4F7D2F902A80DF10701F9F71FFF2046B8
:10DE90004449F4F727F89DF8072002A92046F4F733
:10DEA000C3F902A80DF10701F9F7FEFE20463E492D
:10DEB000F4F718F802A99DF807202046F4F7B4F902
:10DEC000002202A80DF10701FAF704F820463749AD
:10DED000F4F708F802A99DF807202046F4F7A4F902
:10DEE00002A80DF107010022FAF72EF8204630496A
:10DEF000F3F7F8FF02A99DF807202046F4F794F9FC
:10DF0000012202A80DF10701FAF71EF8204629495F
:10DF1000F3F7E8FF9DF8072002A92046F4F784F9FB
:10DF200002A80DF10701F9F7E7FE20462249F3F7B1
:10DF3000D9FF9DF8072002A92046F4F775F902A839
:10DF40000DF10701F9F702FF20461C49F3F7CAFF5C
:10DF50009DF8072002A92046F4F766F902A80DF102
:10DF60000701FAF75FFA20461549F3F7BBFF02A94C
:10DF70009DF807202046F4F757F920461149022260
:10DF8000F4F752F90CB010BDD0410408FC4104086C
:10DF9000044204080D4204081B4204082A420408F3
:10DFA0003442040842420408534204086742040809
:10DFB000714204087B420408854204089342040825
:10DFC000A1420408BB42040810B5BF498AB0044608
:10DFD000F4F79CF802A80DF10701FAF753F920466F
:10DFE000BA49F3F77FFF9DF8072002A92046F4F70E
:10DFF0001BF902A80DF10701FAF754F92046B449BC
:10E00000F3F770FF9DF8072002A92046F4F70CF9FA
:10E0100002A80DF10701FAF755F92046AD49F3F7CB
:10E0200061FF9DF8072002A92046F4F7FDF802A839
:10E030000DF10701FAF756F92046A749F3F752FF09
:10E040009DF8072002A92046F4F7EEF802A80DF18A
:10E050000701FAF757F92046A049F3F743FF9DF867
:10E06000072002A92046F4F7DFF802A80DF1070106
:10E07000FAF758F920469A49F3F734FF9DF807203C
:10E0800002A92046F4F7D0F802A80DF10701FAF72B
:10E0900059F920469349F3F725FF02A99DF8072077
:10E0A0002046F4F7C1F8002202A80DF10701F9F7A4
:10E0B000FDFE20468C49F3F715FF02A99DF80720C5
:10E0C0002046F4F7B1F8002202A80DF10701F9F794
:10E0D00027FF20468549F3F705FF02A99DF8072091
:10E0E0002046F4F7A1F8012202A80DF10701F9F783
:10E0F00017FF20467E49F3F7F5FE9DF8072002A999
:10E100002046F4F791F802A80DF10701FAF764F838
:10E1100020467849F3F7E6FE9DF8072002A920463D
:10E12000F4F782F802A80DF10701FAF76BF8204620
:10E130007149F3F7D7FE9DF8072002A92046F4F7AE
:10E1400073F802A80DF10701FAF772F820466B493F
:10E15000F3F7C8FE9DF8072002A92046F4F764F8FB
:10E1600002A80DF10701FAF779F820466449F3F7A0
:10E17000B9FE9DF8072002A92046F4F755F802A839
:10E180000DF10701FAF740F920465E49F3F7AAFEC0
:10E190009DF8072002A92046F4F746F802A80DF1E1
:10E1A0000701FAF7DFF820465749F3F79BFE9DF881
:10E1B000072002A92046F4F737F802A80DF107015D
:10E1C000FAF7E0F820465149F3F78CFE9DF8072056
:10E1D00002A92046F4F728F802A80DF10701FAF782
:10E1E000F5F820464A49F3F77DFE9DF8072002A97D
:10E1F0002046F4F719F802A80DF10701FAF7D4F850
:10E2000020464449F3F76EFE9DF8072002A92046F8
:10E21000F4F70AF802A80DF10701FAF7E7F820462B
:10E220003D49F3F75FFE9DF8072002A92046F3F76A
:10E23000FBFF02A80DF10701F9F79AFD20463749C7
:10E24000F3F750FE9DF8072002A92046F3F7ECFFF4
:10E2500002A80DF10701F9F7A9FD20463049F3F7AF
:10E2600041FE9DF8072002A92046F3F7DDFF02A832
:10E270000DF10701F9F7C8FD20462A49F3F732FEF0
:10E280009DF8072002A92046F3F7CEFF02A80DF162
:10E290000701F9F7D3FD20462349F3F723FE9DF844
:10E2A000072002A92046F3F7BFFF02A80DF10701DE
:10E2B000F9F7D4FD20461D49F3F714FE9DF8072019
:10E2C00002A9204634E000BFD0410408BE42040841
:10E2D000D2420408E8420408F8420408094304084A
:10E2E0001A4304082B4304086742040871420408D7
:10E2F0007B4204083C430408494304085243040891
:10E300005D4304086743040872430408814304081A
:10E310008F4304089C430408A9430408B943040834
:10E32000C3430408CE430408D8430408E843040860
:10E33000F3F77AFF02A80DF10701F9F74FFD204628
:10E340001649F3F7CFFD9DF8072002A92046F3F701
:10E350006BFF02A80DF10701F9F798FD204610495F
:10E36000F3F7C0FD9DF8072002A92046F3F75CFFF4
:10E3700002A80DF10701FAF755F820460949F3F70D
:10E38000B1FD02A99DF807202046F3F74DFF204676
:10E3900005490222F3F748FF0AB010BDF243040812
:10E3A000FC430408A1420408BB42040810B56049BC
:10E3B0008CB00446F3F7AAFE02A80DF10701F9F7A5
:10E3C000FBFD20465B49F3F78DFD9DF8072002A970
:10E3D0002046F3F729FF02A80DF10701F9F712FE15
:10E3E00020465549F3F77EFD9DF8072002A92046F7
:10E3F000F3F71AFF02A80DF10701F9F715FE204601
:10E400004E49F3F76FFD9DF8072002A92046F3F768
:10E410000BFF02A80DF10701F9F718FE2046484945
:10E42000F3F760FD9DF8072002A92046F3F7FCFEF4
:10E4300002A80DF10701F9F71BFE20464149F3F749
:10E4400051FD9DF8072002A92046F3F7EDFE02A832
:10E450000DF10701F9F71EFE20463B49F3F742FD97
:10E460009DF8072002A92046F3F7DEFE02A80DF171
:10E470000701F9F721FE20463449F3F733FD9DF8F3
:10E48000072002A92046F3F7CFFE02A80DF10701ED
:10E49000F9F724FE20462E49F3F724FD9DF80720C6
:10E4A00002A92046F3F7C0FE02A80DF10701F9F713
:10E4B00027FE20462749F3F715FD9DF8072002A9FE
:10E4C0002046F3F7B1FE02A80DF10701F9F72AFE85
:10E4D00020462149F3F706FD9DF8072002A92046B2
:10E4E000F3F7A2FE02A80DF10701F9F72DFE204671
:10E4F0001A49F3F7F7FC9DF8072002A92046F3F725
:10E5000093FE02A80DF10701F9F78CFF204614498C
:10E51000F3F7E8FC02A99DF807202046F3F784FEF4
:10E52000204610490222F3F77FFE0CB010BD00BF59
:10E53000D04104080F4404081B440408274404087D
:10E540003544040845440408534404085F4404085F
:10E550006B4404087D4404088B4404089B4404086D
:10E56000A1420408BB42040830B5054687B00C46FA
:10E570002749F3F7CBFD28462649F3F7B3FC21469C
:10E580002846FBF711FF2846F3F71EFEADF80600FC
:10E5900080B2431EEC180021C0F10100E954241898
:10E5A000102202A8F3F738FCFBF7ECFE1A490246EA
:10E5B00002A8F9F7F1FA20461849F3F793FC02A9EB
:10E5C0002046F3F78FFC02A80DF10601F9F746FC8F
:10E5D00020461349F3F786FCBDF8062002A9204621
:10E5E000F3F722FE02A80DF10601F9F7F7FB20462A
:10E5F0000C49F3F777FC02A92046BDF80620F3F793
:10E6000013FE20460849F3F76DFC07B030BD00BF8C
:10E61000AF440408DB440408E6440408E944040861
:10E62000E8430408F2430408BB42040830B5054639
:10E6300087B00C462749F3F769FD28462649F3F7CA
:10E6400051FC21462846FBF7C3FD2846F3F7BCFDE5
:10E65000ADF8060080B2431EEC180021C0F10100A5
:10E66000E9542418102202A8F3F7D6FBFBF79EFD0D
:10E670001A49024602A8F9F78FFA20461849F3F71B
:10E6800031FC02A92046F3F72DFC02A80DF106018A
:10E69000F9F7E4FB20461349F3F724FCBDF8062004
:10E6A00002A92046F3F7C0FD02A80DF10601F9F713
:10E6B00095FB20460C49F3F715FC02A92046BDF84E
:10E6C0000620F3F7B1FD20460849F3F70BFC07B02D
:10E6D00030BD00BFAF440408DB440408E64404082E
:10E6E000E9440408E8430408F2430408BB42040870
:10E6F00008B5032009F04CFA06490120FBF70AFD92
:10E700004FF4FA70FDF72CF9FAF7C8FABDE80840A3
:10E71000FAF758BAC790030808B5FAF753FA03494D
:10E720000420BDE80840FBF7F5BC00BFC790030814
:10E7300010B5044623786BB1012009F029FA0220B4
:10E740000A49FBF7E7FCF9F787FEFFF7E5FF4FF40F
:10E75000FA6001E04FF47A70FDF702F940F2F2300E
:10E76000FDF7FEF8FAF7DCFFE4E700BFC790030807
:10E7700008B540F2F230FDF7F3F8BDE80840FAF7CB
:10E78000CFBF00001FB5074B074918700022009249
:10E7900001920292039205488022FCF747FE05B0E1
:10E7A00000BD00BF760D0020F544040831E70208E3
:10E7B0001E4B1B6807B513B11D4A106898471D48CA
:10E7C00001A903F00DFD019B1A78052AF7D8DFE8AF
:10E7D00002F00307151B2028986803680430EDE752
:10E7E000D968986891F82D2012F0600F02D008F0D7
:10E7F00071FB01E004F04EF908200EE003F108007F
:10E8000007C803F01FFC07E0D868196903F0C4FCCF
:10E8100002E09A68D86890470720019901F082F8D1
:10E82000CDE79A68D8689047C9E700BF800D0020FF
:10E830007C0D0020780D0020F8B50E4D2B680646A3
:10E840000F4693B1082001F057F8044678B1012330
:10E8500003708660C7602146284608F089FD38B1FC
:10E860000820214601F05EF801E0FA2000E0FF20D8
:10E8700040B2F8BD780D002037B504460D4600F0D3
:10E88000B3FE094B09481C60094B32211D6008F09A
:10E8900061FD032300930749074800224FF4C87322
:10E8A00008F0D7FD3EBD00BF800D0020780D002090
:10E8B0007C0D0020B1E7020800450408030A43EA82
:10E8C000002080B27047030A43EA002080B27047FC
:10E8D00000BA7047FFF7FCBF037B8B4203D00023D5
:10E8E0000173437343837047038B10B54469E41885
:10E8F00084F8F01041695C1C11FA84F1023381F84C
:10E90000F020038310BD038B4269D218013382F8D3
:10E91000F01003837047038B4269D21810B50C0ABC
:10E9200082F8F04042695C1C12FA84F2023382F8E9
:10E93000F010038310BD038B4269D21810B50C0E82
:10E9400082F8F04042695C1C12FA84F2C1F3074479
:10E9500082F8F04042699C1C12FA84F2C1F3072449
:10E9600082F8F0404269DC1C12FA84F2043382F827
:10E97000F010038310BD90B1038B4269D218FF21C0
:10E98000013382F8F0100383002105E04269D218B8
:10E99000013382F8F0100383038B432BF6D97047C1
:10E9A0002DE9F0410C4617460646002800F08E80FF
:10E9B000002900F08D8000204FF49A71024601F08A
:10E9C00008F92061002800F08580627B434B12B972
:10E9D0001A6801321A601B68426823600123626171
:10E9E000137062695370636996F826209A706369A0
:10E9F0000025DD702068D4F81480FFF769FFC8F89F
:10EA000004006369082F1D725D729D72DD721D73B3
:10EA10005D739D73DD7307D0042F05D0032F05D1DF
:10EA2000227B043A012A01D87268DA6000251D743D
:10EA30005D749D74DD741D755D759D75DD751D7648
:10EA40005D769D76DD7696F826106269ABB29942C6
:10EA500088BF73192A448CBF93F8273000230135EF
:10EA6000102D1377EFD1002319466269D2180133B4
:10EA7000402B82F82C10F8D10022104663699918B7
:10EA800001320023802A81F86C00F7D162696FF0AF
:10EA90007D00632182F8ED00532082F8EC1082F8AB
:10EAA000EE0082F8EF1023836269D21882F8F0300A
:10EAB0000133442BF8D1204635210122FFF714FF02
:10EAC00020463946FFF71FFF002004E0F22002E055
:10EAD000FA2000E0FF2040B2BDE8F08114070020DA
:10EAE00010B5044630B1006908B101F025F80023E3
:10EAF0002361636110BD000073B5046A00230546FD
:10EB0000636220460621FFF7E7FE284621460122E0
:10EB1000FFF746FF0646002830D102222046392161
:10EB2000FFF7E2FE2046A98CFFF7F5FE04222046FF
:10EB30003721FFF7D9FE20460121FFF7E4FE2046EA
:10EB40000321FFF7E0FE20461C21FFF7DCFE062133
:10EB50002046FFF7D8FE2046FFF70DFF218B2069E6
:10EB6000F03189B201F00FF80095606821690F4A11
:10EB7000432303F081FC2046FFF7B2FF637B0133A0
:10EB8000DBB2052B98BF4FF47A7263739ABF02FA17
:10EB900003F39BB24EF660234FF4FA7203F2F313C1
:10EBA00093FBF2F3638330467CBD00BF74450408D9
:10EBB00073B5046A054604212046FFF78DFE2846FA
:10EBC00021460322FFF7ECFE0646D8B90222204672
:10EBD0003921FFF789FEA98C2046FFF79CFE2046CD
:10EBE000FFF7C9FE218B2069F03189B200F0CBFF1D
:10EBF0000095606821690E4A432303F03DFC2046DE
:10EC0000FFF76EFF637B0133DBB2092B637304D81C
:10EC10004FF47A7253439BB201E042F210734FF407
:10EC2000FA7203F2F31393FBF2F3638330467CBD75
:10EC30007445040873B5046A054603212046FFF7AE
:10EC40004BFE284621460322FFF7AAFE064640BB9C
:10EC5000022220463921FFF747FE20464FF410716B
:10EC6000FFF759FE042232212046FFF73DFE606A7D
:10EC7000FFF730FE01462046FFF75DFE2046FFF716
:10EC80007AFE218B2069F03189B200F07CFF00957B
:10EC9000606821690E4A432303F0EEFB2046FFF72C
:10ECA0001FFF637B0133DBB2092B637304D84FF47E
:10ECB0007A7253439BB201E042F210734FF4FA723E
:10ECC00003F2F31393FBF2F3638330467CBD00BF82
:10ECD0007445040873B5046A054601212046FFF710
:10ECE000FBFD284621460322FFF75AFE0646002870
:10ECF00048D1022220463921FFF7F6FD2046A98C93
:10ED0000FFF709FE042232212046FFF7EDFD606A7D
:10ED1000FFF7E0FD01462046FFF70DFE04223621F5
:10ED20002046FFF7E1FD206AFFF7D4FD01462046AB
:10ED3000FFF701FE042220463721FFF7D5FD2046CC
:10ED40000121FFF7E0FD20460321FFF7DCFD20460F
:10ED50001C21FFF7D8FD06212046FFF7D4FD2046F1
:10ED6000FFF709FE218B2069F03189B200F00BFF1B
:10ED70000095606821690F4A432303F07DFB20461C
:10ED8000FFF7AEFE637B0133DBB2052B98BF4FF478
:10ED90007A7263739ABF02FA03F39BB24EF6602352
:10EDA0004FF4FA7203F2F31393FBF2F363833046EA
:10EDB0007CBD00BF7445040838B5046A05460821C7
:10EDC0002046FFF789FD284604F12401002207F0C0
:10EDD00061FF637B013363730123638338BD37B500
:10EDE0000546002859D0046A002C56D0636B581C85
:10EDF0000DD03C221E33B3FBF2F34FF6FF72934269
:10EE000028BF13469BB2A3830BB90123A383A36B33
:10EE1000591C0DD03C221E33B3FBF2F34FF6FF72A8
:10EE2000934228BF13469BB2E3830BB90123E383CC
:10EE3000E38BA28B9A4202D30BB10023A383A37B63
:10EE40000BB1A36A0BE094F824301A0601D4FF2317
:10EE500005E0BF2B8CBF6FF07F434FF6FF7300932D
:10EE6000E36A01932BB9636A009A134043F08073FD
:10EE70000193284604F1240100F06AFD2846694602
:10EE800000F0A6FD01A9284600F09EFD284600F0EE
:10EE9000F5FD20460A21FFF71FFD3EBD2DE9F04F8D
:10EEA00092468BB0BAF80A30D0F8208052682B2BEB
:10EEB000054640F2B8811378022B40F0B48190F8F7
:10EEC0002610002308E0E8180133D41890F8270032
:10EED000E47E844240F0A781D8B28842F3D35068E0
:10EEE000FFF7F8FCD8F80030984240F09C810021F0
:10EEF0000A229D48F2F790FFBAF80A302B2B40F215
:10EF00009281DAF80430BAF80890C8F808304FF067
:10EF1000000BF02204E04FF0000B4FF06C092C22A4
:10EF2000574609E03F68D21AC3EB090992B21FFAAB
:10EF300089F9002F00F077817B899A42F2D27868B4
:10EF40000390DBE07B89501C984203DA0398831816
:10EF50005B7803E03B680BB15B681B78332938D0E2
:10EF600007D8012919D011D303291DD0062955D15D
:10EF700021E036293DD004D8342931D035294DD16E
:10EF800035E03A293CD03B2948D140E0511E0023CE
:10EF900089B24FF0FF341E4644E0042B40F0438119
:10EFA0001E46114606243DE0032B40F23C811146EB
:10EFB0000724042636E0990740F03581082B34BF3A
:10EFC0001E460826F6B2B342C0F02D811146082431
:10EFD00028E0042B40F027811E461146032421E03F
:10EFE000012B40F020811E46114600241AE0012B1F
:10EFF00007E0042B40F017811E461146022411E061
:10F00000042B40F010811E4611461C460AE0042BDA
:10F0100040F009811E461146052403E011464FF0D9
:10F02000FF340026023113FA81F39BB20193002EC4
:10F030004FD0023292B20AA9059200234B4A41F8FE
:10F04000043D02EB84020491069202930598029912
:10F05000454A43184448A2180792225CC1EB060CAB
:10F060009BB25FFA8CFC002A33D1BCF1030F94BF32
:10F070006246042238460499CDF800C000F0AAFE8A
:10F08000DDF800C0BCF1040F0FD91CF0030F40F0F5
:10F09000CA800799099801220A70FFF719FC029BA0
:10F0A00006990134C8500433CFE704D10998FFF71B
:10F0B00011FC099006E0BCF1010F40F0B4809DF80E
:10F0C00024300993284A294801231355099B40F805
:10F0D00024307B89019999420FD3CA1AC3EB0909DD
:10F0E00092B21FFA89F94A45019203D31E4A137856
:10F0F00063B99FE03F687B680393019A0398815C42
:10F10000FF29F3D04A45FFF41DAFEFE7174B16492F
:10F110001B680022012B0A7000F09380022B3FF441
:10F12000FAAE032B40F0868089E0104A1179052958
:10F1300040D198F80C10012935D12C6ADB78C4F83D
:10F1400028B0C4F82CB00BB1D3682363064B1A79EE
:10F1500012B1064A126901E0226B52085B796263C0
:10F1600033B1024B5B6904E094E20020A0E200208E
:10F17000236BA363A368394A1B69636293791646BC
:10F180002BB1374B9869FFF7A3FB0123A062A37350
:10F19000F37923B1324BD869FFF79AFBE062284636
:10F1A000FFF70AFE3FE0033902293CD82846FFF763
:10F1B00016FE38E0062921D198F80C30052B32D8FC
:10F1C00098F90C304FF0B8429A402CD528462C6A5A
:10F1D00000F06EFC2846234900F0BAFB284621497E
:10F1E00000F0F2FB28461F4900F0F2FB20460C21FC
:10F1F000FFF772FB2846FFF77FFC14E0022912D1CB
:10F2000098F80C1006290ED19B78A8F81AB02C6A31
:10F210004BB19068FFF75CFBA36820621B6928462E
:10F220006362FFF757FD0023C8F80830504600F02E
:10F2300083FC10E0BBF1000F7FF46DAE05E04FF0F2
:10F24000010B4FF0EC096C226AE6044B5A78002A55
:10F250007FF46BAFE7E70BB0BDE8F08F94E20020DE
:10F26000A0E200207845040837B50546002837D0CD
:10F27000046A002C34D0237B082B31D10A68636ADE
:10F280009A422DD120460C21FFF726FB2846214625
:10F290000422FFF785FBF0B9042232212046FFF754
:10F2A00023FB606AFFF716FB01462046FFF743FB8E
:10F2B0002046FFF760FB218B2069F03189B200F016
:10F2C00062FC009560682169064A432303F0D4F884
:10F2D0002046FFF705FC637B0133637314236383CC
:10F2E0003EBD00BF7445040873B5046A0546052198
:10F2F0002046FFF7F1FA284621460322FFF750FB8C
:10F300000646E0B9022220463921FFF7EDFAA98C22
:10F310002046FFF700FB2046FFF72DFB218B2069DD
:10F32000F03189B200F02FFC00956068216904F18A
:10F330002002432303F0A0F82046FFF7D1FB637BB4
:10F340000133DBB2092B637304D84FF4FA625343E1
:10F350009BB201E044F620634FF4FA7203F2F31318
:10F3600093FBF2F3638330467CBD000038B5154B48
:10F37000154D1C6823E0236A03B3DA8B511E012A62
:10F38000D9830BD11A7B0A2A18D893F90C3015FAB5
:10F3900003F313D52046FFF70BFC0FE09A8B511EA9
:10F3A000012A99830AD11A7B0A2A07D893F90C30CB
:10F3B00015FA03F302D52046FFF796FF2468002CC8
:10F3C000D9D138BDDCF600200000204473B5046AB2
:10F3D000054600212046FFF77FFA0023236263627F
:10F3E000A362E362A3636363236328462146072283
:10F3F000FFF7D6FA064698B92046FFF7BCFA218BEC
:10F400002069F03189B200F0BEFB00956068216987
:10F4100004F12002432303F02FF82046FFF760FB9E
:10F42000637B0133DBB2092B637304D84FF47A7228
:10F4300053439BB201E042F210734FF4FA7203F2AD
:10F44000F31393FBF2F36383284600F031FB284665
:10F45000064900F07DFA2846044900F0B5FA28462E
:10F46000024900F0B5FA30467CBD00BF784504087B
:10F4700038B5264B00251C6844E0236A002B40D099
:10F480005A8B012A02D9013A5A833AE039D11A7BC0
:10F490005D830C2A28D0062A00D125E0012A06D156
:10F4A0005B7B052B20461DD8FFF714FC29E0082ABA
:10F4B00009D15B7B012B204602D8FFF77DFC20E0C1
:10F4C000FFF78DFC1DE0052A03D12046FFF70CFF56
:10F4D00017E0042A0AD15B7B082B204602D8FFF7ED
:10F4E00067FB0EE0FFF772FF204608E0032A08D111
:10F4F0005B7B012B204602D8FFF79CFB01E0FFF766
:10F50000FBFA2468002CB8D138BD00BFDCF600201F
:10F5100010B598B190F82D30046A23F0080380F8F4
:10F520002D305CB1606818B103F052F800236360BD
:10F5300020460021BDE81040FFF7CEB910BD000005
:10F5400038B5044608B9F22047E090F82D30056A36
:10F5500023F0080203F02003DBB280F82D20002BFB
:10F56000F1D0838CB3F5107F00D22EE035B93C206A
:10F5700000F038F9054640B3206203E0686808B13E
:10F5800003F026F800213C222846F2F745FC03F060
:10F590003BF86860C8B1037A114943F02003037255
:10F5A0004422686802F018FF0D496868432202F09F
:10F5B000DDFF68680B49224603F006F82046FFF796
:10F5C0009BFA20B12046FFF7A3FFFF2005E094F847
:10F5D0002D3043F0080384F82D3040B238BD00BF11
:10F5E000784504089DEE020808B507F02FFF00F0EB
:10F5F0000FF800F05BF900F0A9F902F027FE00F027
:10F600008BFC05F0E1FDBDE8084002F049BD0000BB
:10F610000B4B0C4A0C4823F0030313604FF4A0512A
:10F6200000225A801A715A1802600120107151800C
:10F63000198006481180064A136007F0E9BE00BF32
:10F64000CBE20020900D0020880D00208C0D0020C2
:10F65000840D002070B5044600284CD0264B1B6852
:10F66000984203D3254B1B68984205D307F008FF47
:10F67000BDE8704007F00EBF214807F0D5FE00231B
:10F6800004F8043C1F4B34F8080C1968A4F1080274
:10F690008A4238BF1A60184B1B6819188A4211D069
:10F6A0000D797DB9154D2D68A9420BD0154D2E68E9
:10F6B0008E42195A08BF2A6024F8081C195A591892
:10F6C000D01A488034F8060C191891420ED00D79E2
:10F6D00065B90C4D2E68964234F8082C08BF296095
:10F6E0001A5234F8082C9A18CB1A53800448BDE8F3
:10F6F000704007F0A5BE70BD900D0020880D002061
:10F700008C0D0020840D00202DE9F04103314FF6CF
:10F71000FC750D400B2D044603D9B5F5A05F01D94A
:10F7200053E00C25DFF8B880D8F800309C4203D3B2
:10F73000284A1268944204D307F0A2FE07F0AAFEFA
:10F7400044E0A4F1080634F8087CF61A083FB6B283
:10F75000BF1BBFB2BD4238D838D01F4807F064FE87
:10F76000D8F8003034F8081C5A18107978B95F5A64
:10F7700006F108016D1819490868ADB2904203EB13
:10F78000050208BF0A60002111715F5310E005F106
:10F790001402BA4215D8114806F10802AD180768DC
:10F7A000ADB25A19BA4238BF0260595300201071E5
:10F7B000568024F8085C5A5BB2F5A05F1CBF9B180A
:10F7C0005D80054807F03CFE00E000242046BDE8CF
:10F7D000F08100BF880D00208C0D0020840D0020DA
:10F7E000900D0020F8B5002856D003304FF6FC7479
:10F7F00004400B2C03D9B4F5A05F01D94BE00C24D5
:10F80000264807F011FE264B1968264B1A688B1AFA
:10F810009BB2C4F5A05E39E0D5182F79002F34D102
:10F82000D65AA6F10800C01AA0422ED304F1140E35
:10F83000704510D308341C19A4B210191653438014
:10F840002C80012307712B71135BB3F5A05F04D0EB
:10F85000D218548001E001232B718D420FD1124B3D
:10F860001A68104B19682B4601E01B88CB181879D1
:10F8700010B90B4A136002E09342F6D1F9E707484A
:10F8800007F0DEFD05F10800F8BD2B887345C3DBEA
:10F89000024807F0D5FD0020F8BD00BF8C0D002008
:10F8A000840D0020900D0020880D00200E4A0F4985
:10F8B000F0B500230E4E0F4F22F003021D4641F813
:10F8C000045B33F806C0002008E051F8044C1460D3
:10F8D000DC5B41F8042C0130121980B26045F4D190
:10F8E0000233202BEBD1F0BD970D0020D4C30020B4
:10F8F0000E4504082E4504080F2838B505460BD8D8
:10F9000007F0BEFD064B53F8254014B1226843F8BA
:10F91000252007F0BFFD00E00024204638BD00BFD1
:10F92000D4C3002038B505460C4659B107F0A8FDF0
:10F93000054B53F82520226043F82540BDE83840A8
:10F9400007F0A8BD38BD00BFD4C300207047000039
:10F9500070B504460D4641B9204604F0B5FD0020BF
:10F96000214604F047FEFDB91FE00A6843689A4249
:10F97000F2D0134B186807E002686368C6689A42C1
:10F9800001D100F089FD30460028F5D10D4B1B68F0
:10F9900007E01A6822B161688A4204BF2A681A60C7
:10F9A000DB68002BF5D1D7E72D682046656004F0B1
:10F9B00049FD00202146BDE8704004F0CFBD00BFE6
:10F9C000E8F60020F0F6002001B10968C160704738
:10F9D00038B504460D460020214604F00BFE05B163
:10F9E0002D6800202146A560BDE8384004F0B6BD72
:10F9F00070B5054616461C46FFF7AAFF2846314655
:10FA0000FFF7E6FF04B12468EC6070BDF8B5069E10
:10FA1000C661104E377880F8307001373770089E15
:10FA20000025044645608560C56080F82D5005625C
:10FA30000661FFF7DDFF2046079B984730B9064B6C
:10FA40001A6822601C6004F0E1FB00E02C462046AE
:10FA5000F8BD00BF14C40020DCF6002010B5044639
:10FA60002146012014B904F0C5FD01E004F076FD43
:10FA7000014B1C6010BD00BFE0F6002010B590F8EF
:10FA80002D30DA07044612D443F0010380F82D30FC
:10FA9000383004F055FB94F82D3003F03003302B50
:10FAA00005D12046211DBDE8104007F09DB810BDCE
:10FAB00010B590F82D30D907044611D523F0010375
:10FAC00080F82D30383004F03BFB94F82D3003F0F3
:10FAD0002003DBB223B12046BDE8104007F054B844
:10FAE00010BD10B521B330B3002905DA4B4242896D
:10FAF0009BB29A4201D21DE08BB2027B44680AB1EC
:10FB0000032A05D1641A00F110039C4212D308E0C5
:10FB1000013A012A0ED800290CDA42899A4209D307
:10FB2000641A43894460CB1843810389C918018151
:10FB3000002010BD012010BD70B5044600B30025A3
:10FB400007F09EFCE689013EB6B2E68107F0A2FC12
:10FB5000BEB9237B2668032B01D10F2003E0013BB4
:10FB6000012B04D80E202146FFF7DCFE02E02046E0
:10FB7000FFF770FD0135EDB23446002EE0D100E014
:10FB80000546284670BD38B50389994220D2CA1A65
:10FB90000D46044605E0ED1A2389D3182381246815
:10FBA000ADB263899D42F6D8227B4AB99D4207D007
:10FBB00063681B1BE918204689B2FFF7A5FD0446C0
:10FBC00020686581258108B1FFF7B6FF0023236017
:10FBD00038BD2DE9F0470D46174603287CD8DFE8ED
:10FBE00000F002080406362604E00E2602E0002695
:10FBF00000E02226032F6FD8DFE807F0465E5E02A2
:10FC00000F20FFF779FE044600B965E0821903363C
:10FC100026F003061332C6F5C066032322F0030262
:10FC20000436AE42A8BF2E46037342600023012271
:10FC3000468103600581C281AE1B0746984640F2AB
:10FC4000036940F2046A1CE00F20FFF755FE0546E9
:10FC500018B92046FFF770FF3EE0032300F11002C1
:10FC60000373B3B2038142604B4588BF5346012200
:10FC7000C0F8008080F80D8038604381C281F61A98
:10FC80000746002EE0DC22E006F11300EB1C23F017
:10FC9000030320F00300C01880B2FFF7A3FD044661
:10FCA000D0B186191336002326F00306466005817D
:10FCB0004581036003730AE00E20FFF71DFE044632
:10FCC00050B1002343600581458103600773012320
:10FCD000E3810023637300E000242046BDE8F08741
:10FCE0000346002002E001301B68C0B2002BFAD1AD
:10FCF000704710B5044640B107F0C2FBE3890133F9
:10FD0000E381BDE8104007F0C5BB10BD10B568B178
:10FD100061B103E004891B190381104602680B8955
:10FD2000002AF7D1028901609B18038110BD10B52C
:10FD30000C46FFF7EBFF2046BDE81040FFF7D9BFA8
:10FD40002DE9F0410C46054608B9F2203FE00029B4
:10FD5000FBD002890B899A42F7D300263746B4F8C4
:10FD60000A806B8961686868C6EB0808DB1B43453D
:10FD7000B4BF1FFA83F81FFA88F8C01989194246E0
:10FD8000F1F790FF46446389B6B2B34247446B89AA
:10FD900098BF2468BFB298BF0026BB4205D12D682A
:10FDA00015B9002CD1D10FE000272CB1628923892D
:10FDB0009A4201D123684BB96A892B899A4201D1B1
:10FDC0002B681BB9002CCAD1204600E0FA2040B2B3
:10FDD000BDE8F0812DE9F8438846164628B331B3D3
:10FDE00000240546A1461CE02BB16A89934202D348
:10FDF0009B1A9BB214E06F896968FF1ABFB2B742C1
:10FE000028BF374608EB0900C9183A463C19B944DF
:10FE1000F61BF1F747FFA4B21FFA89F9B6B2002327
:10FE20002D682EB1002DDFD102E0044600E00C4623
:10FE30002046BDE8F88300002DE9F0474368DFF86D
:10FE400074A093F80990194B06461C680025984643
:10FE500023E0237C4B4518D123681BB1DAF800203E
:10FE6000934212D1676987B1A069114B214632468E
:10FE7000B84750B15DB1E368EB60D8F80030C8F81E
:10FE80000040E3600026012303E0002301E001239A
:10FE90002E46E26825462BB91446002CD9D12046BF
:10FEA000BDE8F0870120BDE8F08700BF18C400203E
:10FEB00008F7002010F700206FF0090070470000DD
:10FEC000134B70B51888134D4FF480424FF6FF74F2
:10FED000A04202D0013080B201E04FF44040002344
:10FEE000595909680BE04E8B864207D1013A92B20C
:10FEF000002AEDD1064B1880104670BDC968002954
:10FF0000F1D10433102BEBD1014B188070BD00BF31
:10FF10001C0700205045040870470000F8B5037E18
:10FF200004460D4633BB1AB9FFF7CAFF024618B3A1
:10FF3000144F0021CB591B680AE0588B904206D120
:10FF40001E68DEB1D5B12868C0B1864216D0DB6824
:10FF5000002BF2D104311029ECD115B12B6803B17B
:10FF60002360094B62831A681C60E26002F0DEF8CD
:10FF7000002004E0FA2002E0FE2000E0F82040B279
:10FF8000F8BD00BF50450408F8F6002038B5037EE0
:10FF900004460BB1002038BD0320FFF7ADFC054639
:10FFA0000028F7D023690361638B43830123037621
:10FFB000637E4376237A43F002030372A37A83724B
:10FFC000637A437223680360638BABB1114A136891
:10FFD000A34201D1E3680CE00F4A136007E0D9683F
:10FFE000A14203D11360E268DA6003E00B46002B04
:10FFF000F5D113600023E36002202146FFF792FC55
:020000040803EF
:10000000064B6B61064B1A681D60EA6002F08EF8C1
:10001000284638BDF8F60020F4F60020B9FE0208A4
:10002000F0F6002030B5016B848DC58E826A0346E0
:1000300040F66830854228BF0546601A8018451B87
:10004000002D01DBDC8530BD501A00284FF0000088
:1000500001DDD88530BD8A1ADA8530BD838DC91897
:1000600089B241F2D063994210B58CBF83858185F6
:100070000446FFF7D7FF40F2B353984208DDA37F51
:10008000204643F00203A377BDE8104001F090BD85
:1000900010BD10B5044648B1406808B1FFF74CFDEB
:1000A00004202146BDE81040FFF73CBC10BD10B550
:1000B00003E00468FFF7EDFF20460028F9D110BDEA
:1000C00001617047C167704781677047C0F8881049
:1000D000704741617047C0F8841080F82020704755
:1000E000037E10B50446BBB10A2B15D0012B13D0EB
:1000F000406F18B1FFF720FD002363674FF6FF73D1
:10010000A386E06EFFF7D3FF206FFFF7D0FF002339
:10011000E3662367A4F86A3010BD00009C4B2DE90C
:10012000F74F1A68DFF8848201321A60994B1A7807
:1001300001321A70C146984BDFF858A21C6800269D
:10014000FFE09AF8003094F821209A4201D1E76844
:10015000F6E0217E84F82130022994F8462001D16E
:10016000062A51D00C2A4FD094F89130C3B18B4954
:1001700094F89020C918013211F8011CD2B29142B2
:1001800084F8902000D93DE00022062B84F89020CE
:1001900002D8013384F89130204601F004FF31E0A9
:1001A000A38E180401D40133A386236F53B3B4F98B
:1001B0003400B4F94430984224DB02290BD0B4F95E
:1001C0004010B4F9423003EBE10375498A5C03FA4D
:1001D00002F3A4F844300023B4F84C10A386B4F81A
:1001E0006030994228BF1946E38E49085A0091426F
:1001F000A4F84E10A4F84C30B8BFA4F84E20204606
:1002000001F040FE002500E00125237E062B0CD1E5
:10021000A27F02F01002D2B23AB15D4A1168626A5E
:100220008A1A282A01D90135EDB2277A07F0080782
:10023000FFB24FB3042B01D0072B24D1544BD4F879
:100240008C001A68636AD21A00F5242303F6B843B7
:100250004FF4FA71B3FBF1F39A4203D90135EDB2D1
:10026000012711E094F892304E4F07FB0300B0FBDA
:10027000F1F18A4207D9204601F076FE94F89230D7
:10028000013384F892300027237E032B08D1404BA2
:100290001A68636AD31A282B0AD90135EDB207E030
:1002A000092B05D13A4B1A68636AD31AF02B00D890
:1002B00045B32046FFF714FFE3680EB1F36001E099
:1002C000354A13604FB1638B0093A38B0193206D6C
:1002D000A16A2246231D01F08FFDD4F88850D4F87E
:1002E00010B0E76802202146FFF71CFB002388F8C6
:1002F00000301DB158466FF00901A84799F8003049
:10030000F3B118E7E37F94F82020E7680133DBB20C
:100310009A42E37713D8D4F88430E57788F8005010
:100320001BB120692146984700E0284699F8003023
:10033000002B7FF400AF10B9204601F039FC2646AF
:100340003C46002C7FF4FDAE174B114E1D681F4636
:100350000FE032686B6AD31AF02B10D80CE0E26021
:1003600000E03A6029460220D5F80C80FFF7DAFA5F
:100370004546002DEDD109E02C46ED68F9E7284609
:10038000FFF7AEFEEA68002CE9D1EAE7BDE8FE8F90
:10039000ECF600201DC40020E8F600206D4504089E
:1003A00060450408F8240100FCF60020E4F6002073
:1003B00003688B4210B50C4602D1CB6803600DE098
:1003C000114A136007E0D968A14203D11360E268C3
:1003D000DA6003E00B46002BF5D113600023E360E5
:1003E0002046FFF77DFE237E0A2B0AD0012B08D082
:1003F000A37FDA0705D543F00203A377204601F077
:10040000D7FB0023237610BDF4F60020037E0A2BD1
:100410002DE9F743044689460AD121461B48FFF7D8
:10042000C7FF0220214603B0BDE8F043FFF77ABAC8
:10043000D0F85080876AD0F8885006691448214661
:10044000FFF7B6FF134B206F01221A7008B1FFF7B8
:100450002EFEE06E08B1FFF72AFEB9F1000F09D0B9
:10046000638B0093A38B4046019339462246231D9C
:1004700001F0C2FC02202146FFF754FA1DB13046BC
:100480006FF00901A84703B0BDE8F083FCF6002037
:10049000E8F60020E4F600200121FFF7B7BF0000D6
:1004A00037B50446002943D0037E042B01D0072B27
:1004B0003ED1636F23B9A28D41F2D0639A4237D007
:1004C000638B206D0093A38BA16A01932246231DA9
:1004D00001F092FC2046FFF703FE424A1368A34254
:1004E00001D1E3680CE0404A136007E0D968A142FB
:1004F00003D11360E268DA6003E00B46002BF5D10C
:1005000013603A4B01221A70237E0025042BE5600C
:1005100008D10A232376364B1A681C60E26001F08A
:1005200005FE03E002202146FFF7FCF9284651E0D2
:10053000237E072B53D8DFE803F0041E27353C52F7
:100540005244638BABB12B4A1368A34201D1E368D9
:100550000CE0254A136007E0D968A14203D113607B
:10056000E268DA6003E00B46002BF5D1136000234C
:10057000E360022004E020482146FFF719FF032032
:100580002146FFF7CFF92AE021461648FFF710FF72
:10059000164B0122022021461A70FFF7C3F904F01E
:1005A000AFF81CE0204601F0BEFA98B904F0A8F8B4
:1005B00005E0204601F0B7FA60B904F0A9F8052378
:1005C00006E0204601F0AFFA20B904F0A1F80923B3
:1005D000237601E040B204E0204601F0E9FA002071
:1005E000F8E73EBDE8F60020F4F60020E4F600202F
:1005F000FCF60020F8F60020F0F60020037E012B28
:1006000003D0837F43F0100383770121FFF748BFB6
:1006100010B50846144632B11189FFF71FFD204678
:10062000FFF78AFA04E01BB9BDE81040FFF7E6BF08
:10063000002010BDF8B5456FC66F6F7B00230446E0
:10064000436726B121462A460069B04705E0304697
:1006500021462A463346FFF7DBFFB0B907F02007F3
:10066000FFB2BFB1A38D41F2D062934201D00133FA
:10067000A385E56F05B90CE00022206921461346E9
:10068000A8470A3005D1F62004E040B20A30FAD07B
:100690006567002040B2F8BD2DE9F843184B194FAB
:1006A0001A7801321A7098463C68174D002622E0ED
:1006B00098F8002094F82130934220D084F821202B
:1006C000A27FD10709D542F00202A277204601F0AD
:1006D0006FFAA37F23F00303A377636FD4F80C9022
:1006E0000BB94C4607E020462E70FFF7A3FF2B788E
:1006F000002BD9D1F5E7002CDAD1BDE8F883FEE76D
:100700001DC40020E8F60020E4F6002008B5FFF73D
:10071000C3FF064A13780133DBB2D807137003D541
:10072000BDE80840FFF7FABC08BD00BF1CC40020AC
:10073000034B044A10681A6880181860704700BF9D
:1007400018070020ECF60020F8B505460220FFF758
:10075000D3F80446002836D1394B3A4A1B68116851
:1007600007E05A6A8A1AA24234BF22461846DB685A
:100770001446002BF5D108B1FFF78EFE0220FFF7DB
:10078000BBF80446F8B92F4A2F4B17681B687F2027
:1007900022460CE0597EA94208D8814206D85E6AFA
:1007A000BE1BA64202D3084634461A46DB68002B1D
:1007B000F0D112B11046FFF76FFE0220FFF79CF850
:1007C0000446002839D0002194222046F1F724FB6A
:1007D00041F2D06246F2A863A4F86630A2850023F5
:1007E000E285FF226576A4F868301D466372A27226
:1007F000A4F840304FF406724FF6FF73E286A386EA
:1008000006220123A4F84C30A4F84420A4F8422086
:10081000FFF78EFF0B4BA0651B68206563620B4BD7
:10082000A0641B78E06584F82130094BE577E36725
:10083000084B84F89250C4F88C302046F8BD00BFB5
:10084000FCF60020ECF60020E8F600201DC4002095
:100850001106030800DD6D004020FFF775BF10B5DD
:100860000446084602F0F2F830B1838C23B1283BED
:100870009BB29C4228BF1C46204610BDF8B51E4DB9
:100880002C680646A089FEF71EF8C0F30F30052835
:1008900031D92B689889FEF716F8000B411F8900A3
:1008A000143489B2002340F2B35040F2B45520E032
:1008B000E25C012A05D01ED3022A04EB030214D104
:1008C00001E0013314E05778042F14D1DF1C8F426C
:1008D00011DA9778D27842EA0722571EBFB28742D0
:1008E00088BF2A46F286043302E052781AB1D31840
:1008F0009BB28B42DCD3F8BD20C400202DE9F0412F
:10090000A04B1B7803F01003DBB20446002B00F071
:100910006B819D4A436D1268B0F86050816D981AE2
:1009200000280EDB9342994B03D11868081A00285F
:1009300007DB1B6899421FD1954B1B68DB89AB42D3
:100940001AD9934BB4F862601B68D88962658F4AE4
:10095000A4F8600012688642A26538BFA4F862005D
:1009600094F8912020B93AB984F89000012301E06D
:1009700012B1002384F89130844BA26C1B68981A42
:10098000002834DC0020A4F8640082480088002895
:1009900040F0F481B4F86060A06D691830188842A6
:1009A00040F0EC81B4F934100029C0F2E7819A429A
:1009B00040F0E48194F84720531CDBB2934288BF97
:1009C00084F8473094F84730032B0AD9B4F84C2008
:1009D000E38ED3189BB2934240F2B280A4F84C301D
:1009E000AEE040F0AD80204601F092FAA8E0D1439D
:1009F000D9427ED4216D591A00297ADCA17F01F0F9
:100A00000400C0B230B121F00401A177B4F84E1057
:100A1000A4F84C10B4F94050B4F84200A36400EBC1
:100A2000E5009A1AA4F84400237EB4F86600A4F8FE
:100A3000642000211218032B84F84610A4F86620C5
:100A400084F8471031D9B4F84E20B4F84C309A42AB
:100A5000E28E00D902E0524392FBF3F29A1892B26E
:100A60009A4222D9A4F84C201FE0256F2B686868B1
:100A70002367FFF735F9B4F8643053B1EB68988910
:100A8000FDF721FFC30704D5B4F86430013BA4F897
:100A900064306868B4F86870FFF722F9381AA4F86F
:100AA00068002846FFF7F5FA00E0384E236F1BB9BF
:100AB000226F0023D2B915E0DB685868FDF70AFF02
:100AC000236F1D89DB6807469889FDF7FCFE3368B4
:100AD00010F0030018BF0120FB1A28181B18002B68
:100AE000C3DDE5E74FF6FF72A28600E0A386E37759
:100AF00026E00023A4F8643022E0E56E2B68E3666C
:100B00000BB9A4F86A306868FFF7EAF8B4F8643003
:100B100053B1EB689889FDF7D6FEC70704D5B4F842
:100B20006430013BA4F864306868B4F86870FFF77B
:100B3000D7F8381AA4F868002846FFF7AAFA00E0A8
:100B4000124EE36E13B9A36B33BB4DE0DB6835681F
:100B50005868FDF7BFFEE36E1F89DB688046988901
:100B6000FDF7B1FE10F0030018BF0120C8EB05052A
:100B700038182D1A002DE6DB3268236DD31A002BAE
:100B8000BBDDE0E730C4002024C400202CC40020DA
:100B900020C4002028C400207B49E26B0968521A57
:100BA000002A21DA794AB4F84010126841F3CC00E7
:100BB000D21A121A92B293B2511889B21804A4F838
:100BC000401001D553429BB2B4F8422042F38D004D
:100BD000121AD3189BB241F3CC01A4F842305B182F
:100BE000A4F844300023A363694B6A4A188800289C
:100BF00000F0B380237E062B00F2AF801168A36A59
:100C0000CA43DA4225D45A1C521A101A002820DC92
:100C1000591A614B586843898B420ADA02890025C8
:100C2000521A03E0028145810068C91A43898B4248
:100C3000F8DB494209B2FEF754FF574A5549158976
:100C40000868A36A4019C01A1081D2680B6053600B
:100C500006E0C91A002903DAA37F43F00203A37751
:100C60004C4BA26A1B68991A002971DB591CA08D94
:100C7000891A091A00296BDC9A4269D1464DEB6842
:100C80002E899889FDF71FFE10F0030018BF012080
:100C90003F4B301880B21880A38D834230D2EB686E
:100CA0009889FDF710FEC0070CD5ED68AE89304677
:100CB000FDF709FE00F03E00FDF700FE26F47C562D
:100CC0003043A881A38D344D2B81EB689889FDF7C3
:100CD000FAFD00F0020080B210B12B89013B2B819C
:100CE00068682989FEF74FFFEB682E899889FDF720
:100CF000EAFD10F0030018BF0120254B30181880C2
:100D0000234B244A1B8812689A18A262A28DD31A18
:100D1000A3852046FFF786F91F4B5A68118919B140
:100D20001E490A6000225A60DB689889FDF7CBFDF6
:100D3000C10704D51A4B1A7842F020021A70A37F1B
:100D4000DA0702D523F0010313E043F0010312E0B8
:100D50002046BDE8F04100F009BF1268A36AD11A2D
:100D6000002905DB0132A18DD31A5B1A002B09DDA6
:100D7000A37F43F00203A377BDE8F081002384F84A
:100D80004730DDE6BDE8F0812CC40020ECF6002001
:100D900028C4002024C400203CC4002034C4002007
:100DA00031C400202DE9F74F06460F4603F0B8FC8A
:100DB0007368A74AA74C13601A7802F00F029100DB
:100DC00003EB8203304649422360FEF78AFE002887
:100DD00040F0CE833389132B40F2CA839E4D3946AF
:100DE000286801F043FD002840F0C2832B6803F01F
:100DF000F003E02B00F0BC8323689889FDF763FDC6
:100E00006FF00301C0F3073359433046FEF769FE24
:100E10008346002840F0AC8327683888FDF753FDEF
:100E2000388027687888FDF74EFD788027687868D5
:100E3000FDF750FD894B786027681860B868FDF7AA
:100E400049FD874BB86027681860F889FDF73BFDBE
:100E5000F88123689889FDF736FD824BB6F8088043
:100E6000276810F0030C00F03F0118BF4FF0010C91
:100E70001970C4447C4B29681FFA8CFCA3F800C08D
:100E80007A4BD3F800A07A4B0246D3F80090544630
:100E9000584619E0A58B3B889D4213D1658B7B8812
:100EA0009D420FD163684B450CD123688B4209D119
:100EB000002800F08283E368C3606C4BC4F80CA088
:100EC0001C607AE32046E468002CE3D172E3988B3F
:100ED0003C88844230D1588B7D8885422CD158681B
:100EE000484529D11868884226D102F00401C9B2C8
:100EF000002940F03F8302F00201C9B259B1574ABC
:100F000011689A6A8A1A0BD4988D121A002A07DC83
:100F10000095019441E0D20702D5564A12685A6200
:100F2000BCF1000F00F026839A7F42F002029A770C
:100F3000184600F03DFE1DE3DB68002BC7D14E488C
:100F4000046825460FE0688BB7F80280804508D119
:100F5000D5F80080884500F04283B8F1000F00F01A
:100F60003E832B46ED68002DEDD13CE3E968D96066
:100F7000414BEC601D6002F00403DBB2002B40F03B
:100F8000F98202F010085FFA88F8B8F1000F0CD06F
:100F9000324B196800903B880193314B18686144CB
:100FA0002D4A334B00F028FFE4E202F00202D2B2F5
:100FB000002A00F0DF82687EFFF7C6FB04460028A7
:100FC00000F0D882244B1B6803606B8B4383284B53
:100FD0001B6843601F4B1B6859781A7842EA01224C
:100FE0008283032202761D4A1268511C81620163CA
:100FF000DB89A0F86030A0F86230A0F84E302B6991
:1010000003616B69013A426543612B7A23F07303F4
:101010000372164B1A681860C26001F087F8174B0C
:10102000012220461A70FFF729FC211DE08EFFF7F0
:1010300016FCE08603F05CFB2046122100F028FD40
:1010400020B120464146FFF7E1F993E2204670E7E0
:1010500038C4002020C4002010F7002024C4002041
:101060002CC4002030C4002028C40020E8F6002052
:1010700008F70020ECF60020F0F60020E4F600204F
:10108000737B43F001037373636F63B12046FFF713
:10109000D1FA0A3004D0636F2BB19F4B1B8813B178
:1010A00003F056FB49E29D4B1C609D4B1B7803F0FF
:1010B0000402D2B2AAB1237E022B06D1994B1A6840
:1010C000236D9A4240F0A18296E2974B1A68A36A78
:1010D000D31A00F19A82A18D5B1A002B00F395823E
:1010E0008AE203F00203DBB223B1237E023B012B31
:1010F00000D96BE0A37F03F01003DBB213B98B4B75
:101100001B686362002384F892302046FFF7B6FB29
:10111000237E023B072B00F27882DFE813F0080001
:101120007700C900DA003001C900520186017C4B0A
:101130001B7803F01203122B53D1236F794DDB6818
:101140002E685868FDF7C6FB0130864249D1B4F8D5
:101150006630E08E0133A4F86630734B1B685A1C6E
:10116000A26222632A68A264714A1268013BD28992
:10117000636504232376E118A4F86020A4F86220B4
:10118000FFF76DFB0A234343A4F84E30B4F84C300C
:10119000E086012B01D1400080B2B4F86830A4F899
:1011A0004C00206F013BA4F8683003682367FEF70A
:1011B00070FF236F1BB94FF6FF73A38603E0002374
:1011C000A38684F84630D4F880301BB9A37F43F05F
:1011D000020319E200222069214698470A30F5D11E
:1011E000ABE14F4B1B7803F01003DBB2002B00F098
:1011F0000C824F4B484A1B68118858884A4A12682B
:1012000000901B880193474B18683AE0444B1B78C9
:1012100003F01002D2B2002A39D0424B1868A36CF6
:10122000DB43C34223D4236DC31A002B1FDC0423EA
:101230002376636903B947E1206921460022984774
:1012400018B10A3040F0408177E12046B4F84C50A4
:10125000FFF754FBB4F8643013B1013BA4F86430D9
:10126000E38E012D08BF5B00A4F84C3023E0304B27
:10127000294A1B6811885D882B4A126800951B88D3
:10128000019389182B4B2C4A00F0B6FDBDE103F009
:101290000203DBB2002B00F0B881234AA36A126874
:1012A000013B9A4240F0B181204600F003FEACE1E0
:1012B0002046FFF723FB214B1B7803F02003DBB212
:1012C000002B00F0A281A37F43F00203A377072342
:1012D00053E02046FFF712FB184B1A78104B1B788F
:1012E00002F0200203F01003D2B2DBB2002A3AD09F
:1012F000002B32D00B4B1A68236D9A422DD1A37F5D
:1013000043F00203A3772046FEF7EAFE0C4A136877
:10131000A34217D16DE000BF28C4002000F70020D1
:1013200030C400202CC4002024C40020ECF600208F
:1013300020C4002008F7002010F7002031C400204E
:10134000E8F600208E4A136004E0D968A14200D17B
:1013500057E00B46002BF8D15AE0A37F43F002037D
:10136000A377082309E0002B00F04F81854B1A6812
:10137000236D9A4240F049810623237645E12046B9
:10138000FFF7BCFA804B1B7803F02003DBB2002B85
:1013900000F03B81A37F43F00203A3772046FEF7D2
:1013A0009FFE7A4A1368A34200D122E0744A136078
:1013B00004E0D968A14200D123E00B46002BF8D10C
:1013C00026E02046FFF79AFA714B1B7803F01003D2
:1013D000DBB2002B00F019816A4B1A68236D9A4228
:1013E00040F013812046FEF77BFE684A1368A34253
:1013F00001D1E3680CE0624A136007E0D968A142BA
:1014000003D11360E268DA6003E00B46002BF5D1EC
:101410001360604B01221A700A2323765E4B1A6810
:101420001C60E26000F082FEEFE02046FFF766FA03
:10143000574B1B7803F01003DBB2002B00F0E58064
:10144000504B1A68236D9A4240F0DF804E4B1A7859
:1014500042F010021A70D8E0D4F888309BB12069AD
:101460006FF00A010EE003F01003DBB2A3B1A37F1B
:1014700003F01003DBB233B9D4F888301BB1206914
:101480006FF00B01984721464048FEF791FF02207C
:101490002146FEF747FA50E0B4F864201AB93F4BF2
:1014A0001A684AB926E0A36F002BF8D020692146BC
:1014B00098470A30F3D140E0A37F03F01003DBB27A
:1014C00033B11046FEF738FB2046FEF7E5FF34E067
:1014D000E56F1DB120692146A84704E02846214652
:1014E0002B46FFF795F843B20A3326D010B12B4BA9
:1014F0001B686367244B1B7803F02003DBB2B3B196
:10150000636F23B15A7B42F020025A730FE0A38D20
:1015100041F2D062934201D00133A385E56F35B12A
:101520000022206921461346A8470A3005D01C4BEB
:10153000002220461A6000F03BFB194B194D002495
:101540001C606868154B1C60002867D0FEF7F4FA31
:101550006C6063E0144B154A1B6811885888144A64
:10156000126800901B880193064B8918186817E5CC
:1015700003F0EEF8304603B0BDE8F04FFEF7DCBAFA
:10158000F4F600202CC4002031C40020E8F600202E
:1015900030C40020E4F60020FCF6002034C4002013
:1015A00000F700203CC4002020C4002028C40020F4
:1015B00024C400201B4B1B68BFE41B4B0021196097
:1015C000A3F808805E60DF60184B02F00802196023
:1015D000174BD2B21970002A7FF452AD54E5002B9C
:1015E0007FF4C4ACC7E4B889FDF76DF900F00400DE
:1015F00080B20028BED1ADE70D4B1A7842F0080248
:101600001A70A37F23F00103A377094B1B7803F023
:101610000802D2B2002A7FF41FAF24E703B0BDE86E
:10162000F08F00BFFCF600203CC4002034C4002032
:1016300031C4002070B591420C461E46049D1AD25A
:101640009DF8143003F00203DBB25BB9AB7F03F00B
:101650004003DBB27BB99DF818301BB1E96E09B9C4
:101660002B6F43B104F2B75121F003019142A8BF9F
:10167000114689B200E021460022FEF7AAFA20B105
:1016800043891B1B33800481448170BD2DE9F047E1
:101690009DF8206006F0020716F0010FFFB28046A9
:1016A0009A460CBF00230423002F14BF0C270027E9
:1016B00004200D469146FF18FEF71EF9044618B99E
:1016C0002846FEF739FA30E086722B894560DB1B2D
:1016D00000260660038114212846FEF702FA05461B
:1016E00020B12046FEF7D5FC34461EE06368B8F80A
:1016F0001A005E68E660FDF7E1F83080B8F81C007B
:10170000E668FDF7DBF870805046E668FDF7E0F824
:10171000BF02706007F5A04040EA0900E668FDF7E7
:10172000CDF8B081E3689D74DD742046BDE8F08794
:101730001431F8B589B20546174601200022FEF79C
:1017400048FA0646F8B14468688BFDF7B7F8208080
:10175000A88BFDF7B3F867606080A86AFDF7B8F85A
:10176000A06045F21000FDF7A9F8A081E88DFDF713
:10177000A5F80023E08123746374A374E374EA8DF5
:10178000AB6AD3182B633046F8BD2DE9F04F8FB00C
:10179000914607930023ADF836300446B0F8622036
:1017A000C38E0691002900F06881017E072900F2AE
:1017B000668190F918104FF06450884040F15F81C5
:1017C000B9F1000F0DD0B4F86610494500D203E01E
:1017D000B4F86810472904D9A37F63F07F03A37787
:1017E00051E15208E66EB4F868B09A4228BF1A4632
:1017F0000A920EB966E01E463368002BFBD1B37A1D
:1018000037890A98B4F86A5013F0010F03F0020305
:101810000CBF00210421DBB2C21B002B14BF0C2320
:101820000023521AD21A92B21DB9ADF836502B4687
:101830000AE0A94534BF4B462B46ED1AD21AADF843
:10184000365092B21D4633464D453FD2002A3DD018
:10185000002F3ED00799C5EB090A9245A8BF9246D2
:10186000CB071FFA8AF814D5012301910293009443
:10187000032041460DF13603FFF7DCFE0746002842
:1018800000F0E980069A406851194246F0F70AFADA
:101890000BE0032041460122FEF79BF90746002892
:1018A00000F0D980069843197B603846FEF718FA95
:1018B000A8441FFA88F85844AA461FFA80FB4546F8
:1018C000334607E0B2463546334600E0AA460027D5
:1018D00000E0AA4607994FF0000801F00101CDF899
:1018E0002C80089168E0C5EB09030A9A9BB29342E9
:1018F00038BF1A46089B0992DBB1D8F1010307985B
:10190000009438BF002301900293114600200A9AE8
:101910000DF13603FFF78EFE8446002800F09E800E
:10192000069A4068CDF814C05119099AF0F7BAF92F
:1019300019E0089809990122FEF74BF9034600289F
:1019400000F08C800698421908985A6001460246B9
:101950000593FEF73EF9059B08B9184613E01946B2
:101960000590FEF7D3F9DDF814C06046CDF814C039
:10197000FEF7B6F958441FFA80FBBBF1480FDDF8BB
:1019800014C003D96046FEF7D7F867E0E36D002284
:10199000EB18009220466146FFF778FE03460028C8
:1019A0005CD0B8F1000F02D00B99086000E08046CF
:1019B000099A0B935519ADB24D4594D3BAF1000F66
:1019C00019D0756811E02A8952442A812A685AB9C7
:1019D0006A6868890699059310185246F0F762F90B
:1019E0006A89059B52446A812D68002DEBD13289AA
:1019F0009244A6F808A0BDF83620A4F86A2057B192
:101A0000706805933946FEF781F939893289059B5B
:101A10008A18328103E016B9C4F86C8001E0C6F878
:101A20000080E26DA4F868B04A44E265B4F866202C
:101A3000C9EB0209A4F8669033B3DC680CB3079BCA
:101A400003F00205EDB2E5B90820A689FCF736FFE0
:101A50003043A08115E04FF000084746A37F63F0B4
:101A60007F03A37717B13846FEF766F8B8F1000F89
:101A700009D04046FEF71BFB05E0F22304E0F32308
:101A800002E0002300E0FF2358B20FB0BDE8F08F62
:101A9000B0F86830472B73B504460D4600D914E002
:101AA000B0F86630C1F34006B100002B38D00020FA
:101AB0000246FEF78EF8014600B906E00096204681
:101AC0002A46E36DFFF7E2FD20B9A37F63F07F03B1
:101AD000A37725E0E36E13B9E06604E013461A68C5
:101AE000002AFBD118600023A907A4F86A3007D0A8
:101AF000E36D0133E365B4F86630013BA4F866306A
:101B0000EA0703D5A37F43F02003A3774068B4F826
:101B10006850FEF7E5F84019A4F86800002000E0DE
:101B2000FF2040B27CBDF8B5C46E05460CB90AE092
:101B30001C462368002BFBD1E3689889FCF7C3FEA1
:101B400010F0070605D028460121BDE8F840FFF750
:101B50009FBFE4680120A789FCF7B0FE3843A0814D
:101B6000AB7F43F02003AB773046F8BD37B5044672
:101B7000006DFCF7ADFE002102462046FFF7D8FDC0
:101B8000054688B1A37F627A23F003030092062200
:101B9000A3770192A37A2146221D01F0ABF82846D3
:101BA000FDF7CAFF002000E0FE2040B23EBD00006D
:101BB0008F4B1B6883422DE9F74F044600F01381D9
:101BC000B0F84C30B0F86090C56E994528BF994682
:101BD000837F03F00203DBB283B12DB9204603B04B
:101BE000BDE8F04FFFF7C2BFEB685868FCF772FE24
:101BF0002A89A36CD31A18184845EFD8266F0EB956
:101C0000D1E01E463368002BFBD1CCE0EB6898890D
:101C1000FCF759FE236F9BB1A27F12F0440F0FD146
:101C2000E36E2BB1196859B91989E38E994207D22D
:101C3000B4F8663023B1B4F86830472B40F2CE8058
:101C40002B68E366237E022B0CD0EF681020B7F8D8
:101C50000CB0FCF733FE40EA0B00B881A37F23F001
:101C60000303A37702F064FDA06AEF68FCF730FE7F
